:020000040800F2
:10000000F0FF0120D1780408C5230308E17102083C
:100010004579040845790408457904080000000082
:10002000000000000000000000000000D1230308D1
:10003000CD23030800000000C9230308D9400208AB
:100040004579040845790408457904084579040888
:100050004579040845790408498002087581020839
:1000600039810208FD800208C180020875C00008BD
:1000700065C0000855C0000845C0000831C0000830
:100080001DC0000809C000084579040800000000F0
:100090000000000000000000000000008580020851
:1000A000D9240208C52802084579040885290208D0
:1000B000052802084527020879260208D5E4000829
:1000C000DDE40008C5E40008CDE400084579040833
:1000D00045790408B54102081941020800000000F2
:1000E0000D80020845790408CD6703080000000070
:1000F000000000000000000000000000F5BF000844
:100100000000000045790408A92502084579040883
:1001100000000000000000000000000000000000DF
:10012000E1BF0008CDBF0008B9BF0008A5BF0008A7
:1001300091BF000800000000000000000000000067
:10014000000000000000000000000000B9310308BA
:100150007DBF000869BF000855BF00084579040845
:10016000B5E40008BDE40008000000000000000045
:10017000000000000000000000000000000000007F
:1001800000000000457904080000000000000000A5
:080190004579040845790408D3
:0801980068740400010000007E
:1001A00010020100802B00207C2B002000000000AA
:1001B000F0060008180202005036002038370020F0
:1001C000000000000000000017020B004536002070
:1001D0003C370020000000002984000807020200CC
:1001E000F43600204837002000000000F206000826
:1001F00002000C00CC3600204C370020000000002C
:100200000000000006020C00C03600205837002015
:1002100000000000C9920008081209003C360020C6
:1002200064370020000000006D840008F70106001C
:10023000363600207037002000000000F406000869
:100240000A020A00B83100207837002000000000C0
:10025000FA06000803000100B82C002084370020B3
:10026000000000000000000003123300443E0020A4
:100270001846002000000000040700082500960032
:10028000CC44002062450020000000000000000077
:10029000F6210C0098420020484400200000000095
:1002A000380700081500700068430020D84300207C
:1002B00000000000000000002A006000A8420020AA
:1002C00008430020000000004DF803082C00100037
:1002D000F84500200846002000000000E9960108CB
:1002E0002B0024006F4600204B4600200000000039
:1002F000B996010829107800A84100205444002034
:100300000000000000000000140003006040002016
:10031000A442002000000000440700081010020062
:10032000DC3E0020D84600200000000048070008FE
:1003300028101000CC3E0020DC4600200000000009
:10034000257B010823001000783B0020EC460020AC
:10035000000000003D7B0108F8210600C23C00209F
:10036000FC460020000000004A0700081A023C007A
:1003700000480020004C0020000000009D91000873
:1003800027000400FC4700203C4C00200000000037
:10039000500700080E5020013C5D0020B86400208A
:1003A0000000000075F80308130004003C62002000
:1003B000D865002000000000540700080101040077
:1003C000B65C0020DC65002000000000000000009A
:1003D00000010400AE5C0020E06500200000000089
:1003E0005807000802010300A95C0020E465002012
:1003F00000000000C9EE000809020100606400204E
:10040000E8650020000000005C0700080C106C008C
:10041000865E0020EC65002000000000A1EE0008D0
:1004200001020500BE5C00205866002000000000AC
:100430001192020800020500D061002060660020D1
:1004400000000000000000001B020800AC6100205A
:100450006866002000000000A18400080120080058
:100460002063002070660020000000005E07000886
:1004700019000500D063002078660020000000000D
:100480006607000837001E00A86300208066002071
:10049000000000006C0700081E0005008C5F0020B3
:1004A000A0660020000000008A0700081B00F4007E
:1004B000484C0020A866002000000000EDA20208C1
:1004C0000E020200B86200209C67002000000000BD
:1004D000900700082F00110098640020A0670020FA
:1004E000000000009207000805100600B87D0020FB
:1004F000A882002000000000A4070008F531700069
:10050000187D0020B082002000000000599C0208E5
:1005100026000E0030830020208300200000000011
:10052000E11603080B2010001C7B002064830020D0
:1005300000000000AA0700081F201C006C720020A9
:100540007483002000000000BA07000805020400C0
:10055000E07C00209083002000000000D607000807
:1005600003010A00D47A00209483002000000000D8
:10057000DA07000813020300E0700020A0830020C7
:1005800000000000E4070008160008009484002022
:100590009C84002000000000E807000804008000A0
:1005A000E8B90020A0BA0020000000000000000010
:1005B0000D002C005CB8002020BB002000000000D3
:1005C00055680308F9010400ACAF00204CBB0020C3
:1005D00000000000A1100208FD01240088AF0020E7
:1005E00050BB0020000000002910020818202C0039
:1005F00058AF002074BB0020000000006592000886
:1006000006101800A4A20020A0BB002000000000DB
:10061000D1F80308FB010100DCA10020B8BB0020D9
:100620000000000039920008FC010900A8A0002089
:10063000BCBB002000000000499200080A402000D6
:1006400070A00020C8BB002000000000F0070008D8
:100650003400100018990020E8BB002000000000C2
:10066000A5F8030811020800F0980020F8BB00204C
:10067000000000001008000812120400E898002092
:1006800000BC0020000000001808000812200D0027
:10069000D898002004BC0020000000001C080008BE
:1006A00002020300F484002014BC002000000000BB
:1006B000000000000C020300B084002018BC0020E1
:1006C0000000000019840008FE01090020870020B6
:1006D0001CBC0020000000008D8400081A000E00E1
:1006E0000CC00020B4C10020000000002A0800084F
:1006F0000000013C22010000000000004A01B4009B
:10070000D601000000000000000000000000000012
:1007100000000000000000000000000000000000D9
:1007200000000000000000000000000000000000C9
:1007300000000000000001000000000001000000B7
:10074000020200000300000000050401F40119008A
:100750002003000048040430900100000000E8037A
:100760006400040A0001000028010000200032009B
:10077000C800D0079600140032002800B0044006DC
:100780000005500014000F000801000001000000E7
:100790000000000000000000000000000000000059
:1007A000000000002000030100002B21231E640133
:1007B0000100000001000A01290000000000000102
:1007C000000000050000010203000000000000001E
:1007D00000000000000000000000040101006C1691
:1007E0000000000000000000C409000019012828D2
:1007F000003001000000000064002C010000000037
:10080000000000000000020000019E077D0046324B
:100810000000000001010101FFFFFFFF00000001D7
:100820000000054D4B34310000007E05EA05B4059B
:080830003200E803D0070000CC
:100838000100000080010000080000000400000022
:100848000000000000000000010203040607080978
:10085800010000000000803F0000000000000000D0
:1008680000000000FF000000000000002837002002
:1008780008000000000000001837002008000000F1
:100888004098040805080400000000007CC1040822
:1008980044C2040868C10408000000000000000009
:1008A8006C98040805080A00000000007CC10408D0
:1008B80044C2040848C0040800000000000000000A
:1008C800D6010100000101010001FFFFFFFFFFFF4A
:1008D80001000000685E0C00010102FFFF0000003B
:1008E80000000100E001010101000000E995020893
:1008F8000000000030020020981A050800000000DF
:10090800000000000000000000000000FC0F0508C7
:100918000000000000000000C602002004000000E3
:10092800441A05080D00000079C10208981C00202F
:1009380000000000A81305080D000000A1C102086E
:100948008C1C00200000000010150508080000009D
:1009580000000000801C002004000000141405089A
:100968000D0000009D960208741C00200000000085
:10097800C41405080300000075C40208681C0020A0
:1009880000000000A81A05080300000075C402084A
:100998005C1C002000000000441005080100000055
:1009A800000000000000000000000000000000003F
:1009B8000E00000000000000000000000000000021
:1009C800981A050800000000000000000000000060
:1009D80000000000FC0F05080000000000000000F7
:1009E800C602002004000000F019050803000000FA
:1009F800499D0208501C0020080000001414050836
:100A08000D0000009D960208741C002000000000E4
:100A1800C41405080300000075C40208681C0020FF
:100A280000000000A81A05080300000075C40208A9
:100A38005C1C0020000000004410050801000000B4
:100A4800000000000000000000000000000000009E
:100A58000E00000000000000000000000000000080
:100A6800B01A0508000000000000000000000000A7
:100A780000000000FC0F0508000000000000000056
:100A8800C602002004000000F81905080300000051
:100A980075C40208A41C00200000000044100508CA
:100AA800010000000000000000000000000000003D
:100AB800000000000E000000000000000000000020
:100AC8000000000020700020702D7200FFFFFFFF63
:100AD800010000000000803F080000000000000046
:100AE800000000000C180020FA00000001000000BF
:100AF80001000000FFFF2D202D2D202D2D2D2D2054
:100B08002D2D2D0000000000000000000000000056
:100B180000000000000000000000803F0000803F4F
:100B2800FFFFFFFF18100508201005083C100508F6
:100B380000000000000000000000000000000000AD
:100B4800E90D05080400000041BF0208000000008C
:100B5800000000004410050801000000000000002B
:100B68000000000000000000000000000E0000006F
:100B780000000000000000000000000088BA00200B
:100B88000100C4090000000086BA00200100C40961
:100B98000000000084BA00200100C4090000000021
:100BA80082BA00200100C409000000007EBA0020BB
:100BB8000100C4090000000080BA00200100C40937
:100BC800000000007CBA00200100C40900000000F9
:100BD8007ABA00200100C40900000000D05C00209F
:100BE8000100C80001000000CE5C00203200307512
:100BF80032000000CC5C0020055A0500C95C0020CA
:100C080000FF0100CB5C002001000000F40200207E
:100C1800C75C00200200000070C20408C85C002005
:100C280000FF0100CA5C002001000000F40200205F
:100C3800C65C00200200000070C20408BC5C0020F2
:100C480080C1803E05000000BA5C002080C1803E63
:100C580005000000B45C002080C1803E0500000053
:100C6800B25C002080C1803E05000000AC5C002022
:100C780000FF0100A85C00200A320100A75C0020E8
:100C88000400000028C00408A65C00200200000040
:100C98003CC004080000000000000000FC02002026
:100CA8008C7C00209CFF2C0100000000B600002076
:100CB8000A00000048C004089C5C0020E0150C17DE
:100CC80000000000B80000200800000044C204082A
:100CD800B7000020050000007CC104089E5C0020CD
:100CE8000200000060C004080C5F00200100FF7FC4
:100CF800010000000B5F0020020000006CC0040827
:100D08002F5D0020030000007CC004082E5D002039
:100D1800030000007CC00408665E00200000F401A7
:100D280001000000645E00200000F40101000000E2
:100D3800625E00200000F40101000000605E0020F7
:100D48000000F401010000005E5E00200000803E0B
:100D5800010000005C5E00200000803E01000000F1
:100D6800825E0020E803D0070A000000805E0020B1
:100D7800006401000A000000755E002000640100A4
:100D8800745E0020006401007C5E002000640100A5
:100D98000A0000007B5E0020006401000A000000D9
:100DA8007A5E0020006401000A0000007F5E0020D7
:100DB800006401000A0000007E5E0020006401005B
:100DC8000A0000007D5E0020006401000A000000A7
:100DD800795E002000FF01000A000000785E002014
:100DE80000FF01000A000000775E002000FF0100FC
:100DF8000A000000385D00200000F4010100000036
:100E0800365D00200000F40101000000345D002080
:100E18000000F40101000000325D00200000F40130
:100E280001000000305D00200000F4010100000016
:100E3800725E002000640100705E00201400E80368
:100E4800010000006E5E0020E80330750A00000013
:100E58006C5E002000C801006B5E002000C8010025
:100E68006A5E002000C80100695E0020006401007D
:100E78000A000000005F00200000D0070100000009
:100E8800FB5E002000C80100FA5E002000C80100D7
:100E9800F95E002000C80100FE5E00200000D007B7
:100EA80001000000F85E002000C80100F75E002085
:100EB80000C80100F65E002000C80100FC5E0020AA
:100EC8000000D00701000000F55E002000C8010006
:100ED800F45E002000C80100F35E002000C8010095
:100EE8006C10050800000000000000000000000071
:100EF8000000000058E3040809000000000000009A
:100F0800A00300200400000060E3040809000000BA
:100F1800000000009403002004000000C817050822
:100F28000900000000000000880300200400000001
:100F3800E60E050809000000000000007C03002000
:100F4800040000007C1005080900000000000000F3
:100F58007003002004000000841005080900000048
:100F68000000000064030020040000008C10050845
:100F780009000000000000005803002004000000E1
:100F88009410050809000000000000004C03002030
:100F980004000000441005080100000000000000E3
:100FA8000000000000000000000000000E0000002B
:100FB8000000000000000000000000009412050876
:100FC8000000000000000000000000000000000019
:100FD800D80005080700000000000000C403002036
:100FE80000000000A412050808000000000000002E
:100FF800B803002000000000B01205080800000037
:1010080000000000AC0300200000000044100508A8
:1010180001000000000000000000000000000000C7
:10102800000000000E0000000000000000000000AA
:1010380000000000B81205080000000000000000D1
:101048000000000000000000C81205080D000000A4
:10105800000000000004002000000000D012050875
:101068000D00000000000000F40300200000000054
:10107800D81205080700000000000000EC0300205B
:1010880000000000E01205080D000000000000004C
:10109800E003002000000000E81205080D00000031
:1010A80000000000D403002000000000F012050832
:1010B8000700000000000000CC0300200000000032
:1010C80044100508010000000000000000000000B6
:1010D80000000000000000000E00000000000000FA
:1010E8000000000000000000F812050800000000E1
:1010F800000000000000000000000000D800050803
:101108000C00000000000000D25C0020000000007D
:101118000C1305080C00000000000000D45C00203F
:10112800000000001C1305080C000000000000006F
:101138000A5D0020000000002C1305080C000000C8
:1011480000000000FE5C00200000000040130508BD
:101158000C00000000000000D65C00200000000029
:101168004C1305080C00000000000000D85C0020AB
:1011780000000000541305080C00000000000000E7
:10118800DA5C002000000000681305080C0000006D
:1011980000000000DC5C002000000000701305085F
:1011A8000C00000000000000DE5C002000000000D1
:1011B800781305080C000000000000001C5D0020EA
:1011C80000000000901305080C000000000000005B
:1011D800E05C0020000000009C1305080C000000E3
:1011E80000000000E25C00200000000068E3040842
:1011F8000C00000000000000E45C0020000000007B
:10120800A41305080C00000000000000E65C0020A4
:1012180000000000B01305080C00000000000000EA
:10122800E85C002000000000BC1305080C0000006A
:1012380000000000EA5C002000000000C813050858
:101248000C00000000000000EC5C00200000000022
:10125800D41305080C00000000000000EE5C00201C
:1012680000000000E01305080C000000000000006A
:10127800025D002000000000E81305080C000000D3
:1012880000000000005D002000000000F0130508C9
:101298000C000000000000000E5D002000000000AF
:1012A800FC1305080C00000000000000105D002081
:1012B80000000000081405080C00000000000000F1
:1012C800165D002000000000381105080C00000021
:1012D80000000000F05C0020000000001414050865
:1012E8000C00000000000000F85C00200000000076
:1012F8001C1405080C00000000000000F25C00202F
:1013080000000000281405080C0000000000000080
:10131800F45C002000000000341405080C000000F4
:1013280000000000F65C0020000000003C140508E6
:101338000C00000000000000FA5C00200000000023
:10134800F80005080C00000000000000045D002003
:1013580000000000481405080C0000000000000010
:10136800FC5C002000000000850F05080C00000050
:10137800000000000C5D0020000000005414050867
:101388000C00000000000000065D002000000000C6
:101398005C1405080C00000000000000085D002037
:1013A80000000000641405080C00000000000000A4
:1013B800125D0020000000006C1405080C000000FD
:1013C80000000000145D00200000000074140508EF
:1013D8000C00000000000000265D00200000000056
:1013E8004410050801000000000000000000000093
:1013F80000000000000000000E00000000000000D7
:1014080000000000000000007C1405080000000037
:10141800000000000000000000000000881405081B
:101428000D0000000000000058040020000000002B
:10143800901405080D000000000000004C04002076
:1014480000000000981405080700000000000000D4
:101458004404002000000000A41405080700000050
:10146800000000003C04002000000000B014050843
:101478000900000000000000300400200000000007
:10148800BC14050809000000000000002404002026
:1014980000000000C8140508090000000000000052
:1014A8001804002000000000D814050809000000F6
:1014B800000000000C040020000000004410050893
:1014C8000100000000000000000000000000000013
:1014D800000000000E0000000000000000000000F6
:1014E80000000000EC1405080000000000000000E7
:1014F8000000000000000000FC14050805000000C2
:10150800000000002D5D00200000000044100508C8
:1015180001000000000000000000000000000000C2
:10152800000000000E0000000000000000000000A5
:10153800000000000415050800000000000000007D
:101548000000000000000000FC0F0508000000007B
:1015580000000000201E002004000000E20E050824
:101568000D000000A5BF0208AC0400200000000028
:10157800441A05080D000000A1950208A0040020E7
:1015880000000000A81305080D000000859502085A
:101598009404002000000000101505080800000051
:1015A800000000008804002004000000141405084E
:1015B8000D000000CD9402087C040020000000000B
:1015C800181505080900000000000000700400203C
:1015D80004000000C41405080300000075C40208D4
:1015E8006404002000000000441005080100000009
:1015F80000000000000000000000000000000000E3
:101608000E000000000000000000000000000000C4
:101618002015050800000000000000000000000080
:1016280000000000301505080D0000000000000053
:10163800C404002000000000381505080A00000056
:10164800000000003A5F0020000000004415050873
:101658000A00000000000000425F002000000000B7
:101668004C1505080A000000000000004A5F002031
:1016780000000000541505080800000000000000E4
:10168800B804002000000000441005080100000014
:101698000000000000000000000000000000000042
:1016A8000E00000000000000000000000000000024
:1016B8005C150508000000000000000000000000A4
:1016C80000000000701505080D0000000000000073
:1016D800DC0400200000000080150508040000005C
:1016E8001DC202080000000000000000881505085F
:1016F8000D00000000000000D004002000000000E1
:101708009C15050804000000F9C10208000000004B
:10171800000000004410050801000000000000005F
:101728000000000000000000000000000E000000A3
:10173800000000000000000000000000A4150508DB
:101748000000000000000000000000000000000091
:10175800B815050808000000000000002405002056
:1017680000000000C4150508080000000000000083
:101778001805002000000000D0150508080000002A
:10178800000000000C05002000000000DC15050822
:101798000800000000000000000500200000000014
:1017A800E81505080800000000000000F404002007
:1017B80000000000F4150508080000000000000003
:1017C800E8040020000000004410050801000000A3
:1017D8000000000000000000000000000000000001
:1017E8000E000000000000000000000000000000E3
:1017F8000016050800000000000000009702002005
:10180800000000000C1605080B0000000000000096
:10181800B805002000000000181605080B0000009D
:1018280000000000AC050020000000002416050898
:101838000B00000000000000A005002000000000D0
:10184800301605080B000000000000009405002079
:10185800000000003C1605080B0000000000000016
:101868008805002000000000481605080B0000004D
:10187800000000007C050020000000005416050848
:101888000B000000000000007005002000000000B0
:10189800601605080B000000000000006405002029
:1018A800000000006C1605080B0000000000000096
:1018B8005805002000000000781605080700000001
:1018C80000000000500500200000000080160508F8
:1018D800070000000000000048050020000000008C
:1018E8008C1605080B000000000000003C050020D5
:1018F800000000009816050808000000000000001D
:101908003005002000000000441005080100000018
:1019180000000000000000000000000000000000BF
:101928000E000000000000000000000000000000A1
:10193800A4160508000000000000000000000000D8
:1019480000000000B81605080800000000000000AC
:10195800F405002000000000C41605080800000077
:1019680000000000E805002000000000D01605086F
:101978000800000000000000DC0500200000000056
:10198800DC1605080800000000000000D005002053
:1019980000000000E816050808000000000000002C
:1019A800C4050020000000004410050801000000E4
:1019B800000000000000000000000000000000001F
:1019C8000E00000000000000000000000000000001
:1019D800F016050800000000000000009402002036
:1019E80000000000001705080B00000000000000C0
:1019F80038060020000000000C170508070000004A
:101A0800000000003006002000000000181705083C
:101A18000700000000000000280600200000000069
:101A28002417050807000000000000002006002019
:101A38000000000030170508080000000000000042
:101A480014060020000000003817050808000000F0
:101A580000000000080600200000000040170508EC
:101A68000700000000000000000600200000000041
:101A780044100508010000000000000000000000FC
:101A880000000000000000000E0000000000000040
:101A980000000000000000004C17050800000000CE
:101AA80000000000940200200000000058170508FC
:101AB8000700000000000000A80600200000000049
:101AC800601705080700000000000000A0060020BD
:101AD800000000006817050807000000000000006B
:101AE8009806002000000000701705080800000094
:101AF800000000008C060020000000007817050890
:101B0800070000000000000084060020000000001C
:101B18008017050807000000000000007C06002070
:101B280000000000881705080700000000000000FA
:101B38007406002000000000901705080800000047
:101B48000000000068060020000000009817050843
:101B580007000000000000006006002000000000F0
:101B6800A017050807000000000000005806002024
:101B780000000000A817050807000000000000008A
:101B88005006002000000000B017050808000000FB
:101B98000000000044060020000000004410050872
:101BA800010000000000000000000000000000002C
:101BB800000000000E00000000000000000000000F
:101BC800000000000000000011990208B006002083
:101BD8002B5D00202B0000008CC004082A5D00202B
:101BE80000C80100285D0020E803D00701000000BC
:101BF8004D4154454B46343131000000C55C00204E
:101C080000030100C45C0020000301005998020889
:101C1800319802088C070020ED970208A197020866
:101C2800040800209998020881980208B808002042
:101C38000D970208C1960208D80B002027990208C0
:101C4800C9C10208B40C00200D950208000000006C
:101C5800040D0020899D0208A99B0208E00D0020C0
:101C68004D99020800000000800E0020F599020836
:101C7800C19902080C0F00207D9A0208C99A02082F
:101C8800C00F0020735E0020010601009199020830
:101C98006199020800110020299A020841C202082D
:101CA800A0110020F99A020891C2020868120020C7
:101CB800685E002001030100B81705080000000055
:101CC800000000000000000000000000C417050824
:101CD8000800000000000000B4130020000000000D
:101CE800CC1705080700000000000000AC13002016
:101CF80000000000DC1705080D00000000000000CF
:101D0800A013002000000000E817050803000000E9
:101D180075C4020894130020000000004410050850
:101D280001000000000000000000000000000000AA
:101D3800000000000E00000000000000000000008D
:101D480000000000F0170508000000000000000077
:101D58000000000000000000001805080A0000004C
:101D68000000000008180508000000001018050809
:101D78000A00000000000000B3D0040800000000C2
:101D8800181805080A00000000000000025F002083
:101D980000000000201805080A00000000000000EC
:101DA800C0130020000000004410050801000000D6
:101DB800000000000000000000000000000000001B
:101DC8000E000000000000000000000000000000FD
:101DD80028180508000000000000000000000000AE
:101DE80000000000341805080300000075C402084C
:101DF800F41300200000000040180508030000004C
:101E080075C40208E81300200000000048180508FF
:101E18000300000075C40208DC1300200000000065
:101E2800501805080500000000000000C35C0020F1
:101E38000000000058180508070000000000000016
:101E4800D4130020000000006418050807000000F3
:101E580000000000CC13002000000000441005081A
:101E68000100000000000000000000000000000069
:101E7800000000000E00000000000000000000004C
:101E880000000000701805080000000000000000B5
:101E9800000000000000000084180508030000008E
:101EA80075C40208241400200000000090180508DA
:101EB8000300000075C40208BC00002000000000F8
:101EC800981805080300000075C4020818140020BB
:101ED80000000000A01805080300000075C40208EF
:101EE8000C14002000000000141405080300000072
:101EF80075C4020800140020000000004410050802
:101F080001000000000000000000000000000000C8
:101F1800000000000E0000000000000000000000AB
:101F280000000000AC1805080000000000000000D8
:101F38000000000000000000BC18050807000000B1
:101F4800EDC20208801400200000000038140508C3
:101F58000300000075C4020874140020000000008B
:101F6800C81805080300000075C40208681400209A
:101F780000000000D01805080300000075C402081E
:101F88005C14002000000000D818050807000000B5
:101F9800D1C202085414002000000000DC1C05080F
:101FA8000300000075C40208481400200000000067
:101FB800E41805080300000075C402083C1400205A
:101FC80000000000F01805080300000075C40208AE
:101FD8003014002000000000441005080100000033
:101FE80000000000000000000000000000000000E9
:101FF8000E000000000000000000000000000000CB
:10200800E1980208B198020888140020759B02081C
:1020180000000000141500207D9702085997020857
:10202800A015002000000000000000005416002049
:102038004D9B020809C30208F4160020FC18050885
:102048000000000000000000000000000000000088
:10205800081905080300000075C4020800180020CC
:1020680000000000101905080300000075C40208EC
:10207800F417002000000000F0010508030000002C
:1020880075C40208E8170020000000001C190508A4
:102098000300000075C40208DC17002000000000DF
:1020A800281905080300000075C40208D01700208D
:1020B80000000000301905080200000025C30208CE
:1020C80000000000000000003819050802000000A8
:1020D80025C302080100000000000000441905089B
:1020E8000200000025C302080200000000000000F2
:1020F800000000000E0000000000000000000000CA
:1021080000000000A25C002088136F170100000087
:10211800A45C002088136F17000000005019050800
:1021280000000000000000000000000000000000A7
:10213800601905080800000000000000E0180020F1
:10214800040000006C1905080800000000000000E9
:10215800D418002000000000C41405080400000082
:10216800CDBF020800000000000000004410050870
:102178000100000000000000000000000000000056
:10218800000000000E000000000000000000000039
:1021980000000000A05C002088136F1701000000F9
:1021A800CC7C002088136F170000000051960208AD
:1021B80000000000EC180020396200200100000037
:1021C8003CC10408CE7C00200100000048C104087E
:1021D800C47C00200200000050C10408BE72002028
:1021E8000000000000000000BC7200200000000099
:1021F80000000000BA72002000000000000000008B
:10220800B87200200000000000000000B672002034
:102218000000000000000000B47200200000000070
:10222800000000005C1E002000000000000000000C
:102238009F5C0020020000005CC10408A819050882
:102248000000000000000000000000000000000086
:10225800601905080800000000000000701900203F
:10226800040000006C1905080800000000000000C8
:102278006419002000000000C414050804000000D0
:102288002196020800000000000000004410050824
:102298000100000000000000000000000000000035
:1022A800000000000E000000000000000000000018
:1022B80000000000B8190508000000000000000038
:1022C8000000000000000000C81905080D0000000B
:1022D8001DC10208A019002004000000D419050837
:1022E8000D000000799602089419002004000000EF
:1022F800E01905080D000000E1C002088819002057
:1023080000000000EC19050803000000699D0208A0
:102318007C19002008000000F819050803000000D7
:1023280075C40208A41C0020000000004410050821
:102338000100000000000000000000000000000094
:10234800000000000E000000000000000000000077
:10235800000000003C10050800000000000000001C
:102368000000000000000000E90D0508040000005E
:10237800E5BF020800000000000000004410050846
:102388000100000000000000000000000000000044
:10239800000000000E000000000000000000000027
:1023A800000000004C1A05080000000000000000B2
:1023B80000000000000000005CE704080D000000B9
:1023C80000000000001A0020040000005C1A050844
:1023D8000800000000000000F419002004000000BC
:1023E800681A05080800000000000000E81900202D
:1023F80004000000701A0508080000000000000032
:10240800DC19002004000000781A05080800000004
:1024180000000000D019002004000000801A050800
:102428000800000000000000C4190020040000009B
:10243800881A05080800000000000000B8190020EC
:1024480004000000901A05080800000000000000C1
:10245800AC19002004000000441005080100000029
:102468000000000000000000000000000000000064
:102478000E00000000000000000000000000000046
:1024880039960208000000000C1A00200000000025
:1024980000000000841A0020000000000000000076
:1024A800241B0020CA7C00200400000068C1040826
:1024B800C87C0020E0150C1700000000C77C002035
:1024C8000800000044C20408C67C00200500000083
:1024D8007CC104080000000000000000741B0020FC
:1024E8000403090412010002EF020140830456327A
:1024F8000002010203010000120100020202004072
:10250800830440570002010203010000090264002D
:10251800030100C032090400000103000000092182
:10252800110100012226000705830308000A080B91
:102538000102020201000904010001020201000572
:1025480024001001052401000204240202052406C7
:102558000102070582030800FF09040200020A00BD
:102568000000070501024000000705810240000045
:1025780009024300020100C03209040000010202FE
:1025880001000524001001052401000104240202B1
:102598000524060001070582030800FF090401005D
:1025A800020A000000070501024000000705810239
:1025B80040000000FF00000000FFFF0000000000D6
:1025C800AA5505010000010005010905A101A100A6
:1025D800050109300931093209330935093409403F
:1025E80009381581257F750895088102C0C000004B
:1025F80009022200010100E0320904000001030180
:1026080002000921110100012226000705830308A1
:10261800000A000000000000010203040102030494
:1026280006070809652503082D2C0308A9270308B0
:10263800750B03087D100308850B0308A10B03081D
:102648004D0B03083D0B03080000000000000000CC
:102658002D202D2D202D2D2D2D202D2D2D2D000023
:10266800000000000000000000000000000000AAB8
:10267800550B010000AA5507010000AA55090200E0
:102688000000AA5503009F0001000000C0120000CE
:10269800FF1FFF1F01000000408300200000000012
:1026A800C02300200400000024010508881D050837
:1026B8000000000019680308A0860100040000005B
:1026C8000000000000000000000000000000000002
:1026D80000000000000000000000000024010508C0
:1026E800B41E050800000000C50E0208E80300003B
:1026F80004000000000000000000000000000000CE
:1027080000000000000000000000000000000000C1
:102718003814050874E3040800000000E1FC000810
:102728007D0000000600000000000000000000001E
:102738000000000000000000000000000000000091
:10274800000000007C0005080000000000000000F8
:10275800FD360208E8030000030000000000000046
:102768000000000000000000000000000000000061
:102778000000000000000000BC1E0508000000006A
:102788000000000099FB0308102700000300000068
:102798000000000000000000000000000000000031
:1027A800000000000000000000000000D41A050826
:1027B80000000000ED920108217202085F76000017
:1027C80005000000000000000000000000000000FC
:1027D80000000000000000000000000000000000F1
:1027E800E40205080000000000000000358302082C
:1027F8001027000001000000000000000000000099
:1028080000000000000000000000000000000000C0
:1028180000000000C81E05080000000000000000BD
:10282800C90E0208E80300000500000000000000CF
:102838000000000000000000000000000000000090
:102848000000000000000000D41E05080000000081
:1028580000000000B9F50008204E00000300000049
:102868000000000000000000000000000000000060
:10287800000000000000000000000000E41E050841
:102888000000000000000000BDF30008204E00001A
:10289800030000000000000000000000000000002D
:1028A8000000000000000000000000000000000020
:1028B800F41E05080000000000000000F5130208DF
:1028C800400D0300030000000000000000000000AD
:1028D80000000000000000000000000000000000F0
:1028E80000000000E80105080000000000000000EA
:1028F8009174030810270000010000000000000088
:1029080000000000000000000000000000000000BF
:10291800000000000000000094000508000000000E
:1029280000000000C5D902081027000003000000BD
:10293800000000000000000000000000000000008F
:1029480000000000000000000000000080000508F2
:1029580000000000000000002113020850C300001E
:10296800010000000000000000000000000000005E
:10297800000000000000000000000000000000004F
:10298800381105080000000000000000B11002081E
:10299800A861000001000000000000000000000025
:1029A800000000000000000000000000000000001F
:1029B80000000000041F05080000000000000000DF
:1029C8008DF50208A086010001000000000000004B
:1029D80000000000000000000000000000000000EF
:1029E8000000000000000000EC02050800000000E4
:1029F8000000000005430208A00F000001000000CD
:102A080000000000000000000000000000000000BE
:102A1800000000000000000000000000101F050872
:102A28000000000000000000D19E020810270000EE
:102A3800010000000000000000000000000000008D
:102A4800000000000000000000000000000000007E
:102A5800F00105080000000000000000BD47030861
:102A68001A41000001000000000000000000000002
:102A7800000000000000000000000000000000004E
:102A8800000000004C0305080000000000000000E2
:102A98005113030810270000010000000000000087
:102AA800000000000000000000000000000000001E
:102AB80000000000000000009C1D05080000000048
:102AC80000000000E9C502081A41000001000000EA
:102AD80000000000000000000000000000000000EE
:102AE8000000000000000000000000001C1F050896
:102AF800000000000000000035430308400D0300FB
:102B080000000000000000000000000000000000BD
:102B180000000000000000000000000000000000AD
:102B2800241F05080000000000000000810E0208B4
:102B3800400D03000000000000000000000000003D
:102B4800000000000000000000000000000000007D
:102B5800000000002C1F0508000000000000000015
:102B680051E7020850C30000030000000000000005
:102B7800000000000000000000000000000000004D
:102B88000000000000000000381F050800000000D9
:102B980000000000116E010840420F000000000014
:102BA800000000000000000000000000000000001D
:102BB800000000000000000000000000441F05089D
:102BC80000000000000000002D69030850C3000049
:102BD80000000000000000000000000000000000ED
:102BE80000000000000000000000000000000000DD
:102BF800000200051002700B491003083D0F03087E
:102C08008527030800000000390B0308C12D0308BD
:102C1800BD0E0308BD2403080000000000000000EA
:102C2800F50A0308B90F0308FD0E0308C5260308B3
:102C3800000000000D0B0308C1240308910E0308CF
:102C48001D2403080000000000000000010B030819
:102C580008000000590A0308550A0308510A030826
:102C6800450A0308410A03084D0A0308490A0308EC
:102C7800CD0A0308C10A0308990A0308AD0A030824
:102C8800850A0308710A03085D0A030801000000A9
:102C980000600240106002400000000000000000D8
:102CA800000B000000000000000000000000000011
:102CB800006002402860024001000000000000009F
:102CC800060C0000000000000000000000000000EA
:102CD8000060024040600240020000000000000066
:102CE800100D0000000000000000000000000000BF
:102CF800006002405860024003000000000000002D
:102D0800160E000000000000000000000000000097
:102D180000600240706002400400000000000000F3
:102D2800200F00000000000000000000000000006C
:102D380000600240886002400500000000000000BA
:102D48002610000000000000000000000000000045
:102D580000600240A0600240060000000000000081
:102D6800301100000000000000000000000000001A
:102D780000600240B8600240070000000000000048
:102D8800362F0000000000000000000000000000D6
:102D980000640240106402400000000000000000CF
:102DA80000380000000000000000000000000000E3
:102DB8000064024028640240010000000000000096
:102DC80006390000000000000000000000000000BC
:102DD800006402404064024002000000000000005D
:102DE800103A000000000000000000000000000091
:102DF8000064024058640240030000000000000024
:102E0800163B000000000000000000000000000069
:102E180000640240706402400400000000000000EA
:102E2800203C00000000000000000000000000003E
:102E380000640240886402400500000000000000B1
:102E48002644000000000000000000000000000010
:102E580000640240A0640240060000000000000078
:102E680030450000000000000000000000000000E5
:102E780000640240B864024007000000000000003F
:102E880036460000000000000000000000000000BE
:102E98000000803F0000000000000000000000006B
:102EA8000000803F0000000000000000000000005B
:102EB800000000000000000000000000000000000A
:102EC8000000000000000000010000000000803F3A
:102ED8000000000000000000000000000000803F2B
:102EE800B4260020000000000000000000000000E0
:102EF80000000000000000000000000000000000CA
:102F080000000000000000000000000000000000B9
:102F180000000000000000000000000000000000A9
:102F28000000000000000000000000000000000099
:102F38000000000000000000000000000000000089
:082F4800000000000100000080
:1080000090ED057A90ED004AD0ED066AD0ED014A78
:10801000D0ED047A90ED035AD0ED025AA4EE007A26
:10802000B0EE406AB0EE470AB0EE667AA4EE867A09
:1080300067EEC07AA5EE407AE5EE867A80ED057AA5
:10804000C0ED067A704700BFD0ED057A90ED013A99
:10805000D0ED003AD0ED064A90ED024A90ED077A55
:1080600090ED035A90ED086AD0ED045AC0ED067AFF
:10807000F0EE406A27EE830AC0ED056AA3EEA60A79
:1080800080ED087AA4EE240AA5EE470AA5EEC60AFA
:1080900080ED070A704700BFD0ED007A90ED017ABD
:1080A00030EE670AE7EE007AB0EE670AC0ED007ABC
:1080B000704700BF704700BF2DE9F04714461D46CA
:1080C00006464FF47A720023204629463FF034FAE0
:1080D0004D4BDFF848814D4A4D4F034488FB031058
:1080E0001844D91782FB032CC1EB601088FB0028D1
:1080F00087FB03279C44474AC1EBEC2CC0EB001ED6
:1081000082FB0C29A3EB8E0E1F44434A86F806E03F
:10811000C1EB27474FEAEC7E08EB000ACEEBA90E35
:1081200082FB07824FEAE0780EEB4E0EC8EB6A182E
:10813000ACEBCE0CC8EB0818DFF8E4E086F804C01E
:10814000A0EB880070718EFB0303F817C0EBE212FE
:1081500040F2B55000FB1272C1EBE353B2F5896FE8
:108160004FEA83073CDA40F2DA239A4242DCB2F566
:10817000B77FB4BF4FF0000E4FF0010E4FEA4E092B
:10818000DFF8A08009EB0E0308EBC3031FFA8EFC97
:10819000D88A09EB0E0108EBC10116310B2301E06F
:1081A00031F8020D904218DD013BF9D1CE44012394
:1081B00038F83E00B37007F5FA670132121ABC4472
:1081C000F270A6F800C0204629464FF47A720023C8
:1081D0003FF0B2F93281BDE8F0870133DBB2E9E765
:1081E0004FF0030CE64640F29650DFF838804FF02F
:1081F0000609CEE74FF0020CDFF82880E64640F291
:1082000029404FF00409C4E780BC92C7C5B3A291CE
:1082100007452EC2ABAAAA2A73B06D168988888832
:10822000792D03117092040830B403888278C478E1
:10823000154DA3F5FA6303F0030101EB4101013A87
:1082400002EB81029B0835F812500279611E40F260
:10825000B55404FB03132B4403EB430302EBC303AA
:108260004279847909490089C3EB031302EB830344
:108270002144C3EB031301EB83034FF47A72002113
:10828000C2FB030130BC70477092040880436D3814
:108290000028F0B403DA2D230B7040420131092885
:1082A00004464FF0010307DD03EB83035B00B0FBE3
:1082B000F3F2092AF8D883B10F48A0FB0326B4FBD8
:1082C000F3F2092A02F1570C02F1300709DD03FB32
:1082D0001244F30801F801CBEFD100230B70F0BC7E
:1082E000704703FB1244F30801F8017BE5D100233A
:1082F0000B70F0BC704700BFCDCCCCCC884270B4C2
:108300004FF0010442D301FB04F4B0FBF4F58D42BD
:10831000F9D2ECB142BB092D04FB150005F157065B
:1083200005F130020EDDB4FBF1F403F8016B7CB112
:10833000B0FBF4F5092D04FB150005F1570605F116
:108340003002F0DCB4FBF1F403F8012B002CEFD188
:1083500000221A7070BC704703F8016BB4FBF1F493
:10836000002CF5D0B0FBF4F5092D04FB150005F148
:10837000370605F13002EFDCB4FBF1F403F8012B12
:10838000002CEFD100221A7070BC70470546002AFD
:10839000EAD1C0E703685A1C02601970704700BF39
:1083A0002DE9F047089C2578002B804689460CBFB4
:1083B0004FF0200A4FF0300A661C25B3002A26DD54
:1083C000334601E0024698B113F8011B501E002904
:1083D000F8D1971E60B13D46013D51464046C84721
:1083E0006B1C002BF8DC257827EAE770013045B1DB
:1083F000041B29464046C847301916F8015B002D7A
:10840000F7D1BDE8F087002A03DC2846F9E7002011
:10841000EEE7571EDFE700BF01212C220223017087
:1084200042708370704700BFF0B400250E4E00F11B
:10843000FF3C2F46142165B103788B420BD00346D5
:108440000CEB050403E013F8012F8A4203D0A3428A
:10845000F9D1C155013701350B2D02D016F8011F96
:10846000E9E7F0BC704700BFD092040830B4152390
:10847000162517242D212E2203702F23457084707A
:10848000C1700271437130BC704700BF01232021CD
:10849000212241704271037203700371704700BF63
:1084A00006224FF47A730270436070476D4B2DE9DA
:1084B000F04F1C686C4BB3F80AE0B3F804809A895B
:1084C0004FEA0E2AB4EB0A044FEA1E6B4FF0000588
:1084D00087B065EB0B05CDE900450746009C188980
:1084E000019EA0FB044500FB0655E00940EA4560FB
:1084F0004FEA08448C46E9114FEA184510EB04088E
:10850000D888009C41EB0509CDE90489A0FB04450E
:10851000B3F8028000FB0655200A40EA05604FEAE6
:10852000C83429124FEA584510EB040841EB0509FD
:108530000099A2FB010102FB06114FEAD05A4AEA58
:10854000412A1AF5FA634FEAE15B4BF10004B3F5F7
:10855000FA6FCDE9023474F10003424E64DA052467
:10856000AAFB040104FB0B1100FB0BF40AFB014402
:10857000DDE90423A0FB0A0121444D104FEA300439
:10858000121B4FEA900463EB050344EA8174B8EBD5
:108590000408CDE90423DDE9023434484FEAA1059B
:1085A00069EB05094FF0FF31834274EB010326DAD2
:1085B00040F6AC501AEB00024FF000014BEB010308
:1085C00002FB03F1A2FB022303EB4103D400DD0015
:1085D000101B45EA527563EB0501DDE904452418DB
:1085E0004D41CDE904450B24A2FB040104FB03111A
:1085F00049104FEA3000B8EB000869EB0109DDE9EA
:1086000000325343009ADDE90201A2FB02AB0BEBFF
:10861000430B4FEADA7242EA4B02801A4FEAEB73DD
:1086200061EB0301CDE9020197B17168A1FB082359
:1086300001FB0933540D5D1544EAC324DDE904232D
:10864000A21A65EB03031D46D30B43EA45433B6087
:10865000BCF1000F02D0029BCCF8003007B0BDE89F
:10866000F08F00BF182700209840002024FAFFFF59
:108670002DE9F04FDFF8DCC1754CDCF8085022889A
:10868000B4F90AA0C2EB25135200C2EBE502B4F91B
:1086900002505B436A43B4F904501B135D43AD13AE
:1086A00005EBE225B5F5FA324FEAE57B85B04BF1F3
:1086B000FF33CDE90023DDE900325343009AA56181
:1086C000A2FB0289CDE90201B4F9082001990098C2
:1086D00009EB43095143D31700FB0311A2FB00230D
:1086E0000B444FEAEA7B0AFB09F11F0308FB0B135B
:1086F000AAFB080119444FEA102A4AEA016A160344
:108700004FEA212B47EA12571AEB0602E6884BEB99
:10871000070312F1000A43F5004BAAFB060106FB12
:108720000B114A10CB1752EA030100F08E80B4F906
:108730001060009806FB09F1F71708FB0711A6FB6C
:1087400008673944B4F90E808B4601994FEAE879FD
:1087500008FB01F100FB0911A8FB00898944DCF842
:108760000C104FEA4947C1F5801C47EAD837B2469A
:108770004FEA4846B4F90C801AEB060A66464BEB02
:10878000070BF7174FEAC806019600260096F9076F
:10879000DDE900674FEACC7016EB0A0647EB0B07E2
:1087A00041EA5C01801B61EB070140F6354C8946CC
:1087B000A0FB0C010CFB09113EF0BEFEB4F9162023
:1087C000B4F914A04E13470B47EAC14702FB06FC5D
:1087D000D31707FB03CCA2FB07236344564307FBD5
:1087E0000366A2FB07233344560E46EAC31632182B
:1087F0004FEA636747EB010380460AFB01F14FEA4A
:10880000EA7B08FB0B17AAFB08013944C60C46EAB1
:10881000413612EB06084FEAE147B4F9122043EB68
:1088200007094FEA182141EA096113010B44029A32
:108830000AB11B0A1360039B23B105EB8505803544
:108840002D121D6005B0BDE8F08F0023EFE700BFDB
:10885000AC40002018270020704770472DE9F041F8
:10886000334B344E1A8A7489B6F91450B6F9048021
:10887000B6F90E70B6F920C05B69121B34895443F7
:10888000E213B6F912401544E40294FBF5F4B6F98C
:1088900002501444A4F57A6E0EFB0EF20EFB05F5A1
:1088A0000EFB08FEB6F90C80F4611213574302FB6D
:1088B00008F2121402EB6E32ED1205EBE7270232DA
:1088C000B6F90050B6F806E0921002F5004207EB48
:1088D00085070EFB02F207FA0CF74FEAD23E023789
:1088E0004CF25032A3EBA70742FA0CF37B4355BF7F
:1088F0005B00B3FBFEF3B3FBFEF35B0078B11A122F
:1089000002FB02F540F6DE326A430B4D12145D4362
:1089100002EB254202F6CF6203EB2213036021B182
:108920000A235C43083424110C60BDE8F08100BFC9
:10893000182700207440002043E3FFFF4FF400633A
:10894000838270474FF4006383827047012380F86D
:10895000543070474FF4006383827047F0B4037C57
:10896000456902681F2B37D9203B20215468994064
:108970000C4223D010249C40D160D4605168D9406F
:10898000CE074ED4EFF31183502282F31288EA6BA4
:108990001168C90709D45468002C52D1D5E909617E
:1089A0008E4243D1012285F86020DBB283F3118827
:1089B000037C02681F2B194614D9203B08215068FC
:1089C0009940084200D0D1600421506801FA03F3B5
:1089D000184223D1F0BC7047202416689C402642E0
:1089E0000FD11946082310688B40184200D09360BD
:1089F0000423106803FA01F10842EBD09160F0BC47
:108A0000704710219940946091601168D940CC075B
:108A1000B8D5012101FA03F39360B3E7D360F0BC4A
:108A20007047012101FA03F3D360ABE7AF690F444C
:108A3000D7600ED82E69711A5160AC62002185F89A
:108A40006010116841F00101DBB2116083F31188FD
:108A5000AEE7711A5160AE62F0E700BF70B4037CFC
:108A600001681F2B26D9A3F1200520224C68AA40BB
:108A7000224214BF01220022D2B142691B481C4C81
:108A800002EB420200EB4212257854682068CDB90F
:108A9000E56856892C6824F001042C6082891F2B1C
:108AA00022EA060282811AD8202202FA03F38B609E
:108AB00070BC704720220C689A40224214BF0122E9
:108AC0000022D9E7A469226822F00102226082898B
:108AD00022F480721204120C1F2B8281E4D9A3F1BC
:108AE000200220239340CB6070BC7047D0A20020AE
:108AF000CCA2002070B59D4C2368002B40F005816E
:108B00009B4B1A78002A68D09A4B19789A4B002907
:108B100064D11868B3F82C5141628489012A44EA6F
:108B200005048481A3F82C1157D0D3F83001B3F891
:108B30005C5241628489022A44EA05048481A3F8D4
:108B40005C124AD0D3F86002B3F88C534162848936
:108B5000032A44EA05048481A3F88C133DD0D3F89A
:108B60009003B3F8BC5441628489042A44EA0504A2
:108B70008481A3F8BC1430D0D3F8C004B3F8EC550A
:108B800041628489052A44EA05048481A3F8EC152E
:108B900023D0D3F8F005B3F81C5741628489062A24
:108BA00044EA05048481A3F81C1716D0D3F82007E3
:108BB000B3F84C5841628489072A44EA0504848149
:108BC000A3F84C1809D0D3F85028B3F87C49516267
:108BD000908920439081A3F87C1970BD5C68198945
:108BE00061602568186845F0010540F20D31256087
:108BF000A0F848108489012A44F480748481ECD060
:108C0000D3F83441B3F83851D3F8300165602568A2
:108C100045F001052560A0F848108489022A44F433
:108C200080748481D9D0D3F86442B3F86852D3F801
:108C300060026560256845F001052560A0F84810D0
:108C40008489032A44F480748481C6D0D3F8944381
:108C5000B3F89853D3F890036560256845F0010593
:108C60002560A0F848108489042A44F48074848123
:108C7000B3D0D3F8C444B3F8C854D3F8C004656083
:108C8000256845F001052560A0F848108489052A6B
:108C900044F480748481A0D0D3F8F445B3F8F85537
:108CA000D3F8F0056560256845F001052560A0F85A
:108CB00048108489062A44F4807484818DD0D3F8C6
:108CC0002447B3F82857D3F820076560256845F096
:108CD00001052560A0F848108489072A44F48074AF
:108CE00084813FF47AAFD3F85428B3F85808D3F806
:108CF00050385060106840F001001060A3F8481030
:108D00009A8942F480729A8170BD05461BF090F8F2
:108D1000217AA9B16DB1194A002316890133002EB9
:108D200018BF0021AB4202F16002F6D100293FF4E6
:108D3000E7AE00F51C501030002320602372DFE600
:108D40002368C31A002BFFF648AF637A3BB1013B9F
:108D5000DBB263722BB100F57A702060D0E623603D
:108D6000CEE6636803442360CAE600BF882B002078
:108D7000D0A50020CCA20020D4A50020D0A20020A5
:108D800010B5027C01681F2A4FF020030ED94C68F1
:108D9000203A93401C4208D00B4A406800241470CB
:108DA000026822F001020260CB6010BD0C689340A3
:108DB0001C42FAD0044A406800241470026822F071
:108DC000010202608B60F0E7D84F00202DE9F041EE
:108DD000C40023189B00B749CA585268958AADB29F
:108DE000EFB2FE070B4461D4BE0737D5BFF35F8FE8
:108DF0001D7EEDB2012D00F0BB80AF4E138BBFF393
:108E00005F8F231801EB83031D7E022D00F0CE80BF
:108E1000231801EB83031D7E032D05D19B7E1BB11F
:108E2000737E002B40F01A81938896F918C043F4A2
:108E300080639380231801EB83031B7E013363451A
:108E40000AD1B37E00257576002B40F08A8020443D
:108E500001EB800000234375BDE8F081964E17F0CA
:108E6000040F96F918C04DD117F0400700F0B280FA
:108E7000178A1D6AFFB205F80C705FFA8CF56F1C3B
:108E800093F818E07BB2DF1CBE4533769C4600F0B9
:108E90000981271801EB87073F7EBB42CAD105F144
:108EA000020C4FFA8CFC86F818C0C3E71588824E76
:108EB00025F400652D042D0C1580158845F480657A
:108EC00015809D7E00273776002D3DD0757E002DC4
:108ED00037D0231801EB830301251B7E7576022B07
:108EE00003D1138843F400631380231801EB830339
:108EF0009B7D43F001031382204401EB8000037E3D
:108F0000BDE8F0819F7E757E4FF0010E86F81AE075
:108F1000002F5CD0002D78D1231801EB83035B7EFA
:108F2000002B00F0A48013880CF1010C4FFA8CFC8C
:108F300043F4007386F818C013801388DF05FCD44F
:108F400078E7DB7DFF2BC4D0231801EB83039D7DE5
:108F500005F0FE051582DB7DFF2BCDD0FF23337698
:108F6000CAE7938823F440731B041B0C93806EE7BD
:108F70009B7E514E002B3FF441AF737E002B3FF49C
:108F80003DAF138823F480631B041B0C1380BFF3D5
:108F90005F8F138B1388B57643F400731380938827
:108FA00096F918C043F48063938043E79B7E002BBF
:108FB0003FF42EAF737E002B3FF42AAF138896F94F
:108FC00018C023F480631B041B0C138016E0002DD3
:108FD000A2D0A8E72D067FF52DAFBCF1FF3F6DD0E5
:108FE000DD6915F80C5015820CF1010C1D7E4FFA4D
:108FF0008CF39D429C4633767FF41CAF938823F418
:1090000080631B041B0C938014E71F7ED3F8208021
:109010005FFA8CF5AE44022F4FFA8EFE17882DD9D9
:1090200027F480673F043F0C1780178AFFB208F8C7
:109030000C701788D3F820C047F400731380138A8C
:10904000DBB20CF80E30938805F1020C4FFA8CFC61
:1090500043F4806386F818C093806EE7938896F98E
:1090600018C023F480631B041B0C9380E2E6138872
:10907000012543F48073138075765EE747F400772B
:109080001780178AFFB208F80C70178AD3F820806F
:1090900005F1030C4FFA8CFCFBB286F818C008F8F7
:1090A0000E304AE7978827F480673F043F0C97808B
:1090B000EFE600BF5436002018270020DD7D158222
:1090C0009D7E37761DB91B7E002B7FF415AF9388EC
:1090D00023F480631B041B0C93800DE7F0B58769B4
:1090E00083B0064617B13B68BA885A837069DFF8C7
:1090F000A8E08389C3244FF47A734FF0060C6D46C1
:109100004FF6FF710EF1010E03E0013B9BB28B4263
:1091100020D002899207F8D5A3B283814FF47A73E5
:1091200002E0A3B28B4215D00289D20703F1FF34CB
:10913000F7D5828992B20DB12A700135BCF1000FCA
:109140000BD00CF1FF3CFF24BEF1000FE1D09EF8E4
:109150000040D7E71FF08CF8B76917B13B68BA88B1
:109160001A839DF805009DF801509DF802109DF8A6
:1091700003409DF804209DF8063041EA052143EAAA
:10918000002342EA04220120A6F85010A6F852203B
:10919000A6F8543003B0F0BDDC92040838B51D4B7E
:1091A0001B78044600F1250593B104221A492030AA
:1091B0003EF0A2FC2846142218493EF09DFC0123F3
:1091C00084F83A30164B1B7873B984F83B3038BDBD
:1091D0002846142213493EF08FFC012384F83A30CC
:1091E0000F4B1B78002BF0D00F4B186859689A680A
:1091F000DD68E56020606160A260DD691869596919
:109200009A69A2610123E5612061616184F83B30C4
:1092100038BD00BF293E00202A3E00202F3E0020FE
:10922000083E002020D00408093E0020014B1868A9
:109230001BF064B8B04B002010B50021044601209B
:1092400019F09CFD207010BD38B500240472451E35
:10925000E1B2022019F092FD0134082C05F8010F4B
:10926000F6D138BD38B52C2200213EF007FC03466C
:10927000642140F2DC5240F2022019745A82132118
:10928000202240F21A4540F26C74188399760E2021
:1092900002211A7701229D82DC8240F2753540F668
:1092A000430483F82200197283F82A109A7383F812
:1092B0002920DD831C8419460248BDE8384015F09A
:1092C000DBBB00BF2CD0040810B4292128240122C4
:1092D0000023047041708270C3705DF8044B7047C6
:1092E000F8B584894FF6FF764FF47A7433B319B327
:1092F0000F78013101E0B44218D00589013CAD0777
:10930000A4B2F8D5BCB284814FF47A7402E0BCB246
:10931000B4420BD00589ED0704F1FF37F7D58589F5
:10932000ADB20AB115700132013BDFE71EF0A0FFBC
:10933000003018BF0120F8BDFF27DEE70120F8BD8F
:1093400008B540F2E93300E0A3B10289013B12F015
:10935000020F9BB2F8D089B2818140F2E93300E07C
:1093600043B10289013B12F0010F9BB2F8D0808912
:10937000C0B208BD1EF07CFFC0B208BD427A4AB13F
:1093800010B5044604F10A01D0E9003098470023E3
:10939000637210BD704700BF437A5A1C0344D2B2B7
:1093A00042729972037A93420AD84AB110B50446C0
:1093B00004F10A01D0E9003098470023637210BD20
:1093C000704700BF28B1302801D0312802D129B31D
:1093D000002070473228FAD03328F8D03428F6D04D
:1093E0003528F4D02028F2D02128F0D01028EED053
:1093F0001128ECD01228EAD01328E8D01428E6D09F
:109400001528E4D0162803D1B1FA81F0400970473D
:109410001728DDD1B1FA81F040097047012070476B
:10942000302829D0312829D0322829D0332829D0F2
:10943000342829D0352829D020282BD021282BD0FA
:10944000102825D0112829D0122829D0132829D056
:10945000142829D0152829D0162805D0172808BF88
:109460000F2302D0002070470E23114A03EB430361
:10947000134493F8760070470023F6E70123F4E7DE
:109480000223F2E70323F0E70423EEE70523ECE7EA
:109490000823EAE70623E8E70723E6E70923E4E7EA
:1094A0000A23E2E70B23E0E70C23DEE70D23DCE7EA
:1094B00070920408024A136823EA000010607047A3
:1094C0003C620020F8B50468C4F30D0405460E465E
:1094D00004B32F6829F052FD092840F08880454CDC
:1094E000236923F440732361236943F400732361E8
:1094F000236943F0010323613E6029F03FFD2369A6
:10950000092823F00103236171D12B6804332B60F8
:10951000002035E0384B394A93422BD902F580427E
:10952000934226D902F5804293422AD902F580421D
:10953000934228D902F58032934226D902F50032AF
:10954000934224D902F50032934222D902F5003227
:10955000934220D902F5003293421ED902F58022AF
:1095600093421CD9B3F1016F1BD3052019F0B6FE4D
:10957000FBE7082429F002FD092814D04FF0FF3042
:10958000F8BD1024F6E71824F4E72024F2E7282495
:10959000F0E73024EEE73824ECE74024EAE74824FB
:1095A000E8E75824E6E7134F3B6923F440733B6137
:1095B0003B6943F400733B613B6923F0F8033B6173
:1095C0003B6943F002031C433C613B6943F4803335
:1095D0003B6129F0D3FC3B6923F002033B613B690B
:1095E000092823F0F8033B613FF473AFC6E76FF03F
:1095F0000100C5E7003C024000400008FF3F0008B2
:10960000F8B504460D468E180027B542206900D1F2
:10961000F8BDE368591CE160234415F8012B1A7268
:109620000429F2D118B9A1682046FFF74BFFC4E91D
:109630000370EAE730B402681146531C036011F866
:10964000024B0160D31C517803609378151D0560AF
:109650001B0443EA0123D078234343EA006030BC73
:10966000704700BF0368591C1A46016012F8021BBC
:109670000260587841EA0020704700BF03685A1C16
:1096800002601878704700BF70B5044608460E4661
:109690003DF066FA31460546024620683EF088F9FC
:1096A00020682844206070BD38B50446006815461F
:1096B0003EF07EF922682A44226038BD036810B467
:1096C0000A0E5C1C04601A7003680A0C5C1C0460BF
:1096D0001A7003680A0A5C1C04601A7003685A1C3A
:1096E000026019705DF8044B704700BF036810B446
:1096F0000A0A5C1C04601A7003685A1C0260197024
:109700005DF8044B704700BF03685A1C026010B438
:10971000197003680A0A5C1C04601A7003680A0C5A
:109720005C1C04601A700368090E5A1C02601970F0
:109730005DF8044B704700BF03685A1C0260197043
:109740000368090A5A1C02601970704710EE103A3B
:10975000C3F3160242F07E5207EE102ADFED167AAE
:10976000DFED164A9FED165ADFED165A9FED166A89
:10977000DFED163ADFED166A9FED164AE7EE274A4F
:10978000DB1507EE903AA4EE875AF8EEE77AE5EE9D
:10979000075A67EEA37AA5EE876AB5EEC00AE6EE31
:1097A000077AF1EE10FAD4BFB0EE440AB0EE660AC2
:1097B00037EE800A704700BFDACDFE3CB9D593BEC4
:1097C0005CB8903FAA841DC022E061401872313F0E
:1097D00007F1B3C2000080FFDFED1D3ADFED1D7A17
:1097E0009FED1D7A9FED1D4ADFED1D4A9FED1D5A2D
:1097F000DFED1D5A9FED1D6ADFED1D6AE0EE237A55
:10980000F4EEC77AF1EE10FA88BFF0EE477AF4EE84
:10981000C47AF1EE10FAB8BFF0EE447AFDEEE77AC2
:1098200017EE903AC3F3160242F07E5207EE102A6A
:10983000A7EE245A03F0FF4300EE103AE5EE075A74
:10984000A5EE876AE6EE076A26EE800A704700BF3B
:109850003BAA384B00007E4E0000FF4E0000000087
:10986000ED185E3C81900FBBAF9D2A3EB2D19F3E6A
:10987000E886023F07EE901AF8EE677A9FED837A4A
:1098800027EE800A20EE070AFDEEC07A17EE903A26
:109890002033402B00F28180DFED7D7AB4EEE70AC1
:1098A000F1EE10FA40F3E680B0EE407A9FED796A6F
:1098B000DFED796A01E0B0EE677AB4EEE67AF1EEB8
:1098C00010FA77EE467AF6DC9FED747AF4EEC77AFA
:1098D000F1EE10FA40F1D1809FED6E6ADFED706A13
:1098E00001E0F0EE477AF4EEE67AF1EE10FA37EEA8
:1098F000867AF6D4DFED6B7AB4EEE77AF1EE10FA01
:1099000040F3A780DFED627A37EEC77A27EE076A69
:10991000DFED655ADFED657ADFED656A9FED655A2B
:10992000E6EE257A67EE065AE6EE276AF7EE007A4B
:10993000A5EEA67AF0EE675AE7EE055AE7EE457A0D
:1099400087EEA55ADFED577A30EE277AFDEEC76A2B
:1099500016EE903A2033402B24D99FED577AF6EE3D
:10996000006AB7EE006AF7EE004AC4EEA57A00235B
:10997000836143610362C36180ED045A67EEA66AA6
:1099800027EE866A27EE877AC0ED006AC0ED026A8C
:1099900080ED016A80ED037A7047B7EE005AF0EE71
:1099A000455ACFE7B4EEE70AF1EE10FA6BDD9FED12
:1099B000396ADFED396A01E0B0EE677AB4EEE67A33
:1099C000F1EE10FA77EE467AF6DC9FED347AF4EE9B
:1099D000C77AF1EE10FA53D59FED2E6ADFED306AAB
:1099E00001E0F0EE477AF4EEE67AF1EE10FA37EEA7
:1099F000867AF6D4DFED2B7AB4EEE77AF1EE10FA40
:109A000033DCDFED2E7AB4EEE77AF1EE10FA44BFE4
:109A1000DFED227A37EEC77A27EE076ADFED224ABA
:109A2000DFED226ADFED227AE6EE246A67EE064A6F
:109A3000E6EE267AB7EE006AA4EEA77AF6EE006AA2
:109A400036EE476AF8EE007A27EE277A66EE266A47
:109A500089E7DFED1A7AB4EEE77AF1EE10FA44BF47
:109A6000DFED0E7A37EEC77A50E7DFED097A37EE91
:109A7000C77AD1E7F0EE407A26E7B0EE677A39E7A9
:109A8000B0EE677AB6E7F0EE477A9EE727D4D23693
:109A9000DB0F4940DB0FC940E4CB1641DB0F49C067
:109AA000E4CB16C1DB0FC93F92E741B99730083CC0
:109AB00015A82ABEF304353F00000000DB0FC9BF24
:109AC000FDEEC07A17EE903A2033402B45D8DFEDFB
:109AD0002D7AB4EEE70AF1EE10FA4DDDDFED2A6AD9
:109AE0009FED2A7A01E0B0EE670AB4EEC70AF1EE04
:109AF00010FA70EE667AF6DC9FED257AF4EEC77AFE
:109B0000F1EE10FA3BD5DFED206A9FED227A01E0FD
:109B1000F0EE407AF4EEC77AF1EE10FA37EEA60ACC
:109B2000F6D4DFED1D7AB4EEE70AF1EE10FA17DD98
:109B3000DFED147A37EEC00A60EE006A9FED176A17
:109B40009FED177ADFED177AA6EE867A20EE266A69
:109B5000E6EE877AA6EE270A70479FED130A704754
:109B6000DFED127AB4EEE70AF1EE10FA44BFDFED52
:109B7000087A37EEC00ADFE7F0EE407ABCE7B0EED5
:109B8000670ACEE7DB0F4940DB0FC940E4CB164143
:109B9000DB0F49C0E4CB16C1DB0FC93F92E741B9E7
:109BA0009730083C15A82ABE00000000DB0FC9BF93
:109BB000DFED2E7AB4EEE70AF1EE10FA4ADDDFEDC2
:109BC0002C6A9FED2C7A01E0B0EE670AB4EEC70A6A
:109BD000F1EE10FA70EE667AF6DC9FED277AF4EE7D
:109BE000C77AF1EE10FA3ED5DFED216A9FED237AB8
:109BF00001E0F0EE407AF4EEC77AF1EE10FA37EEBB
:109C0000A60AF6D4DFED1E7AB4EEE70AF1EE10FAFA
:109C100014DDDFED167A37EEC00A60EE006A9FEDC4
:109C2000196A9FED197ADFED197AA6EE867A20EE91
:109C3000266AE6EE877AA6EE270A7047DFED147AE9
:109C4000B4EEE70AF1EE10FA44BFDFED0B7A37EE1F
:109C5000C00AE2E79FED087AF0EE407AF4EEC77AA8
:109C6000F1EE10FAC0D4B0EE670ACBE7DB0F494043
:109C7000DB0FC940E4CB1641DB0F49C0E4CB16C172
:109C8000DB0FC93F92E741B99730083C15A82ABEBF
:109C9000DB0FC9BFDFED317A30EE277AFDEEC76A00
:109CA00016EE903A2033402B02D99FED2D0A7047D3
:109CB000B4EEE70AF1EE10FA4DDD9FED2A6ADFED12
:109CC0002A6A01E0B0EE677AB4EEE67AF1EE10FAB5
:109CD00077EE467AF6DC9FED257AF4EEC77AF1EE60
:109CE00010FA35D5DFED1F6A9FED217A01E0F0EE25
:109CF000407AF4EEC77AF1EE10FA37EEA60AF6D4FF
:109D0000DFED167AB4EEE70AF1EE10FA1BDCDFEDB8
:109D1000197AB4EEE70AF1EE10FA44BFDFED137AD8
:109D200037EEC00A60EE006A9FED136A9FED137A6A
:109D3000DFED137AA6EE867A20EE266AE6EE877AC3
:109D4000A6EE270A7047DFED0F7A37EEC00AE9E783
:109D5000B0EE670AD4E7F0EE477ABCE7DB0FC93F05
:109D600000000000DB0FC940E4CB1641DB0F49C007
:109D7000E4CB16C1DB0FC9BF92E741B99730083C6D
:109D800015A82ABEDB0F49402DE90048FEF74CFA22
:109D9000054A064B1268B0EB020B61F1000CC3E9F7
:109DA00000BC0120BDE80088308500202060002034
:109DB0000F4B2DE93048D3E9004554EA05020AD19A
:109DC000034640F2011200201880988098715A8052
:109DD0001881BDE83088074B1A6814EB020B45F177
:109DE000000C5A466346FEF767F90120BDE830884B
:109DF000206000203085002002B370B48E1803E08C
:109E0000121B14D1B14215D010F8012BA2F141035D
:109E1000192B11F8013BA3F1410598BF2032192DF0
:109E200003F12004ECD9D21A01D1002BEAD110465B
:109E300070BC70470022104670BC704710467047D7
:109E400070B5044608460D463CF08AFE064602E020
:109E500014F8013F43B1324629462046FFF7CCFFB4
:109E60000028F5D1204670BD1C46204670BD00BFBD
:109E70004FF0FF32FFF7C0BFA0F16103192B98BF6D
:109E800020387047A0F14103192B98BF203070474C
:109E9000202805D0093804288CBF002001207047F5
:109EA000012070472DE9F0411F46064603461C7805
:109EB0002046FFF7EDFF1D4601330028F7D12B2C7C
:109EC00051D02D2C24D0102A804628D04FF0FF33BB
:109ED000B3FBF2F302FB03FC6FEA0C0C5FFA8CFCA1
:109EE000013500200BE0303CE4B2944225DA984280
:109EF0002E461DD81AD002FB004015F8014B392C14
:109F0000F1D944F02004602C17D9573CE4B2ECE7B7
:109F10004FF00108102A6C7805F10105D6D1302CDC
:109F200023D06FF070434FF00F0CD9E76445E2D9AE
:109F300007EA08084FF0FF30DFE701B10E60B8F123
:109F4000000F08D027B1B0F1004F28BF4FF00040FC
:109F50004042BDE8F081002FFBD06FF000439842F3
:109F600028BF1846F5E78046D4E76C782046FFF70F
:109F700089FF782805F1010605D035466FF070435A
:109F80004FF00F0CACE7AC786FF0704302354FF038
:109F90000F0CA5E701230A22002183E76138192865
:109FA0008CBF002001207047413819288CBF002049
:109FB00001207047303809288CBF002001207047ED
:109FC000A0F13003092B07D920F0200041381928CF
:109FD0008CBF002001207047012070470378202BA0
:109FE000024600F10100F9D0092BF7D02D2B00F02B
:109FF000A4802B2B03BF5378B7EE000A0246B7EEBE
:10A00000000AA3F13001C8B209289FED577A10D891
:10A01000F2EE046A07EE901AF8EEE77A12F8013FC2
:10A02000E7EE267AA3F13001C8B20928B0EE677ACC
:10A03000F0D92E2B63D003F0DF03452B02D020EEA6
:10A04000070A704710B451782D294FD02B2979D0A9
:10A05000A1F13003092B02F101027AD80024002378
:10A0600003EB830301EB430312F8011FA1F130005E
:10A070000928A3F13003F3D9B3F59A7F1A4628BF14
:10A080004FF49A72072B6CD9DFED386A1346F7EE5E
:10A09000007A083B072B67EEA67AFAD802F007028F
:10A0A000DAB1F2EE046A012A67EEA67A15D0022A26
:10A0B00067EEA67A11D0032A67EEA67A0DD0042A9D
:10A0C00067EEA67A09D0052A67EEA67A05D067EE74
:10A0D000A67A062A18BF67EEA67A002C3BD087EE38
:10A0E000277A5DF8044B20EE070A70479178A1F1BA
:10A0F0003003092B02F1020230D80124AFE7537874
:10A10000A3F13001C8B2092802F1010293D8F2EE9E
:10A11000046AF0EE665A07EE901AF8EEE77A12F843
:10A12000013F87EEA66AA3F13001C8B2092866EEA6
:10A13000A56A37EE067AEED97DE75378BFEE000ABE
:10A1400002465EE79178A1F13003092B02F1020289
:10A1500084D9F7EE007A27EE277AC2E7F7EE007A85
:10A16000BDE7F7EE007A9BE70000000020BCBE4C84
:10A17000B5EEC00ADFED317AF1EE10FACCBF30EE69
:10A18000270A30EE670ADFED2E7A20EE270A30B577
:10A19000FDEEC07A87B017EE904A054684EAE47077
:10A1A000002303A9A0EBE470CDE90033029334F05F
:10A1B000AFFB002CACBF20232D2303A88DF800306B
:10A1C0003CF0CEFC012803A924D002282DD003287E
:10A1D00005BF3023684668468DF801303DF056FCD7
:10A1E00068463CF0BDFC0338C4B2224669462846A6
:10A1F0003DF082FC00232B5528463CF0B1FC2E227A
:10A20000431C2A540DEB0401E8183DF05BFC284682
:10A2100007B030BD302368468DF801308DF802302C
:10A220008DF803303DF032FCDAE7302368468DF8D4
:10A2300001308DF802303DF029FCD1E76F12033A6E
:10A2400000007A44F8B5064615460846B6FBF2F417
:10A2500034B905FB14640C4B1B5D00F8013BF8BDE1
:10A26000B4FBF2F75FB905FB1747074B05FB146416
:10A27000DA5D00F8012B1B5D00F8013BF8BD3846A4
:10A28000FFF7E0FFEFE700BF38D0040870B40668BE
:10A290008E4217D90139751E002311F8014F08228B
:10A2A000634013F0800F4FEA430318BF83F0D503D8
:10A2B000013ADBB2F5D18D42EFD1721C02603370EE
:10A2C00070BC7047721C00230260337070BC704712
:10A2D0000A44914215D010B40139541E11F8012FCF
:10A2E0000823504010F0800F4FEA400018BF80F064
:10A2F000D500013BC0B2F5D1A142EFD15DF8044BCE
:10A30000704770474840082310F0800F4FEA400024
:10A3100018BF80F0D500013BC0B2F5D1704700BF37
:10A320000A44914215D030B40139551E41F2210240
:10A3300011F8014F082380EA042004044CBF82EA8C
:10A3400040004000013B80B2F7D18D42F0D130BCDB
:10A350007047704770B502221349144C144E4FF6E3
:10A36000FF70FFF7DDFF22884AB1A518B54218D269
:10A37000052A16D92146FFF7D3FF2C46F3E72146DD
:10A380000222FFF7CDFF0222A118FFF7C9FF094BF8
:10A39000E41A094B1C8041F60F53C31A5842584126
:10A3A00070BD0020FCE700BF00400008024000082C
:10A3B00000800008FA3F0008D63C00202DE9F04359
:10A3C000002489B006460D461F46A04605E0252913
:10A3D0000CD030460134A847039A531C03931178DC
:10A3E0000029F4D1204609B0BDE8F083931CCDE9E3
:10A3F00003385078302842D0A0F13003DBB2092B6B
:10A400004FF0000945D96C282AD0642873D019D997
:10A41000732858D063D9752840F0828007F1040C66
:10A42000386805AB00220A216746FDF767FF05ABD8
:10A43000049A009329464B463046FDF7B1FF039A34
:10A440000444CAE725283CD051D958286BD063284A
:10A45000C2D139783046A84704370134039ABCE7A3
:10A46000039B5A1C03921B78642B52D016D8252BC1
:10A4700027D064D9582B18D0632BEAD0ADE7D31C72
:10A4800003939078A0F13003DBB2092B4FF0010960
:10A49000B9D804AA03A932F0CDF8B4E7732B12D0CF
:10A4A00051D9752B2DD0782B97D1A3F15802B2FA40
:10A4B00082F23868520905AB10210437FDF71EFF00
:10A4C000B5E7252185E73B68049A009329460023D8
:10A4D0003046FDF765FF04370444039A7DE76E2894
:10A4E0007FF47AAF039A3B6804371C6075E7002855
:10A4F0003FF478AF70E7386805A9FDF7C9FE043767
:10A5000095E7386805AB00220A21FDF7F7FE04370E
:10A510008DE73B1D386805A91F46FDF7B9FE86E7A4
:10A5200078287FF459AFA0F15802B2FA82F2386865
:10A53000520905AB1021FDF7E1FE043777E7002B48
:10A540003FF450AF49E76E2BCDD046E70EB400B5CF
:10A5500084B005AB019053F8042B0649039301A87E
:10A56000FFF72CFF019B00221A7004B05DF804EB8A
:10A5700003B07047958300082DE9F04707468CB07B
:10A580001E469246002A5CD1154614460A88B2F54A
:10A59000FA6F36D38B78581E0B2832D891F803C047
:10A5A0000CF1FF301E282CD891F804E0BEF1170FF3
:10A5B00027D891F80590B9F13B0F22D888793B282C
:10A5C0001FD8B1F80880B8F57A7F1AD24FF0010889
:10A5D0005EBB09890491002CB4BF2D212B21002CD6
:10A5E000B8BF6442CDE90290CDE905140795CDE9E5
:10A5F00000CE38462A49FFF7A9FF40460CB0BDE817
:10A60000F08700232749ADF828304FF0010C184699
:10A610008DF82A30ADF82C3099469E461A46984659
:10A620000991634609A9002ED3D0CDE90290CDE966
:10A6300000CE38461C49FFF789FF40460CB0BDE804
:10A64000F0871A4C84FB0234A318D417C4EB6314AC
:10A65000C4EB0415A2EB85052DB2002D0846B8BF4A
:10A660006D42FDF7E1FD4FF47A7200238046894682
:10A670003CF062FF3C230AFB030A4FF47A7200238A
:10A68000404649463CF058FF4FF47A7192B200239D
:10A69000C1FB0A2309A8FDF70FFD24B209A975E73C
:10A6A00080D004080000010160D0040889888888EF
:10A6B00010B44C09012250F8243001F01F0102FAB5
:10A6C00001F10B4340F824305DF8044B704700BFA4
:10A6D0004B0901F01F0150F82320012303FA01F177
:10A6E000114214BF18460020704700BFF0EEC07A38
:10A6F000B0EEE07AB4EEE77AF1EE10FAB4BFB0EE65
:10A70000676AB0EE476AB5EE406AF1EE10FA46D0DD
:10A71000B4EEE77AF1EE10FA8CBFF0EE675AF0EE85
:10A72000475AC5EE866A9FED1F3A9FED1F6A9FED5F
:10A730001F4A9FED1F5ADFED1F3ADFED1F4ADFED85
:10A740001F5AA6EEC36AE6EEA34AA6EE864AB7EE05
:10A75000006AA6EE845AA6EEA46AE6EE855AC5EE15
:10A76000866AB4EEE77AF1EE10FA48BFDFED147AAC
:10A77000F5EEC00A48BF77EEE66AF1EE10FA48BF80
:10A78000DFED107AB5EEC00A48BF77EEE66AF1EE6B
:10A7900010FA48BFF1EE666AB0EE660A7047DFED68
:10A7A000076ADEE739094E3DE3B59E3E88FA163E5C
:10A7B00045FE7F3F99FB243F69A2163EA7DFA834E0
:10A7C000DB0FC93FDB0F494070B544880546C4F331
:10A7D0000B04224608460E4600213DF04FF92B6936
:10A7E000094A934202D3094A934205D35BB12146F9
:10A7F0003046BDE870401847224630461946BDE84D
:10A8000070403DF0D5B870BDF0060008380800086B
:10A8100038B5064C064DAC4206D261682046143469
:10A82000FFF7D2FFAC42F8D338BD00BFA00100084B
:10A83000F0060008084B09498B4203D309E01433A2
:10A840008B4206D21A88C2F30B029042F7D1184607
:10A850007047002318467047A0010008F006000862
:10A860002DE9F84FDFF8B08298F8003003B1FEE729
:10A87000A64EB368012288F8002013B11A689B889D
:10A880005383A34B012204461A708B46706840F232
:10A89000E93302E0002B00F07C810289013B12F0D9
:10A8A000020F9BB2F6D00023838140F2E93302E02D
:10A8B000002B00F06E810289013B12F0010F9BB268
:10A8C000F6D0838940F2E93302E0002B00F0758175
:10A8D0000289013B12F0020F9BB2F6D00023838164
:10A8E00040F2E93302E0002B00F067810289013B6E
:10A8F00012F0010F9BB2F6D0838940F2E93302E0F7
:10A90000002B00F056810289013B12F0020F9BB22E
:10A91000F6D00923838140F2E93302E0002B00F0F6
:10A9200048810289013B12F0010F9BB2F6D0838966
:10A9300040F2E93302E0002B00F037810289013B4D
:10A9400012F0020F9BB2F6D0A4B2848140F2E93338
:10A9500002E0002B00F029810289013B12F0010F77
:10A960009BB2F6D083896B4F0BF1FF3B00254FF074
:10A970000A0A4FF00B0940F2E93302E0002B00F025
:10A98000E5800289013B12F0020F9BB2F6D0A0F8DD
:10A990000CA040F2E93302E0002B00F0D7800289DE
:10A9A000013B12F0010F9BB2F6D0838940F2E933EC
:10A9B00002E0002B00F0D6800289013B12F0020F6A
:10A9C0009BB2F6D0ABB2838140F2E93302E0002BB8
:10A9D00000F0C8800289013B12F0010F9BB2F6D053
:10A9E00083891BF8014F40F2E93302E0002B00F0AD
:10A9F000B1800289013B12F0020F9BB2F6D0A0F8A1
:10AA00000C9040F2E93302E0002B00F0A3800289B1
:10AA1000013B12F0010F9BB2F6D0838940F2E9337B
:10AA200002E0002B00F09A800289013B12F0020F35
:10AA30009BB2F6D0A4B2848140F2E93302E0002B4D
:10AA400000F08C800289013B12F0010F9BB2F6D01E
:10AA500083893B6833B11A689B8851690B4214BFE4
:10AA6000538313830135362D85D140F2E93302E05B
:10AA7000002B00F096800289013B12F0020F9BB27E
:10AA8000F6D00823838140F2E93302E0002B00F086
:10AA900088800289013B12F0010F9BB2F6D08389B6
:10AAA00040F2E93301E0002B77D00289013B12F03C
:10AAB000020F9BB2F7D0A023838140F2E93301E07B
:10AAC000002B6AD00289013B12F0010F9BB2F7D034
:10AAD0008389A025002440F2E93301E0002B45D012
:10AAE0000289013B12F0020F9BB2F7D0858140F240
:10AAF000E93301E0002B39D00289013B12F0010F4C
:10AB00009BB2F7D0838940F2E93308E0A4840020A7
:10AB1000D6610020FC840020D561002053B3028957
:10AB2000013B12F0020F9BB2F8D0848140F2E9336E
:10AB300000E0FBB10289013B12F0010F9BB2F8D09B
:10AB40008089C0B283061AD57068C4E71DF090FBF7
:10AB500070682BE71DF08CFB70685FE71DF088FBC9
:10AB6000706876E71DF084FB70683AE71DF080FBA3
:10AB70007068C8E71DF07CFBC0B28306E4D4B368FC
:10AB800013B11A689B881383002388F80030BDE84E
:10AB9000F88F1DF06DFB706894E61DF069FB70681E
:10ABA00097E71DF065FB70687AE71DF061FB706840
:10ABB000D9E61DF05DFB7068BAE61DF059FB7068C0
:10ABC0009BE600BF30B5204D83B06B6840F2E932A0
:10ABD00000E062B31C89013A14F0020F92B2F8D07F
:10ABE00080B2988140F2E93200E002B31889013A5C
:10ABF00010F0010F92B2F8D09A8940F2E93200E0E9
:10AC0000E2B11889013A10F0020F92B2F8D089B27D
:10AC1000998140F2E93200E082B11989013A11F0DC
:10AC2000010F92B2F8D09889C0B203B030BD184677
:10AC300001911DF01DFB6B680199DEE718461DF0C0
:10AC400017FBC0B2F1E700BFA48400202DE9F84F44
:10AC5000DFF8BCB3DBF8083013B11A689B88538364
:10AC6000DBF8040040F2E93302E0002B00F08982B7
:10AC70000289013B12F0020F9BB2F6D005238381BB
:10AC800040F2E93302E0002B00F07B820289013BB5
:10AC900012F0010F9BB2F6D0838940F2E93302E053
:10ACA000002B00F069820289013B12F0020F9BB277
:10ACB000F6D00023838140F2E93302E0002B00F05C
:10ACC0005B820289013B12F0010F9BB2F6D08389AF
:10ACD00040F2E93302E0002B00F067820289013B79
:10ACE00012F0020F9BB2F6D00623838140F2E933C3
:10ACF00002E0002B00F059820289013B12F0010FA3
:10AD00009BB2F6D0838940F2E93302E0002B00F0D9
:10AD100047820289013B12F0020F9BB2F6D000235A
:10AD2000838140F2E93302E0002B00F0398202898E
:10AD3000013B12F0010F9BB2F6D08389B14BDC7E50
:10AD400040F2E93344F0010402E0002B00F02382DA
:10AD50000289013B12F0020F9BB2F6D004238381DB
:10AD600040F2E93302E0002B00F015820289013B3A
:10AD700012F0010F9BB2F6D0838940F2E93302E072
:10AD8000002B00F003820289013B12F0020F9BB2FC
:10AD9000F6D0A4B2848140F2E93302E0002B00F047
:10ADA000F5810289013B12F0010F9BB2F6D0838935
:10ADB000954E3388002B49D0DFF85892DFF858823F
:10ADC0004F464FF0200A072518F8014FFF2C40F29C
:10ADD000E93303D17BE1002B00F0A7810189013B1E
:10ADE00011F0020F9BB2F6D0858140F2E93302E008
:10ADF000002B00F09A810189013B11F0010F9BB2F9
:10AE0000F6D0838940F2E93302E0002B00F088811C
:10AE10000189013B11F0020F9BB2F6D0A4B28481EC
:10AE200040F2E93302E0002B00F07A810189013B16
:10AE300011F0010F9BB2F6D0838998F8003007F823
:10AE4000013B3188A7EB09039942BDDC40F2E933AD
:10AE500002E0002B00F0BB810289013B12F0020FDF
:10AE60009BB2F6D00723838140F2E93302E0002B46
:10AE700000F0AD810289013B12F0010F9BB2F6D0C8
:10AE8000838940F2E93302E0002B00F09B810289C4
:10AE9000013B12F0020F9BB2F6D0FF23838140F2F8
:10AEA000E93302E0002B00F08D810289013B12F0B2
:10AEB000010F9BB2F6D08389524BDC7E40F2E9331E
:10AEC00002E0002B00F079810289013B12F0020FB1
:10AED0009BB2F6D00423838140F2E93302E0002BD9
:10AEE00000F06B810289013B12F0010F9BB2F6D09A
:10AEF000838940F2E93302E0002B00F05B81028994
:10AF0000013B12F0020F9BB2F6D0A4B2848140F252
:10AF1000E93302E0002B00F04D810289013B12F081
:10AF2000010F9BB2F6D083893388002B00F0C680D6
:10AF3000364D00244FF0FF08072703E00134A342F9
:10AF400040F3BC8015F8012BFF2AF7D14FEA2429E2
:10AF5000DBF8040040F2E93302E0002B00F0078147
:10AF60000289013B12F0020F9BB2F6D005238381C8
:10AF700040F2E93302E0002B00F0F9800289013B46
:10AF800012F0010F9BB2F6D0838940F2E93302E060
:10AF9000002B00F0E7800289013B12F0020F9BB208
:10AFA000F6D01FFA89F9A0F80C9040F2E93302E0DC
:10AFB000002B00F0D7800289013B12F0010F9BB2F9
:10AFC000F6D083895FFA84F940F2E93302E0002B7E
:10AFD00000F0C3800289013B12F0020F9BB2F6D051
:10AFE0000623838140F2E93302E0002B00F0B580B4
:10AFF0000289013B12F0010F9BB2F6D0838940F227
:10B00000E9330EE018270020B4000020D04D0020C6
:10B01000A484002034270020CF4D0020002B00F016
:10B0200097800289013B12F0020F9BB2F6D01FFA03
:10B0300089F9A0F80C9040F2E93302E0002B00F00F
:10B0400087800289013B12F0010F9BB2F6D0838901
:10B0500040F2E93301E0002B75D00289013B12F088
:10B06000020F9BB2F7D0878140F2E93301E0002B59
:10B0700069D00289013B12F0010F9BB2F7D083899E
:10B0800040F2E93301E0002B59D00289013B12F074
:10B09000020F9BB2F7D0A0F80C8040F2E93301E038
:10B0A000002B4CD00289013B12F0010F9BB2F7D06C
:10B0B000838933880134A3423FF744AFDBF808307B
:10B0C00013B11A689B881383BDE8F88F93B3018985
:10B0D000013B11F0020F9BB2F8D0858140F2E933B9
:10B0E00000E03BB30189013B11F0010F9BB2F8D0A6
:10B0F000838940F2E93300E093B10189013B11F00B
:10B10000020F9BB2F8D0A0F80CA040F2E93300E0A7
:10B1100033B10189013B11F0010F9BB2F8D08BE6EE
:10B120001DF0A6F8DBF8040087E61DF0A1F8DBF8B7
:10B13000040067E61DF09CF8DBF80400D9E71DF079
:10B1400097F83388FAE61DF093F8DBF8040097E7E8
:10B150001DF08EF8DBF804007AE71DF089F8DBF8C3
:10B1600004004CE71DF084F8DBF804002AE71DF02A
:10B170007FF8DBF8040008E71DF07AF8DBF804003C
:10B18000A6E51DF075F8DBF8040086E51DF070F803
:10B19000DBF804000CE61DF06BF8DBF80400ECE5CE
:10B1A0001DF066F8DBF80400C8E51DF061F8DBF877
:10B1B0000400A8E51DF05CF8B6E61DF059F8DBF8D0
:10B1C000040096E61DF054F8DBF8040074E61DF068
:10B1D0004FF8DBF8040054E62DE9F0419C4CA368DD
:10B1E00013B11A68998851839A4A60681278012AC3
:10B1F00000F0AC81C0F06481022A00F05381964DCA
:10B200002A7812F0400F0CBF4FF4C3724FF4F07263
:10B21000924E328013B11A689B88538310274FF0E7
:10B22000010840F2E93302E0002B00F0418102897D
:10B23000013B12F0020F9BB2F6D0BBB2838140F209
:10B24000E93302E0002B00F033810289013B12F068
:10B25000010F9BB2F6D0838940F2E93302E0002B64
:10B2600000F02A810289013B12F0020F9BB2F6D056
:10B27000A0F80C8040F2E93302E0002B00F01C81C2
:10B280000289013B12F0010F9BB2F6D0838901378E
:10B29000202FC6D1A3681BB11A689B8813835383E0
:10B2A0002D7840F2E93302E0002B00F0588102894A
:10B2B000013B12F0020F9BB2F6D00023838140F2D3
:10B2C000E93302E0002B00F04A810289013B12F0D1
:10B2D000010F9BB2F6D0838940F2E93302E0002BE4
:10B2E00000F041810289013B12F0020F9BB2F6D0BF
:10B2F000ADB2858140F2E93302E0002B00F03381EA
:10B300000289013B12F0010F9BB2F6D08389544AA7
:10B3100040F2E933157802E0002B00F02881028921
:10B32000013B12F0020F9BB2F6D00223838140F260
:10B33000E93302E0002B00F01A810289013B12F090
:10B34000010F9BB2F6D0838940F2E93302E0002B73
:10B3500000F011810289013B12F0020F9BB2F6D07E
:10B36000ADB2858140F2E93302E0002B00F00381A9
:10B370000289013B12F0010F9BB2F6D08389394A52
:10B3800040F2E933157802E0002B00F0F8800289E2
:10B39000013B12F0020F9BB2F6D00323838140F2EF
:10B3A000E93302E0002B00F0EA800289013B12F051
:10B3B000010F9BB2F6D0838940F2E93302E0002B03
:10B3C00000F0E1800289013B12F0020F9BB2F6D03F
:10B3D000ADB2858140F2E93302E0002B00F0D3806A
:10B3E0000289013B12F0010F9BB2F6D083891E4BFC
:10B3F000DD7E40F2E93345F0040502E0002B00F069
:10B40000C6800289013B12F0020F9BB2F6D00423E2
:10B41000838140F2E93302E0002B00F0B88002891A
:10B42000013B12F0010F9BB2F6D0838940F2E93361
:10B4300002E0002B00F090800289013B12F0020F25
:10B440009BB2F6D0ADB2858140F2E93310E000BF87
:10B45000A4840020F0840020A8020020B400002072
:10B46000F7840020F884002018270020002B73D0D8
:10B470000289013B12F0010F9BB2F7D08389A368C8
:10B4800013B11A689B881383474C328847480021C0
:10B490003CF0F4FA23781BB1FFF7D8FB00232370AC
:10B4A000BDE8F081424D08222A704FF4C372AFE626
:10B4B0001CF0DEFE6068CFE61CF0DAFE6068E6E6AF
:10B4C00040F2E93301E0002B69D00289013B12F020
:10B4D000020F9BB2F7D0A023838140F2E93301E051
:10B4E000002B5CD00289013B12F0010F9BB2F7D018
:10B4F000838940F2E93301E0002B4CD00289013B03
:10B5000012F0020F9BB2F7D00023838140F2E9339F
:10B5100001E0002B3FD00289013B12F0010F9BB2EA
:10B52000F7D08389D8B200F00603022B204D08D053
:10B5300000F00503012B04D14822D4E901032A704D
:10B5400007E00822D4E901032A70AEE7184D48222B
:10B550002A704FF4F0725BE61CF08AFE8FE71CF055
:10B5600087FE6068B8E61CF083FE6068CFE61CF0DA
:10B570007FFE6068E8E61CF07BFE6068FFE61CF07A
:10B5800077FE606818E71CF073FE60682FE71CF018
:10B590006FFE60684AE71CF06BFEC0B2C3E71CF0A8
:10B5A00067FE6068A5E700BF000000203427002088
:10B5B000A80200202DE9F041574CA36813B11A6886
:10B5C0009B885383606840F2E93301E0002B4BD045
:10B5D0000289013B12F0020F9BB2F7D080238381D6
:10B5E00040F2E93301E0002B3ED00289013B12F02A
:10B5F000010F9BB2F7D0838940F2E93301E0002BC1
:10B600002ED00289013B12F0020F9BB2F7D000232B
:10B61000838140F2E93300E013B30289013B12F069
:10B62000010F9BB2F8D08089C0B2A36813B11A6829
:10B6300099881183394D3A4E2A78376882420CD165
:10B64000384A12783AB9DFF8E880D8F8FC21BA1AFB
:10B65000B2F57A7F0CD8BDE8F081BDE8F041BBE5DA
:10B660001CF006FEC0B2E0E71CF002FE6068C3E713
:10B6700013B11A689B885383A0216068FDF760FEB0
:10B6800000216068FDF75CFEA36813B11A689B880F
:10B690001383254C2378182B0FD12B78234A03F0E2
:10B6A0004003002B00F007010CBF4FF00D0C4FF0D2
:10B6B000100C13805180A2F806C0410706D5002364
:10B6C000C8F80032C8F8FC71BDE8F08100F0050050
:10B6D000012819D00028F5D12B785B06F2D5D8F8CF
:10B6E00000223368A2B19B1A642BEBD9FFF774FDDB
:10B6F0002378182BE6D1B8F804320C4A01339BB2F8
:10B70000A8F804329380DDE72B785A06E7D5D9E70D
:10B71000C8F80032D6E700BFA4840020A8020020A9
:10B7200030850020F0840020E5840020E88400209B
:10B73000182700202DE9F84F2D4A2E4E01231370B3
:10B74000FFF738FFB6F806222B4BDFF8B8E0B3F866
:10B75000008002F1640C1FFA8CFC00234FF0050BF3
:10B760004FF0060A4FF0070901E062453CD0B418DB
:10B770001EF80200217F814202F1010503F105015B
:10B7800010D07718F1182077140A81F808B281F8E0
:10B790000AA281F80B2281F80C9281F80942063343
:10B7A00087F80802AAB24245DFD30022A6F8062293
:10B7B00023B90F4A00231370BDE8F88F0F4CA2681D
:10B7C00012B1116892884A8300220D496068FDF722
:10B7D00087FDA368002BECD01A689B881383044A6A
:10B7E00000231370BDE8F88FA6F80622E0E700BF3B
:10B7F000D561002018270020B4000020A484002078
:10B8000020290020D04D00200E4B10B41C888CB194
:10B810000D4B0E4A1878117F88420FD11C441C3200
:10B82000013305E013F8011B12F8010F884205D11E
:10B83000A342F7D101205DF8044B704700205DF86A
:10B84000044B7047B4000020D04D00201827002082
:10B850001378C3B130B41E240B4D14FB01012944ED
:10B86000801A84181D2C07DC01F8013B12F8013FF7
:10B87000002BF6D130BC704712F8013F0131002B8C
:10B88000EFD130BC70477047D04D002070B5264DC9
:10B89000C1F10301AB6841EA8006F6B213B11A6840
:10B8A0009B885383B6B21024686840F2E93301E004
:10B8B000002B31D00289013B12F0020F9BB2F7D06E
:10B8C000A3B2838140F2E93300E02BB30289013B4C
:10B8D00012F0010F9BB2F8D0838940F2E93300E007
:10B8E000F3B10289013B12F0020F9BB2F8D08681BE
:10B8F00040F2E93300E09BB10289013B12F0010FF5
:10B900009BB2F8D083890134202CCDD1AB6813B120
:10B910001A689B88138370BD1CF0AAFC6868DCE77A
:10B920001CF0A6FCEFE700BFA484002038B5264B2E
:10B93000DD7E00283ED105F0F705244CDD76A368B6
:10B9400013B11A689B885383606840F2E93301E0C1
:10B95000002B35D00289013B12F0020F9BB2F7D0C9
:10B960000423838140F2E93300E04BB30289013BB9
:10B9700012F0010F9BB2F8D0838940F2E93300E066
:10B98000DBB10289013B12F0020F9BB2F8D0ADB2DD
:10B99000858140F2E93300E07BB10289013B12F07E
:10B9A000010F9BB2F8D08389A36813B11A689B88F2
:10B9B000138338BD45F00805BFE71CF059FCF3E7D9
:10B9C0001CF056FC6068D8E718270020A4840020EB
:10B9D000144B984223D003F5806398421FD003880C
:10B9E00023F040031B041B0C0380038823F038035F
:10B9F0001B041B0C59B141F48071002991FAA1F18B
:10BA0000B1FA81F108BF4FF0FF310139C900194384
:10BA100089B20180038843F04003038070474908DE
:10BA2000DDE700BF00380040F0B587B00023604A72
:10BA300000930193136843F48033136003E0009B89
:10BA4000B3F5A04F09D0136803F400330193009BB2
:10BA500001330093019B002BF1D0554B1B6813F46D
:10BA6000003318BF01230193019B012B63D0514D7B
:10BA70004F4B514AEA605149586F514A0860AA60D9
:10BA80005E6B504C504F514A514826F080065E6321
:10BA90005E6F46F080765E67196B0C431C63596BD2
:10BAA0005963196C39431964596C06AC0A4348F25E
:10BAB000FF715A6444F8101D0123002621468DF8B9
:10BAC0000F304FF6FF778DF80C608DF80D608DF814
:10BAD0000E6027F0EBFE21463E48029727F0E6FE77
:10BAE00021463D48029727F0E1FE21463B4827F0DA
:10BAF000DDFE21463A4827F0D9FE204627F00EFB0E
:10BB0000384B394C1B68029A38483949A4FB034327
:10BB10009B09A0FB0202013B920CB3F1807F0A60FB
:10BB200007D2344AF0200721536085F8230096603D
:10BB3000116007B0F0BD1E4B2F4C1A6C2F4942F01C
:10BB400080521A64206840F44040D1E90152C9682B
:10BB500020609868986098689860120642EA85129A
:10BB6000986842F48002490842F00802013942EA2A
:10BB7000014240F4805098605A601A6842F0807226
:10BB80001A601A689201FCD51D49094A40F20270F8
:10BB90000860996821F003019960996841F00201F9
:10BBA0009960936803F00C03082BFAD15FE700BF9C
:10BBB0000038024000ED00E00005FA0584AF0020E7
:10BBC000000000081F906700FFC9FE36335F0700C2
:10BBD000000002400004024000080240000C024045
:10BBE00000100240A0A20020D34D621083DE1B4350
:10BBF0003485002010E000E00070004000000020CC
:10BC0000003C0240074A08B51168074B994208D129
:10BC1000064B00201968106081F308885B6898471C
:10BC2000FEE708BDC4C20020EFBEADDE0000FF1F6E
:10BC300008B5054B1B6803B19847044B044A1A60CA
:10BC400072B63BF087FE00BF003C0020C4C200205B
:10BC5000EFBEADDE08B5034B1B6803B1984772B663
:10BC60003BF078FE003C0020074A002302E001334D
:10BC7000102B07D05168814202F12002F7D1581CE5
:10BC8000C0B2704700207047602400200138F0B532
:10BC900040013C4CDFF820C125583B4FDCF83060B8
:10BCA000BD420CBF4FF400154FF4800527182E43FA
:10BCB0007D68CCF83060354EF960B54283B07B6169
:10BCC00051D0334B9D424ED0A3F57A739D4236D06E
:10BCD00003F580639D4232D0A3F57A739D4246D02E
:10BCE00003F580639D4242D0A3F57A739D4240D014
:10BCF00003F580639D423CD0A3F57A739D4234D016
:10BD000003F580639D4230D0A3F57A739D4232D013
:10BD100003F580639D422ED0A3F57A739D422CD00B
:10BD200003F580639D4228D0A3F57A739D4226D007
:10BD30001849194B8D420CBF1D46002500E0174DD8
:10BD400004449209667CE5610021012301A88DF875
:10BD500004608DF805208DF806108DF807302FF05F
:10BD60000BFA03B0F0BD0E4DEAE70E4DE8E70E4DBD
:10BD7000E6E70E4DE4E70E4DE2E70E4DE0E7064D37
:10BD8000DEE700BF60240020006002401060024037
:10BD900010640240B864024000800028008800104F
:10BDA00020800010208000200080201000800018DB
:10BDB0000088002000802020003802400138F0B4C4
:10BDC00044010948094D0359094F2E6B2044BB42D9
:10BDD0000CBF4FF400134FF4800333432B63017601
:10BDE0004276F0BC704700BF60240020003802405B
:10BDF000006002402DE9F04F534C54F8204083B0CE
:10BE0000002C00F09C80656E002D00F09A80984612
:10BE1000174604F16A034D4A0646286922606361A9
:10BE200004F1EA028023A261E3604FF480726B6840
:10BE3000A1602261E365A24668B1FFF715FF721C9D
:10BE4000D2B20C21FFF7BAFFE36DA9682A69A26399
:10BE500004332164A365E868A0B1FFF705FF721CF5
:10BE60008146D2B20B21FFF7A9FF2346EA7F38496A
:10BE70004846FFF70BFFD5E90212E36D6164043316
:10BE80006365E26394F8690016F0FEFA814694F85F
:10BE9000680016F0F9FA8346287F00284CD118F084
:10BEA000080F36D1BA070DD5B9F1000F0AD00B2211
:10BEB000731C89F8062089F8073048466A7F2221DA
:10BEC00016F07CF9FB0715D4236C7BB995F820207C
:10BED000A97F8DF8063001A8930901228DF805305D
:10BEE0008DF804108DF807202FF046F9504603B066
:10BEF000BDE8F08FBBF1000FE6D0701C0C238BF86F
:10BF000007008BF8063058466A7F222116F056F952
:10BF1000DAE7B9F1000F05D0701C0B2389F8070090
:10BF200089F8063018F0100F484614BF022112217C
:10BF30006A7F16F043F9C7E72FF040F9AFE7A24652
:10BF4000D4E7AA46D2E700BF1C36002014930408A9
:10BF50005D8900080348D0F8EC3113B100F5F070AA
:10BF600018477047602400200348D0F8CC3113B143
:10BF700000F5E07018477047602400200348D0F8AF
:10BF8000AC3113B100F5D070184770476024002021
:10BF90000348D0F88C3113B100F5C07018477047D2
:10BFA000602400200348D0F86C3113B100F5B07064
:10BFB00018477047602400200348D0F84C3113B173
:10BFC00000F5A07018477047602400200348D0F89F
:10BFD0002C3113B100F59070184770476024002091
:10BFE0000348D0F80C3113B100F580701847704742
:10BFF000602400200348D0F8EC300BB1E030184743
:10C00000704700BF602400200348D0F8CC300BB14B
:10C01000C0301847704700BF602400200348D0F8A4
:10C02000AC300BB1A0301847704700BF602400202F
:10C030000348D0F88C300BB180301847704700BFF0
:10C04000602400200248C36E0BB16030184770476F
:10C05000602400200248C36C0BB140301847704781
:10C06000602400200248C36A0BB120301847704793
:10C07000602400200248C36803B11847704700BF1E
:10C0800060240020F8B5624D04012F190646387A65
:10C090002FF094F83B7A03F01F015B090122032B78
:10C0A00002FA01F26DD0042B66D0022B5CD02B1962
:10C0B0000136187916F0E8F9F6B2074610B11223E6
:10C0C000C67183712B19587916F0DEF910B113235C
:10C0D000C67183712B19987916F0D6F910B1142313
:10C0E000C67183712E190A21F279384616F066F866
:10C0F000707916F0C9F9F2790A2116F05FF8B07973
:10C1000016F0C2F9F2790A2116F058F82B59414A73
:10C11000934246D0404A93424ED0404A934256D032
:10C120003F4A93425ED03F4A93422FD03E4A9342C9
:10C1300063D02B191B7BE3B9012002222B591988EC
:10C1400001F4415141F445710A4302431A809A8B2C
:10C1500022F400621204120C07219A8319821A88B1
:10C1600042F040021A80F8BD304B596A0A435A62C5
:10C170009DE700200246E1E72C4B19690A431A614A
:10C1800095E72A4B196A0A431A6290E702F568425A
:10C190004FF48010536A43F48013536226F000FF7B
:10C1A000C7E702F584324FF48050536A43F480535A
:10C1B000536226F0F5FEBCE702F500324FF48040F2
:10C1C000136A43F48043136226F0F2FEB1E702F5EE
:10C1D000FE324FF40040136A43F40043136226F02A
:10C1E000E7FEA6E702F582324FF40050536A43F4AB
:10C1F0000053536226F0D4FE9BE702F564424FF4ED
:10C200000010536A43F40013536226F0C9FE90E70E
:10C21000B48400200030014000380040003C004061
:10C2200000340140005001400054014000380240F9
:10C23000431C00F010812DE9F04F4FEAC00B0BEBCF
:10C2400000039B00DFF8808258F803A087B008EB5A
:10C250000304BAF1000F00F0FB80143308EB030174
:10C260000022DAF8047048F80320C1E90122CA600C
:10C27000D4E90259431CDBB215B11522EB71AA7146
:10C28000B9F1000F04D0162289F8073089F806208A
:10C2900001909AF818002EF091FFBB8823F44073A8
:10C2A0001B041B0CBB8028461AF072FF48461AF08C
:10C2B0006FFF112128461AF0C9FE112148461AF0D5
:10C2C000C5FE0926332405E0013C4FF00A0006D0E4
:10C2D00017F000FE28461BF08FFE0028F4D02846F9
:10C2E0001AF050FF052017F0F5FD28461AF050FF10
:10C2F000052017F0EFFD013EE4D128461AF042FF79
:10C30000052017F0E7FD48461AF03CFF052017F01E
:10C31000E1FD28461AF03CFF052017F0DBFD4846FA
:10C320001AF036FF019B0BEB030408EB840428464C
:10C33000E37C227C002B0CBF1221322115F03EFF42
:10C34000E37C627C002B0CBF12213221484615F0A1
:10C3500035FF534B9F4200F08580524B9F4200F0C7
:10C360009580514B9F4200F08780BB884F4A504CCC
:10C3700023F440731B041B0CBB80019B9B443B8834
:10C3800008EB8B0843F0010398F812103B80BD883E
:10C3900002A8002918BF144626F0C0FE049A45489A
:10C3A000B2FBF4F325F03F05A0FB02122D04900C24
:10C3B0002D0C0543BD8039883F4C4FF496729BB2DB
:10C3C00002FB00F2002BA4FB020221F0010108BFD6
:10C3D00001239209090443F400430132090C398016
:10C3E0003A84BB833A88354B42F001023A803A885E
:10C3F000134043F480634FF480423B803A813B8892
:10C4000023F080031B041B0C3B809AF81A308DF834
:10C410000830002402A801258DF809408DF80A4053
:10C420008DF80B502EF0A8FE9DF80B209AF81930CD
:10C430008DF808308DF809408DF80A4062B95A0924
:10C44000203203F01F031E4905FA03F341F822309E
:10C4500007B0BDE8F08F704702A82EF08DFE07B040
:10C46000BDE8F08F174A136A43F4001313624FF4C8
:10C47000001026F09DFD78E7124A136A43F400038A
:10C4800013624FF4000026F093FD6EE70D4A136A25
:10C4900043F4800313624FF4800026F089FD64E7C3
:10C4A0000054004000580040005C0040009F240001
:10C4B000804F120083DE1B43D34D6210F5FBFFFF5C
:10C4C00000E100E000380240543600202DE9F04140
:10C4D0000678012E82B0054655D0022E59D18068CB
:10C4E00041F0800110B1046880886083686840F280
:10C4F000E93402E0002C00F098800689013C16F037
:10C50000020FA4B2F6D089B2818140F2E93102E093
:10C51000002900F08A800489013914F0010F89B2E2
:10C52000F6D0818981894FF0000C4FF47A714FF673
:10C53000FF764FF0FF0E03E0013989B2B1422CD0F3
:10C540000489A707F8D5A0F80CE04FF47A7102E04F
:10C55000B9B2B14221D00489E40701F1FF37F7D520
:10C560008489A4B20AB1147001320CF1010C634544
:10C57000E6D1AB68002B56D01A689B881383012044
:10C5800002B0BDE8F08190F90400441C01D00328FA
:10C5900006DD002002B0BDE8F0811BF069FEE8E78F
:10C5A0004FEAC00EDFF8BCC00EEB00070CEB8707AC
:10C5B0007C68002C48D06D793A626D004FF000081D
:10C5C000EDB2BD75F97587F81980BE763B767E753C
:10C5D00087F81480A388FA61990512D42388DA05B4
:10C5E0000BD44FF4805501E0013D2FD023889B05EB
:10C5F000FAD4238843F480732380A38843F44073E0
:10C60000A38086440CEB8E024FF4805401E0013C81
:10C6100013D0537D002BFAD10CEB8E0E9EF8140034
:10C6200080F00100B6E70120B4E7CDE900231BF05C
:10C630001FFE6868DDE9002374E7094A13880133A7
:10C640009BB21380FFF7F4FD2046A3E7044A13884A
:10C6500001339BB21380FFF7EBFD28469AE700BF3A
:10C66000D43C00205436002007B5032301AA002142
:10C67000FFF72CFF9DF805309DF804001B0243EAEC
:10C6800000439DF80600184303B05DF804FB08B5AD
:10C69000FFF7EAFF014B586008BD00BF18270020D4
:10C6A00008B5FFF7E1FF014B186008BD182700200F
:10C6B00007B506236A46F721FFF708FF9DF801300A
:10C6C0009DF800100B4A1B0143EA01339DF802104C
:10C6D00043EA1113D3609DF804309DF803101B0149
:10C6E00043EA01339DF8051043EA1113936003B048
:10C6F0005DF804FB1827002007B5032301AAF621E3
:10C70000FFF7E4FE9DF805309DF804201B0243EA84
:10C7100002439DF806201343054AB2F92020C2F1D6
:10C720000802D340034A536103B05DF804FB00BF25
:10C73000744000201827002007B5022301AAF62123
:10C74000FFF7C4FE9DF804209DF8053043EA02235C
:10C75000024A138203B05DF804FB00BF18270020D3
:10C7600070B582B00446062310306A464321FFF7B5
:10C77000ADFEC0B19DF804009DF800609DF8011069
:10C780009DF802509DF803209DF8053041EA0621EE
:10C7900043EA002342EA0522A4F85010A4F85220EC
:10C7A000A4F85430012002B070BD00BF2DE9F04F55
:10C7B00090F8653085B00546002B40F025825C4B33
:10C7C000686993F8603405F11006002B00F0B4801E
:10C7D000584B984200F0FB8103F58063984200F0CB
:10C7E000F681038823F040031B041B0C038003889D
:10C7F00023F038031B041B0C3822134303800388E7
:10C8000043F04003038095F85F30032B00F28D80E6
:10C8100095F86240012C00F00884A4F10204B4FAF7
:10C8200084F46409AB6913B11A689B88538340F29E
:10C83000E93304E0013B9BB2002B00F03D85028907
:10C840009107F7D51A23838140F2E93304E0013BD5
:10C850009BB2002B00F030850289D207F7D583897F
:10C8600040F2E93304E0013B9BB2002B00F020854D
:10C8700002899707F7D5848140F2E93304E0013B50
:10C880009BB2002B00F014850289D107F7D583896C
:10C89000AB6913B11A689B881383012017F01AFB48
:10C8A0006A69244B9A4200F0AA8303F580639A4296
:10C8B00000F0A583138823F040031B041B0C138096
:10C8C000138823F038031B041B0C08210B4313802F
:10C8D000138843F0400313803046062302AA432105
:10C8E000FFF7F4FD002800F0D1829DF80A609DF862
:10C8F0000B309DF808409DF809109DF80C009DF83C
:10C900000D2043EA06231BB2A5F852305BB241EA80
:10C91000042142EA00220133A5F85010A5F8542062
:10C9200000F0BA8205B0BDE8F08F00247AE700BFBE
:10C930001827002000380040AB4B984200F0AA8432
:10C9400003F58063984200F0A584038823F0400338
:10C950001B041B0C0380038823F038031B041B0CEF
:10C960004FF4807242F48072002A92FAA2F2B2FA74
:10C9700082F208BF4FF0FF32013A43EAC2039BB292
:10C9800003800388994CDFF874A2DFF868B2984FEF
:10C9900043F04003038080226B2130461BF084FC6F
:10C9A0009623DFF85CE2DFF85CC20093DBF804302A
:10C9B000C3F30803002B40F03C84EFF31183002BFA
:10C9C00040F037842068BA6823689842FAD1DCF8CE
:10C9D00000309A42F6D8DAF800804FF47A7101FB01
:10C9E00008F39B1AB3FBF8F301FB00304FF47A789D
:10C9F000DBF80430C3F30803002B40F0C683EFF3E9
:10CA00001183002B40F0C1832368B96822689342E8
:10CA1000FAD1DCF800209142F6D8DAF8009008FB51
:10CA200009F2521AB2FBF9F208FB03231B1AB3F501
:10CA30007A7FDDD3009B013B0093B7D103226821AD
:10CA400030461BF031FC6A4FDFF8B4E1DFF8B4C1C7
:10CA50004FF0960B674B5B68C3F30803002B40F065
:10CA6000C583EFF31183002B40F0C0832068BA68C0
:10CA700023689842FAD1DCF800309A42F6D8DAF806
:10CA800000804FF47A7101FB08F39B1AB3FBF8F3B3
:10CA900001FB00304FF47A78564B5B68C3F3080310
:10CAA000002B40F05183EFF31183002B40F04C83B7
:10CAB0002368B96822689342FAD1DCF800209142D9
:10CAC000F6D8DAF8009008FB09F2521AB2FBF9F234
:10CAD00008FB03231B1AB3F57A7FDDD3BBF1010BEF
:10CAE000B8D103226B2130461BF0DEFB0F2017F07C
:10CAF000F1F910226A2130461BF0D6FB0F2017F007
:10CB0000E9F95A466C2130461BF0CEFB0F2017F096
:10CB1000E1F995F86420192130461BF0C5FB0F2080
:10CB200017F0D8F918221B2130461BF0BDFB0F204F
:10CB300017F0D0F918221C2130461BF0B5FB0F204E
:10CB400017F0C8F91022372130461BF0ADFB0F203B
:10CB500017F0C0F90122382130461BF0A5FB0F2049
:10CB600017F0B8F96A69204B9A4200F0868303F502
:10CB700080639A4200F08183138823F040031B04F2
:10CB80001B0C1380138823F038031B041B0C042197
:10CB900041F48071002991FAA1F1B1FA81F108BF45
:10CBA0004FF0FF31013943EAC1039BB21380138870
:10CBB00043F040031380012017F08CF90E4A686996
:10CBC000012382F86034084B98427FF405AE038855
:10CBD00023F040031B041B0C0380038823F038035D
:10CBE0001B041B0C302208E6003800403085002072
:10CBF00010E000E000ED00E0182700203485002060
:10CC00002C850020388500201E09013E032E03F0EC
:10CC10000F0300F20182964A32F8160040FA03F23E
:10CC2000D40740F1F981012404FA03F3013B1840D1
:10CC30003AF0D2FC8F4B904A9B5D184412EBC00631
:10CC400000F0EA8120210023B171F37152F83030F5
:10CC50008A4903F13F4202F57E02920A895C01F0A3
:10CC60001F024909032904FA02F200F0688204292C
:10CC700000F06082022903D18149486C02434A6472
:10CC8000B288D1070BD5196821F003011960196822
:10CC90001960D96821F00301D960D968D960970774
:10CCA0000BD5196821F00C01196019681960D96851
:10CCB00021F00C01D960D968D96054070BD51968E7
:10CCC00021F03001196019681960D96821F030012C
:10CCD000D960D968D96010070BD5196821F0C00157
:10CCE000196019681960D96821F0C001D960D96844
:10CCF000D960D1060BD5196821F440711960196803
:10CD00001960D96821F44071D960D968D960970653
:10CD10000BD5196821F44061196019681960D96848
:10CD200021F44061D960D968D96054060BD51968DF
:10CD300021F44051196019681960D96821F44051F3
:10CD4000D960D968D96010060BD5196821F4404123
:10CD5000196019681960D96821F44041D960D9680F
:10CD6000D960D1050BD5196821F4403119601968D3
:10CD70001960D96821F44031D960D968D960970524
:10CD80000BD5196821F44021196019681960D96818
:10CD900021F44021D960D968D96054050BD51968B0
:10CDA00021F44011196019681960D96821F4401103
:10CDB000D960D968D96010050BD5196821F44001F4
:10CDC000196019681960D96821F44001D960D968DF
:10CDD000D960D1040BD5196821F040711960196828
:10CDE0001960D96821F04071D960D968D960970479
:10CDF0000BD5196821F04061196019681960D9686C
:10CE000021F04061D960D968D96054040BD5196804
:10CE100021F04051196019681960D96821F040511A
:10CE2000D960D968D96010040BD51A6822F0404245
:10CE30001A601A681A60DA6822F04042DA60DA682A
:10CE4000DA6029460F4B41F80C3F30462EF048FA85
:10CE5000B388B3FA83F3C3F11F03012212FA03F379
:10CE60003FF4ADAC08490A6813430B60A7E400BF68
:10CE700034C704083CC704083C8500206CC504087E
:10CE8000003802404D890008003C0140B5F952309D
:10CE90005BB201337FF446AD95F9503001337FF436
:10CEA00041AD0A23C94CDFF83CA3C94FC94DCA4E56
:10CEB00001932DF0CBFF4FF4FA73DFF82CE30093CE
:10CEC0004FF010087B68C3F30803002B40F0EE809E
:10CED000EFF31183002B40F0E9802068AA682368F3
:10CEE0009842FAD133689A42F7D8DAF800C04FF482
:10CEF0007A7101FB0CF39B1AB3FBFCF301FB0030CE
:10CF00004FF47A7C4FF001097B68C3F30803002BD0
:10CF100040F0AD80EFF31183002B40F0A880236830
:10CF2000A96822689342FAD132689142F7D8DAF8B8
:10CF300000200CFB02FBABEB0101B1FBF2F10CFB9F
:10CF400003131B1AB3F57A7FDED3009B013B0093DA
:10CF5000B8D107202DF0D6FD4FF47A73DFF888E2C0
:10CF600000934FF010087B68C3F30803002B40F0D8
:10CF7000BF80EFF31183002B40F0BA802068AA68CD
:10CF800023689842FAD133689A42F7D8DAF800C099
:10CF90004FF47A7101FB0CF39B1AB3FBFCF301FB1A
:10CFA00000304FF47A7C4FF001097B68C3F308032B
:10CFB000002B3DD1EFF31183002B39D12368A968F1
:10CFC00022689342FAD132689142F7D8DAF8002009
:10CFD0000CFB02FBABEB0101B1FBF2F10CFB031309
:10CFE0001B1AB3F57A7FE0D3009B013B0093BAD1C3
:10CFF000019B013B01937FF45CAFFEF719FE1388A0
:10D0000023F040031B041B0C1380138823F0380308
:10D010001B041B0C002159E42946704B41F80C3FBE
:10D0200000202EF05DF9FFF7CABB0724FFF7FABB1B
:10D03000EFF3118188F31288D5F808B02B68DB0371
:10D0400044BFCEF80090D5F808B02368DEF8002081
:10D05000C9B281F31188DAF8001013440CFB01F215
:10D06000A2EB0B02B2FBF1F20CFB0323B8E7EFF3E8
:10D07000118188F31288D5F808B02B68DB0344BF10
:10D08000CEF80090D5F808B02368DEF80020C9B2C9
:10D0900081F31188DAF8001013440CFB01F2A2EBC3
:10D0A0000B02B2FBF1F20CFB03234AE7EFF311830F
:10D0B00088F31288D5F808C02A68D20304D5012263
:10D0C000CEF80020D5F808C02068DEF80090DBB26A
:10D0D00083F31188DAF800104FF47A72484402FBA7
:10D0E00001F3A3EB0C03B3FBF1F302FB003007E702
:10D0F000EFF3118388F31288D5F808C02A68D203A9
:10D1000004D50122CEF80020D5F808C02068DEF84A
:10D110000090DBB283F31188DAF800104FF47A72D2
:10D12000484402FB01F3A3EB0C03B3FBF1F302FB56
:10D13000003036E72A49086B02430A63A0E5284914
:10D14000086C02430A649BE5EFF31181102383F31B
:10D150001288D7F808903B68DB0304D50123CEF88A
:10D160000030D7F808902368DEF80020C9B281F3B8
:10D170001188DAF80010134408FB01F2A2EB09024F
:10D18000B2FBF1F208FB0323A4E4EFF311811023B7
:10D1900083F31288D7F808903B68DB0304D501239A
:10D1A000CEF80030D7F808902368DEF80020C9B226
:10D1B00081F31188DAF80010134408FB01F2A2EBA6
:10D1C0000902B2FBF1F208FB03232FE430850020B3
:10D1D00000ED00E010E000E0388500204D890008F7
:10D1E00000380240348500202C850020EFF31183A5
:10D1F000102282F31288D7F808803A68D20304D547
:10D200000122CEF80020D7F808802068DEF80090D0
:10D21000DBB283F31188DAF800104FF47A724844D5
:10D2200002FB01F3A3EB0803B3FBF1F302FB0030B5
:10D2300030E4EFF31182102383F31288D7F80880CB
:10D240003B68D90304D50123CEF80030D7F8088015
:10D250002368DEF80000D2B282F31188DAF80010F9
:10D260004FF47A72184402FB01F3A3EB0803B3FBFB
:10D27000F1F302FB0030FFF7B9BB138823F0400342
:10D280001B041B0C1380138823F038031B041B0C96
:10D2900002217DE4038823F040031B041B0C038060
:10D2A000038823F038031B041B0C8022FFF75ABBB2
:10D2B0001AF0DEFFFFF7ECBA1AF0DAFF6869FFF741
:10D2C000CFBA00BF70B582B00446062308306A4664
:10D2D0003B21FFF7FBF8A8B19DF804009DF8006022
:10D2E0009DF801109DF802509DF803209DF805302F
:10D2F00041EA062143EA002342EA0522E182228331
:10D300006383012002B070BDF0B5C60033189B00E6
:10D31000244DEA585468A28A83B092B20192019ACD
:10D320002B4412F4706F1CBF01221A75019B13F479
:10D33000E06F07460CD1A38A3E4423F4706305EBEB
:10D3400086051B041B0C0022A3826A7503B0F0BD86
:10D35000238BA38823F480631B041B0CA380019BF5
:10D360009B05E8D423889805E5D42388D9050DD5F5
:10D370002388DA05FCD4238843F4007323802388B0
:10D380009B05FCD43846FEF753FFD4E7238843F4CB
:10D3900000732380A38823F440731B041B0CA38019
:10D3A000C9E700BF54360020F0B583B0441C8DF8A7
:10D3B000073001D0032802DD002003B0F0BDC70014
:10D3C000274E3B1806EB83035C68002CF4D0490021
:10D3D000C9B2997501250021DA755D7699761D76B9
:10D3E0005D751975A1880DF107028905C3E907224A
:10D3F00012D42388DA050BD44FF4805501E0013DA7
:10D4000025D023889B05FAD4238843F48073238096
:10D41000A38843F44073A380074406EB87024FF4CC
:10D42000805401E0013C09D0537D002BFAD106EB7A
:10D430008707387D80F0010003B0F0BD094A1388EA
:10D4400001339BB21380FEF7F3FE2046B5E7054A91
:10D45000138801339BB21380FEF7EAFE2846ACE73F
:10D4600054360020D43C00200378012B47D0022BF7
:10D4700043D183682DE9F04101F07F0113B11C68AD
:10D480009B88638305461746406840F2E93401E013
:10D49000002C3FD00689013C16F0020FA4B2F7D051
:10D4A00089B2818140F2E93101E0002932D003895B
:10D4B000013913F0010F89B2F7D0838940F2E931C5
:10D4C00000E021B30489013914F0020F89B2F8D0C9
:10D4D000BFB2878140F2E93300E0C3B10289013B6A
:10D4E00012F0010F9BB2F8D08389AB686BB11A6858
:10D4F0009B8813830120BDE8F0810020704713460C
:10D500000A46417990F904004EE70120F3E71AF04A
:10D51000AFFEEAE71AF0ACFE6868CFE701224821C7
:10D52000A2E7012258219FE73122F4219CE7044B16
:10D5300093F820209201343202F0FC02F42193E7A8
:10D54000744000202E22F4218EE700BF2DE9F04F19
:10D5500089B0039090F86500002840F03786039B5F
:10D5600093F85C30072B00F027861823CDE90433AD
:10D57000039BC64CC64EDFF82483C64F10331846B3
:10D5800080226B210293FFF76FFF6423DFF810E323
:10D59000C14801934FF01009DEF80430C3F30803CB
:10D5A000002B40F06284EFF31183002B40F05D8488
:10D5B0002568826823689D42FAD13B689A42F7D871
:10D5C000D6F800C04FF47A7101FB0CF39B1AB3FB41
:10D5D000FCF301FB05354FF47A7C4FF0010ADEF8CD
:10D5E0000430C3F30803002B40F0FF83EFF31183F3
:10D5F000002B40F0FA832368816822689342FAD1B5
:10D600003A689142F7D832680CFB02FBABEB0101A0
:10D61000B1FBF2F10CFB03135B1BB3F57A7FDED396
:10D62000019B013B0193B7D1072268210298DFF8E3
:10D630006C82984FFFF718FF6423DFF864E2964886
:10D6400001934FF01009DEF80430C3F30803002BF8
:10D6500040F0EA83EFF31183002B40F0E583256867
:10D66000826823689D42FAD13B689A42F7D8D6F87F
:10D6700000C04FF47A7101FB0CF39B1AB3FBFCF36F
:10D6800001FB05354FF47A7C4FF0010ADEF80430D7
:10D69000C3F30803002B40F08A83EFF31183002BC0
:10D6A00040F085832368816822689342FAD13A6802
:10D6B0009142F7D832680CFB02FBABEB0101B1FBE6
:10D6C000F2F10CFB03135B1BB3F57A7FDED3019BF6
:10D6D000013B0193B7D11A466B210298DFF8BC8158
:10D6E0006C4FFFF7C1FE6423DFF8B4E16A48019391
:10D6F0004FF01009DEF80430C3F30803002B40F0AC
:10D70000F783EFF31183002B40F0F28325688268E2
:10D7100023689D42FAD13B689A42F7D8D6F800C0F8
:10D720004FF47A7101FB0CF39B1AB3FBFCF301FB82
:10D7300005354FF47A7C4FF0010ADEF80430C3F36C
:10D740000803002B40F01583EFF31183002B40F00A
:10D7500010832368816822689342FAD13A68914223
:10D76000F7D832680CFB02FBABEB0101B1FBF2F125
:10D770000CFB03135B1BB3F57A7FDED3019B013BEC
:10D780000193B7D101226B210298DFF81081414F3C
:10D79000FFF76AFE0F23DFF808E13F4801934FF0DF
:10D7A0001009DEF80430C3F30803002B40F07F8338
:10D7B000EFF31183002B40F07A8325688268236899
:10D7C0009D42FAD13B689A42F7D8D6F800C04FF490
:10D7D0007A7101FB0CF39B1AB3FBFCF301FB0535DB
:10D7E0004FF47A7C4FF0010ADEF80430C3F30803EB
:10D7F000002B40F0A082EFF31183002B40F09B82BE
:10D800002368816822689342FAD13A689142F7D836
:10D8100032680CFB02FBABEB0101B1FBF2F10CFB3C
:10D8200003135B1BB3F57A7FDED3019B013B0193AE
:10D83000B7D1039A92F85F30032B09D992F863307D
:10D84000012B049B0CBF43F0010343F0020304933C
:10D850009DF810200298DFF844800E4F1B21FFF73F
:10D8600003FE0F23DFF838E00B4801934FF0100957
:10D87000DEF80430C3F30803002B40F07C83EFF3A1
:10D880001183002B40F077830CE000BF308500202F
:10D89000348500203885002010E000E02C85002031
:10D8A00000ED00E02568826823689D42FAD13B685C
:10D8B0009A42F7D8D6F800C04FF47A7101FB0CF306
:10D8C0009B1AB3FBFCF301FB05354FF47A7C4FF058
:10D8D000010ADEF80430C3F30803002B40F00D8288
:10D8E000EFF31183002B40F00882236881682268DF
:10D8F0009342FAD13A689142F7D832680CFB02FBA6
:10D90000ABEB0101B1FBF2F10CFB03135B1BB3F5B5
:10D910007A7FDED3019B013B0193A9D1059A02983E
:10D92000DFF81483C24F1C21FFF79EFD0F23DFF8A1
:10D930000CE3C04801934FF01009DEF80430C3F344
:10D940000803002B40F0F682EFF31183002B40F028
:10D95000F1822568826823689D42FAD13B689A4229
:10D96000F7D8D6F800C04FF47A7101FB0CF39B1A7C
:10D97000B3FBFCF301FB05354FF47A7C4FF0010A51
:10D98000DEF80430C3F30803002B40F09881EFF376
:10D990001183002B40F093812368816822689342B1
:10D9A000FAD13A689142F7D832680CFB02FBABEB34
:10D9B0000101B1FBF2F10CFB03135B1BB3F57A7FA2
:10D9C000DED3019B013B0193B7D1039A92F85F30FC
:10D9D000032B00F2EF8392F86220012A00F0EC8220
:10D9E000A2F10202B2FA82F252091A210298DFF879
:10D9F00048828F4FFFF738FD0F23DFF840E28D4854
:10DA000001934FF01009DEF80430C3F30803002B34
:10DA100040F04C83EFF31183002B40F047832568DF
:10DA2000826823689D42FAD13B689A42F7D8D6F8BB
:10DA300000C04FF47A7101FB0CF39B1AB3FBFCF3AB
:10DA400001FB05354FF47A7C4FF0010ADEF8043013
:10DA5000C3F30803002B40F00B83EFF31183002B7B
:10DA600040F006832368816822689342FAD13A68BD
:10DA70009142F7D832680CFB02FBABEB0101B1FB22
:10DA8000F2F10CFB03135B1BB3F57A7FDED3019B32
:10DA9000013B0193B7D1039B029893F86420DFF810
:10DAA0009881634F1921FFF7DFFC6423DFF88CE1D5
:10DAB000604801934FF01009DEF80430C3F3080307
:10DAC000002B40F03583EFF31183002B40F03083BF
:10DAD0002568826823689D42FAD13B689A42F7D84C
:10DAE000D6F800C04FF47A7101FB0CF39B1AB3FB1C
:10DAF000FCF301FB05354FF47A7C4FF0010ADEF8A8
:10DB00000430C3F30803002B40F09482EFF3118339
:10DB1000002B40F08F822368816822689342FAD1FB
:10DB20003A689142F7D832680CFB02FBABEB01017B
:10DB3000B1FBF2F10CFB03135B1BB3F57A7FDED371
:10DB4000019B013B0193B7D1102237210298DFF8E6
:10DB5000E880374FFFF788FC0F23DFF8E0E0354817
:10DB600001934FF01009DEF80430C3F30803002BD3
:10DB700040F0BD82EFF31183002B40F0B88225689E
:10DB8000826823689D42FAD13B689A42F7D8D6F85A
:10DB900000C04FF47A7101FB0CF39B1AB3FBFCF34A
:10DBA00001FB05354FF47A7C4FF0010ADEF80430B2
:10DBB000C3F30803002B40F01F82EFF31183002B07
:10DBC00040F01A822368816822689342FAD13A6849
:10DBD0009142F7D832680CFB02FBABEB0101B1FBC1
:10DBE000F2F10CFB03135B1BB3F57A7FDED3019BD1
:10DBF000013B0193B7D10298DFF83C800C4F012222
:10DC00003821FFF731FC0F23DFF830E0094801939A
:10DC10004FF01009DEF80430C3F30803002B40F086
:10DC2000A882EFF31183002B40F0A38208E000BF2D
:10DC30003885002010E000E02C85002000ED00E099
:10DC40002568826823689D42FAD13B689A42F7D8DA
:10DC5000D6F800C04FF47A7101FB0CF39B1AB3FBAA
:10DC6000FCF301FB05354FF47A7C4FF0010ADEF836
:10DC70000430C3F30803002B40F0A081EFF31183BD
:10DC8000002B40F09B812368816822689342FAD17F
:10DC90003A689142F7D832680CFB02FBABEB01010A
:10DCA000B1FBF2F10CFB03135B1BB3F57A7FDED300
:10DCB000019B013B0193ADD109B0BDE8F08FEFF3BB
:10DCC000118189F31288D0F808B00368DB0344BFE0
:10DCD000C8F800A0D0F808B02368D8F80020C9B26E
:10DCE00081F31188316813440CFB01F2A2EB0B02A3
:10DCF000B2FBF1F20CFB03235FE6EFF3118189F332
:10DD00001288D0F808B00368DB0344BFC8F800A04D
:10DD1000D0F808B02368D8F80020C9B281F3118880
:10DD2000316813440CFB01F2A2EB0B02B2FBF1F2DF
:10DD30000CFB0323EAE5EFF3118189F31288D0F895
:10DD400008B00368DB0344BFC8F800A0D0F808B0EF
:10DD50002368D8F80020C9B281F3118831681344D0
:10DD60000CFB01F2A2EB0B02B2FBF1F20CFB032362
:10DD700057E5EFF3118189F31288D0F808B00368F2
:10DD8000DB0344BFC8F800A0D0F808B02368D8F877
:10DD90000020C9B281F31188316813440CFB01F2F1
:10DDA000A2EB0B02B2FBF1F20CFB0323E2E4EFF374
:10DDB000118189F31288D0F808B00368DB0344BFEF
:10DDC000C8F800A0D0F808B02368D8F80020C9B27D
:10DDD00081F31188316813440CFB01F2A2EB0B02B2
:10DDE000B2FBF1F20CFB03236DE4EFF3118189F335
:10DDF0001288D0F808B00368DB0344BFC8F800A05D
:10DE0000D0F808B02368D8F80020C9B281F311888F
:10DE1000316813440CFB01F2A2EB0B02B2FBF1F2EE
:10DE20000CFB0323FFF7F8BBEFF3118389F3128890
:10DE3000D0F808C00268D20304D50122C8F8002037
:10DE4000D0F808C02568D8F800A0DBB283F31188A9
:10DE500031684FF47A72554402FB01F3A3EB0C03D3
:10DE6000B3FBF1F302FB05350CE4EFF3118389F307
:10DE70001288D0F808C00268D20304D50122C8F87D
:10DE80000020D0F808C02568D8F800A0DBB283F3E2
:10DE9000118831684FF47A72554402FB01F3A3EB09
:10DEA0000C03B3FBF1F302FB0535FFF794BBEFF373
:10DEB000118389F31288D0F808C00268D20304D510
:10DEC0000122C8F80020D0F808C02568D8F800A0C2
:10DED000DBB283F3118831684FF47A72554402FB48
:10DEE00001F3A3EB0C03B3FBF1F302FB053577E47D
:10DEF000EFF3118389F31288D0F808C00268D203C7
:10DF000004D50122C8F80020D0F808C02568D8F848
:10DF100000A0DBB283F3118831684FF47A72554464
:10DF200002FB01F3A3EB0C03B3FBF1F302FB05359A
:10DF3000FFF7FFBBEFF3118389F31288D0F808C015
:10DF40000268D20304D50122C8F80020D0F808C026
:10DF50002568D8F800A0DBB283F3118831684FF44C
:10DF60007A72554402FB01F3A3EB0C03B3FBF1F30C
:10DF700002FB053500E5EFF3118389F31288D0F831
:10DF800008C00268D20304D50122C8F80020D0F8E6
:10DF900008C02568D8F800A0DBB283F31188316887
:10DFA0004FF47A72554402FB01F3A3EB0C03B3FB6D
:10DFB000F1F302FB053588E4072216E5EFF3118142
:10DFC00089F31288D0F808B00368DB0344BFC8F8AF
:10DFD00000A0D0F808B02368D8F80020C9B281F3B7
:10DFE0001188316813440CFB01F2A2EB0B02B2FB67
:10DFF000F1F20CFB032357E6EFF3118189F312884A
:10E00000D0F808B00368DB0344BFC8F800A0D0F81C
:10E0100008B02368D8F80020C9B281F311883168AC
:10E0200013440CFB01F2A2EB0B02B2FBF1F20CFB6E
:10E030000323D8E5EFF3118189F31288D0F808B0F3
:10E040000368DB0344BFC8F800A0D0F808B0236819
:10E05000D8F80020C9B281F31188316813440CFB51
:10E0600001F2A2EB0B02B2FBF1F20CFB032363E51E
:10E07000EFF3118189F31288D0F808B00368DB034D
:10E0800044BFC8F800A0D0F808B02368D8F8002032
:10E09000C9B281F31188316813440CFB01F2A2EB81
:10E0A0000B02B2FBF1F20CFB0323ECE4EFF3118360
:10E0B00089F31288D0F808C00268D20304D501227F
:10E0C000C8F80020D0F808C02568D8F800A0DBB256
:10E0D00083F3118831684FF47A72554402FB01F3DF
:10E0E000A3EB0C03B3FBF1F302FB0535AAE4EFF35A
:10E0F000118389F31288D0F808C00268D20304D5CE
:10E100000122C8F80020D0F808C02568D8F800A07F
:10E11000DBB283F3118831684FF47A72554402FB05
:10E1200001F3A3EB0C03B3FBF1F302FB053539E577
:10E13000EFF3118389F31288D0F808C00268D20384
:10E1400004D50122C8F80020D0F808C02568D8F806
:10E1500000A0DBB283F3118831684FF47A72554422
:10E1600002FB01F3A3EB0C03B3FBF1F302FB053558
:10E17000C1E4EFF3118389F31288D0F808C0026874
:10E18000D20304D50122C8F80020D0F808C02568C1
:10E19000D8F800A0DBB283F3118831684FF47A72AB
:10E1A000554402FB01F3A3EB0C03B3FBF1F302FBB9
:10E1B000053558E5019A18E4039B93F86130002B6C
:10E1C00046D11023CDE90433FFF7D2B914F05CF93E
:10E1D000039B044603F10C0500283FD00068284942
:10E1E00000F13F4303F57E039A0A01238A5C02F0A3
:10E1F0001F01520920268B40032A4FF00001A6710F
:10E20000E17138D0042A31D0022A03D11D4A516C61
:10E210000B435364A388069306A90023079325F0B4
:10E2200045FB039A184BD360294620462DF058F839
:10E23000A388B3FA83F3C3F11F03012212FA03F395
:10E240003FF48DA911490A6813430B60FFF787B9A2
:10E2500018231021CDE90431FFF78AB91A460A4B79
:10E26000D36029462DF03CF8FFF779B9054A116BC8
:10E270000B431363CEE7034A116C0B431364C9E7E6
:10E280006CC50408003802404D890008003C01407C
:10E290002DE9F04F804B426983B09A42019000F023
:10E2A000D88003F580639A4200F0D380138823F06E
:10E2B00040031B041B0C1380138823F038031B043A
:10E2C0001B0C30210B431380138843F04003138051
:10E2D000012015F0FFFD019C2046FFF737F9A369E7
:10E2E00013B11A689B885383019B586940F2E93344
:10E2F00002E0002B00F0C7800289013B12F0020F00
:10E300009BB2F6D06A23838140F2E93302E0002B0E
:10E3100000F0B9800289013B12F0010F9BB2F6D0E8
:10E32000838940F2E93302E0002B00F0B1800289DA
:10E33000013B12F0020F9BB2F6D01023838140F212
:10E34000E93302E0002B00F0A3800289013B12F0C8
:10E35000010F9BB2F6D08389019B9B6913B11A68A8
:10E360009B88138364234D4CDFF83C91DFF83C819C
:10E370004B4DDFF83CA14B4E009315F059FD4FF487
:10E380007A774FF0100C4FF0010ED8F80430C3F339
:10E390000803002B3ED1EFF31183002B3AD1236801
:10E3A000A96822689342FAD132689142F7D8D9F825
:10E3B000002007FB02FBABEB0101B1FBF2F107FB15
:10E3C00003131B1AB3F57A7FDFD3009B013B009345
:10E3D000D3D1019B5A69304B9A4247D003F58063F1
:10E3E0009A4243D0138823F040031B041B0C138074
:10E3F000138823F038031B041B0C08210B431380E4
:10E400001388012043F04003138003B0BDE8F04FB0
:10E4100015F060BDEFF311818CF31288D5F808B0C8
:10E420002B68DB0344BFCAF800E0D5F808B02368C6
:10E43000DAF80020C9B281F31188D9F8001013442A
:10E4400007FB01F2A2EB0B02B2FBF1F207FB032385
:10E45000B7E7138823F040031B041B0C13801388B9
:10E4600023F038031B041B0C28212BE7138823F00F
:10E4700040031B041B0C1380138823F038031B0478
:10E480001B0C0021BAE719F0F3FE019B586948E71D
:10E4900019F0EEFE60E700BF003800403085002034
:10E4A00010E000E0388500203485002000ED00E019
:10E4B0002C8500200220FAF789BC00BF0220FEF75D
:10E4C00023BF00BF0120FAF781BC00BF0120FEF787
:10E4D0001BBF00BF0020FAF779BC00BF0020FEF789
:10E4E00013BF00BF044B187828B1044A12685207C2
:10E4F00044BF0020187070473E32002000200140C9
:10E5000043680B4A23F0407323F4807343F4807311
:10E51000436083681A4042F002028260C36A013994
:10E52000C9B223F4700343EA0153C362704700BFCA
:10E53000FDF7FFC01D4B1B68022B30B432D81C4ABC
:10E540001C4903EB43035B0098189B5A4288808860
:10E550004B60C1E90202B3FBF2F21748174D1849AC
:10E56000184B194C00FB02F22A60D1F8882042F4C3
:10E570007002C1F888201A68002042F001021A6077
:10E5800098601A6822F0847222F480321A605C600B
:10E590001A684FF0006422F480221A60D8608C6000
:10E5A00030BC7047034A5368D268D4E7C8C2002021
:10E5B000C89604080000002040420F00A0A20020DE
:10E5C00000ED00E00038024010300024D0E90920BE
:10E5D000101AB0FA80F04009704700BF017170470F
:10E5E00003799B070AD5436A8269D154436A01695A
:10E5F0000133B3FBF1F201FB12334362704700BFFA
:10E60000037913F0010317D0D0E90731C26810B4C1
:10E610005B1A541E23400BD043694C1C5B5CB4FB5B
:10E62000F2F102FB114202625DF8044BD8B270476E
:10E6300018465DF8044B704718467047037913F08D
:10E64000020308D0D0E909210369581E531A034078
:10E65000DBB2C01A70471846704700BF037913F049
:10E66000010306D0D0E90731C268581A531E18407A
:10E6700070471846704700BF10F8113C0133DBB2F9
:10E680000A2B00F8113C07D9044A10F8131C002388
:10E6900022F8113000F8113C704700BF303A0020DA
:10E6A000F0B45D4E5D4832785D4B5E4DDC6B2D788D
:10E6B0000132A0FB0270000900EB8000A2EB800099
:10E6C0001A683070914201EB04005C6811D293F833
:10E6D0004520002A4ED000F58030B0FBF5F0844292
:10E6E0000BD2041B4FF4803292FBF5F2A21A9A600F
:10E6F0000AE0B0FBF5F0844244D34FF4803292FB41
:10E70000F5F2121B02449A6040F68C240025A242C6
:10E71000C3E9001083F8455017D993F8402093F9C6
:10E7200042108A4256B241D0002093F9411083F83A
:10E7300043008A4247D00121002283F8426083F8D7
:10E74000441083F84020F0BC704793F8441000292F
:10E75000F9D0A2F2EF2040F2DA5188421AD893F8A9
:10E7600040100B2916D803EB81000131C26083F8F9
:10E770004010E8E7B0FBF5F08442BED2041BA21AB9
:10E780009A60C1E793F84520002AAAD1041BA21A77
:10E790009A60B9E7244A002102F1300083F844105E
:10E7A00042F8041F8242FBD1F0BC7047111F0829B8
:10E7B000BAD893F84310182926D8013183F84310AA
:10E7C00093F94110B5E793F844100029B3D0FAB19A
:10E7D0001649154C0FFA82FC084601EB4C0754F819
:10E7E000045F20F8025BB842F9D10B2A07DC10481D
:10E7F00001EB4C02002122F8021B9042FBD10D4993
:10E800000A7801320A7096E783F84160314690E752
:10E8100094460649EBE700BF842B0020CDCCCCCC3E
:10E8200094A100205C2400209CA10020303A00200C
:10E83000483A0020243A002030B40E4D0E4B2A787E
:10E840000E4C0132A3FB02031B09E06B03EB8303B5
:10E85000A2EB83034FF6FF72914200F101002B708F
:10E86000084408BF0123E06308BF84F8453030BC8A
:10E87000704700BF842B0020CDCCCCCC94A10020CD
:10E88000002800F03881B14B1A7CF0B4002A40F027
:10E890009D801968002201280A6043D093F828104F
:10E8A000002941D19969002202280A603AD093F8E0
:10E8B0004010002961D1196B002203280A6031D071
:10E8C00093F85810002940F09680996C0022042893
:10E8D0000A6027D093F87010002940F00D81196E5E
:10E8E000002205280A601DD093F88810002940F006
:10E8F0003981996F002206280A6013D093F8A0107E
:10E90000002940F05781D3F89010002207280A60B0
:10E9100008D093F8B810002940F0B980D3F8A83097
:10E9200000221A60F0BC7047DC69894DA10AA94237
:10E9300000F0B88140F2D580864DA94208D0864AC1
:10E94000914200F0AD814D3A914200F08D81FE225E
:10E95000EFF31181502585F31288804E676AA58AEE
:10E9600002EB820206EBC202013745F00105576255
:10E97000C9B2A58281F3118894E75C6B744DA10A3A
:10E98000A94200F0658140F23D81724DA94208D054
:10E99000714A914200F05A814D3A914200F08681CD
:10E9A000FE22EFF31181502585F312886B4E676AC2
:10E9B000A58A02EB820206EBC202013745F001058F
:10E9C0005762C9B2A58281F3118874E75C68604917
:10E9D000A20A8A4200F058813CD95E498A4200F07E
:10E9E000558110318A4200F04B814D398A4200F046
:10E9F0003781FE2136E0DC6C554DA10AA94200F0BA
:10EA0000578140F20881534DA94208D0524A9142A1
:10EA100000F022814D3A914200F04C81FE22EFF34A
:10EA20001181502585F312884C4E676AA58A02EB46
:10EA3000820206EBC202013745F001055762C9B2F6
:10EA4000A58281F31188996C002204280A607FF462
:10EA500041AF67E7B2F5801F00F0148101398A42A7
:10EA6000C7D10221EFF31182502585F312883B4E66
:10EA7000676AA58A01EB810106EBC101013745F008
:10EA800001054F62D2B2A58282F3118801E7D3F863
:10EA9000AC002F4C810AA14200F0248140F2CD80CD
:10EAA0002C4CA14208D02C4A914200F01F814D3AD3
:10EAB000914200F01981FE22EFF31181502484F37A
:10EAC0001288264D466A848A02EB820205EBC20553
:10EAD000013644F001046E62CAB2848282F3118866
:10EAE0001CE7B1F5801F00F0DF801D4A91427FF4E2
:10EAF0002EAF02222CE770475C6E154DA10AA94289
:10EB000000F0DC8040F29080124DA94208D0124AF9
:10EB1000914200F0A7804D3A914200F0CD80FE2254
:10EB2000EFF31181502585F312880C4E676AA58A90
:10EB300002EB820206EBC202013745F00105576283
:10EB4000C9B2A58281F31188C9E600BFE0A1002007
:10EB5000020010004000100050001000508F0020F4
:10EB600001001000DC6F624DA10AA94200F0AE80E6
:10EB70007ED9604DA94208D05F4A914200F0A28040
:10EB80004D3A914200F09C80FE22EFF31181502516
:10EB900085F31288594E676AA58A02EB820206EB5A
:10EBA000C202013745F001055762C9B2A58281F35F
:10EBB00011889EE6D3F894404D4DA10AA94200F079
:10EBC000898065D94B4DA94207D04B4A914200F04C
:10EBD00085804D3A91427FD0FE22EFF3118150257E
:10EBE00085F31288454E676AA58A02EB820206EB1E
:10EBF000C202013745F001055762C9B2A58281F30F
:10EC0000118880E6B1F5801F24D03D4A91427FF4FF
:10EC1000C7AE0222C5E6B1F5801F1FD0384A914227
:10EC20007FF4FCAE0222FAE6B1F5801F1ED0344A12
:10EC300091427FF474AF022272E7B1F5801F4FD08A
:10EC40002F4A91427FF437AF022235E70522A8E62A
:10EC50000322A6E60122A4E60522E0E60122DEE682
:10EC60000421FFE605225BE7042271E6012257E753
:10EC7000B1F5801F28D0224A914285D1022284E733
:10EC80000521EFE60121EDE60321EBE60021E9E6AF
:10EC9000B1F5801F1CD01A4A91429DD102229CE7F7
:10ECA000052255E6032253E6012251E6042278E6C6
:10ECB0000322B4E60422B2E6042231E703222FE75E
:10ECC000042262E7052260E701225EE703225CE797
:10ECD000012282E7032280E704227EE705227CE707
:10ECE0000122E9E60322E7E60422E5E60522E3E65F
:10ECF000020010004000100050001000508F002053
:10ED000001001000704700BF70B4150BC2F303245C
:10ED1000064605EB450504EB44044800C2F3031323
:10ED20001835183402F00F02356003EB430346F840
:10ED3000214002EB420201441833183246F82030D9
:10ED4000062046F8212070BC704700BF2DE9F04F27
:10ED500012F4004F14BF4FF00E0B4FF0070B12F4DC
:10ED6000804F14BF4FF00E0A4FF0070A12F4005FF5
:10ED700014BF4FF00E094FF0070912F4805F14BF63
:10ED80004FF00E084FF007084FEA410C12F4006FE5
:10ED900083B001EB0C0714BF4FF00E0E4FF0070EBF
:10EDA00012F4806F01EB070614BF0E2307238D19A1
:10EDB0000193034612F4007F01EB0504C3F800B091
:10EDC00018BF0E2043F821A008BF072043F82C905D
:10EDD00012F4807F01EB040C43F8278043F826E00F
:10EDE00001EB0C0714BF4FF00E084FF00708019E0F
:10EDF00043F8256012F0800F01EB070614BF4FF0B7
:10EE00000E0E4FF0070E12F0400F43F8240001EBF6
:10EE1000060514BF0E20072012F0200F43F82C80A7
:10EE200001EB050414BF4FF00E0C4FF0070C12F06D
:10EE3000100F43F827E043F8260018BF0E2701EB18
:10EE4000040008BF072712F0080F43F825C018BFB9
:10EE50000E2643F8247008BF07260C1812F0040F82
:10EE600043F8206018BF0E2501EB040008BF0725FA
:10EE700012F0020F43F82450014414BF0E2407245B
:10EE800012F0010F43F8204014BF0E220722122077
:10EE900043F8212003B0BDE8F08F00BF704700BFEA
:10EEA00070B4044600F16C06064D0FCD2D88258206
:10EEB00020606160A260E3601234B442F4D170BC9F
:10EEC000704700BF44930408034B33F8142F0280AB
:10EED0009B788370704700BF4493040807280AD8C2
:10EEE00000EB4000044B10B553F8304014B138F03B
:10EEF000D9FE206010BD70472899002070B50546E6
:10EF00006C0038F0CFFE2849631901EB43131E7BD8
:10EF100006B970BD254A566880B21EB1167B0EB97F
:10EF2000567B66BB2C4401EB4414214B227D20818F
:10EF300042EA400290B2021282EA1012424002F00B
:10EF40000F0242EA00121B781A480026267592B278
:10EF50000668DBB9602000FB051018300121B047BE
:10EF600021696368B1F82C216489DB682243A1F828
:10EF70002C2158601A6842F001021A6070BD2A44C0
:10EF8000907B0028CED001221A75CBE763682069F8
:10EF90005B7903F0FC030C3318440421B047236968
:10EFA0008000188170BD00BFD0A20020842B0020FB
:10EFB000CCA20020C4A2002038B500EB4000084DD0
:10EFC000C4002B1993ED027AD3ED037AE7EE007AB1
:10EFD000B0EE670A38F066FE2B59186038BD00BFE6
:10EFE000E0A10020F8B5A0F5197423796179DB0759
:10EFF00046D594F84832206C0BBB94F84B32012B69
:10F000003FD0002B41D194F84A3294F849629E4295
:10F010000CD9B4F85222012707FA03F501332A4329
:10F02000DDB2AE4292B2F7D8A4F852220123C9430E
:10F0300084F84B321940BDE8F8402CF035BF026827
:10F04000D36A5B08536294F85932012B07D094F8C5
:10F050004D3223B1B4F854320133A4F85432C943C9
:10F0600001F001012CF020FF0023012284F84B2243
:10F0700084F8493284F84A32A4F8523284F848328B
:10F08000F8BD94F8493284F84A32002384F84B32B0
:10F0900001F00101BDE8F8402CF006BF436CC06BE5
:10F0A0001BB11A7A012113F089B8012117F0CEBFE4
:10F0B00010B5437903F0200113F0010F036C0446EF
:10F0C0001A7A806B17D000290CBF4221022113F05D
:10F0D00075F8226C012384F84C32A4F84832517937
:10F0E00012688B40118C9BB221EA03011184118CB0
:10F0F0000B43138410BD00290CBF2221022113F001
:10F100005DF8E6E70A4B1A6810B41446B4FBF1F355
:10F11000B3F5803F07D3012CFAD96408B4FBF1F3AF
:10F12000B3F5803FF7D299B25DF8044B13F020BDE0
:10F13000A0A200208160006CE4E700BF4379C06BAF
:10F14000DB0748BF81F0010109B918F01BB818F0BE
:10F150001FB800BF38B5A0F517742379990747D4B5
:10F16000D80700D438BD94F84832002BFAD194F86F
:10F1700049320133DBB2092B84F8493270D00A2BB3
:10F18000F0D194F84B52B4F85232002D00F0A9801F
:10F19000990503F0010200F1AB80002A00F0A8807D
:10F1A0001A46E36A5208002B00F0AC80D0B2216B03
:10F1B000984794F84B5201220023954284F8493233
:10F1C00084F84822CED1617984F84B321140206C0A
:10F1D0002CF06AFE236C1A68597905FA01F3118C38
:10F1E0009BB221EA03011184118C0B43138438BDB7
:10F1F00094F84D226ABBD4E90950854294F84C1228
:10F2000046D0451CA369A5621B5C2069DBB2854220
:10F210004FEA430328BFA26243F400730A2001228D
:10F22000A4F8503284F84E0284F84D2211B161796D
:10F230000D073FD45A08A4F8502203F001012046DC
:10F24000FFF77CFF94F84E222379013A84F84E228E
:10F2500086E794F94E22002A63D184F84D227FE795
:10F2600094F84B32002B7FF47DAF94F84A32082B90
:10F270003FF678AFB4F85222012000FA03F10133CF
:10F280000A43D9B2082992B2F7D9A4F8522238BD5C
:10F2900000297FF465AF627912077FF561AF636C77
:10F2A000E06B5BB31A7A12F089FF2046FFF700FF8C
:10F2B000237955E7216CA06B0B684D79198CAA4016
:10F2C00021EA02021A841A8C92B21A84002117F0E1
:10F2D000BDFE002384F84C322046FFF7DFFE237981
:10F2E0003EE743F001029B05A4F852227FF559AF97
:10F2F000B4F856320133A4F856325CE7194617F0D9
:10F30000A5FED2E7E3696169D2B2CA54E369E16854
:10F3100094F84B520133B3FBF1F201FB1233E3617A
:10F3200049E7B4F8503285E710B5242013F0ACF863
:10F33000044618B1112200238271C3712021204696
:10F3400017F084FE0A2014F0C5FD204618F054FE84
:10F35000034B00280CBF012202221A7010BD00BF0F
:10F3600028BC0020F8B5044627F052FB0F4A104B8A
:10F37000B2F90260B2F900701D780E4900FB04F08A
:10F38000020B42F2107303FB02F393FBF7F33344D7
:10F3900081FB0310222D4FEAE373C3EBA00000D0E2
:10F3A000F8BD054B1A805880F8BD00BFAE5C002048
:10F3B000E584002067666666E88400206A4B1B7857
:10F3C000002B37D070B5694B694D9B79AC69A8614A
:10F3D000013B041B032B00F28180DFE803F04402B1
:10F3E000302A36F09FF8634B63491A784B8802F055
:10F3F0000102002878D06148AB65D0ED037A002A7D
:10F4000040F0868003FB04F007EE900ADFED5C6AB3
:10F410005C4AB8EEE77AD5ED157AE7EE267AC2E9CE
:10F420000033BDEEE77AC5ED157A85ED147A82EDED
:10F43000027A70BD534AC2E9003393607047524B61
:10F440001B681B01F5D5FF2025F03EF918B10378A4
:10F450000A2B6BD9002003464A4AC5E91703C2E9C3
:10F460000033906070BD494A494BD27933F812603D
:10F47000B6B23046FFF776FF07EE906AA862B8EEA4
:10F48000670A4448F8F7BCFDBCEEC00A10EE103A1B
:10F4900098B2FFF767FFA96AD5ED087ADFED386A01
:10F4A000384B3D4A686201FB04F407EE104AB8EE9F
:10F4B000C77A1860E7EE267A107859602228BDEEE8
:10F4C000E77AC5ED087A17EE102A83ED027A85ED0A
:10F4D000077AAED1314B9980DA8070BD294B00227A
:10F4E000C3E900229A6070BD274E3668F60682D5C1
:10F4F000AB65002A86D0B1F90010294A00FB01F063
:10F5000082FB0012C017C0EBA2100344AB6579E781
:10F51000FDEEE77A234E17EE900AA0F57A7000FB15
:10F5200000F2A6FB026200EB1210E4E71E4A1F4B3A
:10F5300051881A68D0ED027ADFED1D6A1D4C4368D0
:10F5400002FB01F207EE102AF8EEE77AB8EE477AEE
:10F55000A4FB0121E7EE267A03EBD103FDEEE77A67
:10F5600017EE900A78E700BF0A7B00201C7B002082
:10F57000842B0020DE7A0020B65C00200C7B00206B
:10F580002FE33E312C7B0020A0A000200C87002020
:10F5900030870020B02B0020E5840020E884002084
:10F5A000D34D62101F85EB51E07C00203085002098
:10F5B0007D219534CDCCCCCC2DE9F84F2DED028BAF
:10F5C000494B5B79012B35D0022B10D0474B0022E1
:10F5D0001A60474B1B78022B05D1444A454B518892
:10F5E000128819805A80BDEC028BBDE8F88F424B1F
:10F5F0001B681B01EDD5FF2025F066F800286ED0B2
:10F6000003780A2B5DD99FED3D0A00233C4C04F1A1
:10F610006800A4F86630F8F7F3FCBCEEC00A10EE00
:10F62000103A9BB2A4F86430304AB4F866105180A6
:10F630001380CEE7334A344B9278314D33F8128041
:10F64000324C334E1FFA88FB07EE90BA05F190005A
:10F65000B8EE670AF8F7D4FCB0EE408A27F0D8F984
:10F66000BCEEC80A94F800806378A77810EE102AE0
:10F6700008FB00F490B204FB00F4A6FB042444F65B
:10F68000FB79C3EB033A09EB5414B4FBFAF4B4FB73
:10F69000F7F4A4B2A5F88C4027F0BAF908FB0BF8F0
:10F6A00008FB00F3A6FB0323104A09EB5313B3FB3B
:10F6B000FAF3B3FBF7F39BB2A5F88E3053801480B6
:10F6C00087E7B0F902201349D31781FB0212C3EB7D
:10F6D000A2039BB207EE903AB8EE670A96E7084C91
:10F6E000B4F86430A0E700BF1C7B0020047B00203E
:10F6F000E5840020E8840020A0A000200000000095
:10F70000842B00200C87002030870020A95C00207B
:10F710001F85EB516766666670B52B4D2B4C2C49E7
:10F720006A792C4E2C4804230B7084F8B4300021E5
:10F730006423012A84F8BD30A4F8B610A4F8B810E8
:10F7400084F8BC10C4F8C010317001601FD0022AC8
:10F7500010D0A979214A00230129136084F8C4300C
:10F76000C2E9013321D0022903D11D4A2365C2E930
:10F77000013370BD2822E01838F080F944F620618A
:10F780009FED180A04F16800FAF774F8E1E72822FF
:10F7900004F18C0038F072F944F620619FED110AF3
:10F7A00004F19000FAF766F8D3E70F4AE361C2E983
:10F7B0000133D3609FED0D0A02F1100044F6206181
:10F7C000BDE87040FAF756B81C7B0020842B00205F
:10F7D000CC7D00200A7B0020047B00202C7B0020B5
:10F7E000D42B0020CDCCCC3DA02B0020CDCCCC3ECA
:10F7F0002DE9F84FAD4E3468E50500F1F880AC4ACC
:10F80000AC4B92F80090DFF8F08200221A70B9F148
:10F81000000F00F0FA800921A748FAF759FF0028E5
:10F8200000F0DB8044F01004A44AA54B1768346054
:10F8300017F48057B3F9065040F08D80A14B9B8A96
:10F84000AB4200F39F8044F040049F4B346093F838
:10F8500000B01BF0080F06D11E219748FAF738FFB9
:10F86000002800F0FE8024F08004984B1B88642B55
:10F87000974B1B688CBF44F4806424F48064580761
:10F8800004D5B8F8C620002A40F08180B8F8C82016
:10F89000002A7AD18F4BD3F8B03024F4006A002BC1
:10F8A00075D18D4CC6F800A004F17805234602E01E
:10F8B0000633AB421DD01A781F2AF9D19978DA782D
:10F8C000914202D35A79002AF2D01F217A48FAF7DE
:10F8D000FFFE20B1814B1B785A0740F1D580237879
:10F8E0004AF4007A0A2BC6F800A005D00634AC42D0
:10F8F00018D023780A2BF9D1A278E3789A4202D360
:10F900006379002BF2D0764B1B7F002B68D01BF065
:10F91000010F65D1714B1B789B0761D44AF4802A93
:10F92000C6F800A022216448FAF7D2FE90BBB9F1D4
:10F93000000F36D0BAF1000F4DD1002388F8CA303D
:10F9400014F076FAD8F8CC30C01A00284DDBBDE8A8
:10F95000F84F27F0F5BA18215748FAF7B9FE0028F2
:10F960007FF46CAF5F4B1A7B002A7FF467AF554979
:10F97000DA884B8A991AA942BFF665AF1344AB42A5
:10F980007FF761AF24F040045FE7990782D544F424
:10F99000006A86E74AF4003AC6F800A0B9F1000F01
:10F9A00019D1514B1C78002C51D1002F5CD1002172
:10F9B0004148FAF78DFE002839D0BAF1000FBCD0CB
:10F9C0004CB9002F65D030B92AF4002AC6F800A03F
:10F9D000BAF1000FB1D00223B0E724F0100423E7FE
:10F9E0002AF4802AC6F800A09CE7BDE8F88F3F4AB9
:10F9F0003F4B91791A684FF47A7303FB01F39342FA
:10FA00009CBF24F480743460F9E63A4A98F8C53013
:10FA10001578002B33D1002D33D049462648FAF70C
:10FA200057FE00286AD124F00804346029E02AF047
:10FA3000200A01462048C6F800A0FAF749FEBAF1AC
:10FA4000000F2ED0002CBED1002FBCD121E02AF413
:10FA5000002424F40064B4FA84F46409002FA6D0CE
:10FA600002E044F0800400E718211348FAF730FE62
:10FA7000A8B91C4B1B7B002B44D0074697E7002DF1
:10FA800048D188F8C550C6E62AF4007AC6F800A026
:10FA90002FE7002898D04AF4002333609BE7002723
:10FAA00085E700287FF449AF8EE700BF887D0020FE
:10FAB00020000020B0640020903E0020A0A0002084
:10FAC0007ABA002058AF0020A87D0020DA3C002040
:10FAD0001C720020E8990020A8410020DE7A002056
:10FAE000A86300200CC00020DC3E0020D898002035
:10FAF00030850020C54D0020842B002044F00804F0
:10FB00003460BEE72AF4002727F04007B7FA87F7EA
:10FB10007F094CE749460348FAF7DAFD0028B0D1DF
:10FB200081E700BF903E0020F8B55B4A1378D90703
:10FB300000D4F8BD23F00103137014F079F9574B8A
:10FB4000574D9A78C5F8D00002BB564B1B88002B46
:10FB500043D1554A554B1178186881F0010117F0CF
:10FB60001DFB534E534C33782BB123781BB1524BB2
:10FB70001B68DA043AD5514B1B6800229B062270A1
:10FB8000D7D40420BDE8F84027F044BC1B79022BF1
:10FB9000DBD04B4C23780B2B18D801229A4040F62F
:10FBA000030112EA0106D0D112F4C06F0ED0093B56
:10FBB000012B0BD845201FF005FFFF201FF002FF8F
:10FBC00040481FF0EBFE30461FF0FCFE3E4A3F4B24
:10FBD00012685A600B232370B7E73D4B5A69002A1D
:10FBE000BFD0196800220A605A74BAE7394B1F78EF
:10FBF00014F01EF93378002BBDD06A68002ABAD100
:10FC000000F51C5010300A214FF47A726860697355
:10FC1000AA60002F3BD03A4614212F4837F02EFF20
:10FC20002E4A1389012FB3FA83F34FEA53132ED0D0
:10FC3000B2F86810002918BF0023022F27D0B2F8AD
:10FC4000C810002918BF0023032F20D0B2F82811B4
:10FC5000002918BF0023042F19D0B2F888110029F9
:10FC600018BF0023052F12D0B2F8E811002918BFE1
:10FC70000023062F0BD0B2F84812002918BF00232A
:10FC8000072F04D0B2F8A822002A18BF002383F05F
:10FC900001032B736FE700BFDE7A0020B87D0020E0
:10FCA000842B0020088500200A8500200C85002078
:10FCB000BCA20020B0640020A0A00020887D00200D
:10FCC0000A5F0020E0D0040830850020C03E0020FC
:10FCD0001085002075710020922B0020D0A20020FA
:10FCE0002DE9F04FDFF8A4B2964ADBF8D410136880
:10FCF000954CCBF8D4002DED108B411A97B00B44E6
:10FD00000790136020466368089198470690002882
:10FD100000F09C80D4F8B050002384F86030002DAF
:10FD200040F04085894B0993987DB4F95010B4F99F
:10FD3000522094ED086AD4ED096AB4F954300028D1
:10FD400000F0908407EE901AB8EEE77A07EE902A5A
:10FD5000F8EEE77A37EE467A77EEE67A84ED0B7ABC
:10FD6000C4ED0C7A07EE903A94ED0A7A94F85E109E
:10FD70007748F8EEE77A77EEC77AC4ED0D7A0EF0A1
:10FD800093F8744B1D78002D00F02784724BDFF838
:10FD9000C091724E1F783568D4ED077A059309F546
:10FDA000B678B9EC018A132F05F000554FF0000A20
:10FDB00028EE278A42D0062F06D1B0EE480A37F047
:10FDC00071FF674B23F81A001DB1BAF1000F03F061
:10FDD000F582B0EE480AD4F8943140469847D4F8FA
:10FDE000043208F170009847D4F8B430A8F1E0006C
:10FDF0009847D4F82431A8F170009847356805F089
:10FE00000055B0EE408A0AF1010A2B46002D41F060
:10FE10009580059A1778032F01F08280BAF1030FBD
:10FE200089ED028A00F00984B9EC018AD4ED077AE1
:10FE3000132F08F1240828EE278ABCD104EB4A03CB
:10FE4000474AB3F8503022F81A30BDE7424B454AD2
:10FE50001F78059306921146D4ED0E7AD4ED0F6A01
:10FE600094ED107A94F8E8323F4D94F8F022C1ED09
:10FE7000017AC1ED026A81ED037A8BF8D8302A70DD
:10FE800053BBDBED374A394BCBED377A77EEA47AAB
:10FE9000DDED084ADBED383A9BED394A93ED005A27
:10FEA00093ED026AD3ED015ACBED386AFAEEEF4AD0
:10FEB00076EEA33A37EE044AA4EEA75AF0EE467A5D
:10FEC000E4EEA35AE4EE247A83ED005AC3ED015A1E
:10FED000C3ED027A8BED397A052F00F07583244A41
:10FEE000DBF8E8301178B3FBF1F201FB1232013399
:10FEF000CBF8E8304AB1059B1B78012B00F0578303
:10FF000017B0BDEC108BBDE8F08F1A4B1B78002B9F
:10FF100042D0194A194BB2F906209B8A9A423BDC1F
:10FF2000174B1B78012B33D0192B31D00E2B33D02C
:10FF3000082B31D01349144A0A91002393608B6037
:10FF40002CE000BF34BC0020E899002070A0002005
:10FF5000149A0020FD3B0020E5840020A0A0002092
:10FF6000E884002090A0002050C0002038BC002071
:10FF7000C23C0020200000207ABA002058AF0020A8
:10FF800060400020A0C100200C7B0020842B0020BA
:10FF9000D44B9B7B002BCDD0D34B0A9335F03AFD4D
:10FFA000059B1A78052A01F0298300230D932978EF
:10FFB0000991CE49CE4B096808911B78CD499BED3C
:10FFC0003BAA91ED008A002B40F0E082CA4B1B78DF
:10FFD000002B00F0DB82C949C94BD1ED006A1B88B8
:10FFE000DFEDC87AC849B0EEE67AA3F57A7327EE5A
:10FFF000277A07EE903AF8EEE77AF7EE009AE7EE06
:020000040801F1
:10000000879A2B2AC1ED009A01F07387BF4B9FEDB1
:10001000C06AD3ED007ABF4BDFF870A3D3ED006A5E
:10002000BD4DDFF86C93DFF86C83BC4FB7EE007A00
:1000300037EE488A10AE68EE277A0024F4EEC77ACD
:10004000F1EE10FA88BFF0EE477AF4EEC67AF1EEE0
:1000500010FAB8BFF0EE467A67EEA67A67EEA99A74
:10006000AF4AD9F80030BAEC010A10199847AD4AE6
:10007000D8F800301019984728463B689847243430
:100080006C2CA6EC010A05F10805E9D1A64B1A78FB
:10009000A64BD3ED005A069BD3ED018A002A40F00F
:1000A0004183F5EEC05AF1EE10FA3FDD994B9FED1A
:1000B000A06AD3ED007A069B67EE867AD3ED026ADA
:1000C00093ED037A27EEA86A66EEA76A67EE277AB1
:1000D0008DED136ACDED146ACDED157A954BDDEDFE
:1000E000136AD3ED025A93ED016AD3ED004A9DEDF8
:1000F000147ADDED157AB0EE655AA6EEC65AA6EE74
:10010000A56AF0EE645AE7EE455AA7EE245AF0EEDF
:10011000464AE7EEE54AE7EE865A83ED025AC3ED1A
:10012000014AC3ED005A002A40F01A83824F834AE5
:10013000834BB2F800A0804CDFF85C929FED81BA4F
:100140009FED81DADFED81AA9FED71CADFED80CAF4
:10015000DFED80BADFF844820C97002635461F4653
:100160007D4B3344D3ED007A0A9BF5EE407A33445D
:10017000F1EE10FA0B93D3ED00DA17D0774B33443E
:1001800093ED007A7DEEC76AB0EEE66AF4EEC67AC9
:10019000F1EE10FA08D5F5EEC06AF1EE10FACCBF18
:1001A00077EE87DA77EE67DAC3ED00DA40F6030C14
:1001B0001AEA0C0C00F09886022D00F09886684B25
:1001C000684953F825300898674A90F82D0081FB5C
:1001D00003E1DB17C3EB611307EE903A07EE100A59
:1001E0003244B8EEC76AF8EEE77AD2ED006A4342CD
:1001F00007EE103AE6EE267AB8EEC77AF4EEC77A42
:10020000F1EE10FA0AD407EE100AB8EE477AB4EE0F
:10021000E77AF1EE10FA88BFB0EE677A534B544993
:1002200003EB450331F91520B3F90C30D21A07EE70
:10023000902A40F60103F8EEE77A1AEA030FA7EED8
:10024000EC7A00F0E2854B4BD3ED00DA67EE2DDA65
:10025000494B9BF808011A78002800F05384002AC3
:1002600000F0B483089B3DEEE8EA93F84E10434B50
:10027000DBF8142107981B68821A9A4240F3AB837B
:10028000022901F049823E4B022D186840F09F87F9
:100290003C4B93ED007AF1EE477AF4EECE7AF1EE34
:1002A00010FA08DCB4EECE7AF1EE10FA8CBFF0EE64
:1002B0004E7AF0EE477A824284ED01CA01F3528110
:1002C000B0EE67EA0B4B93ED007AF7EE007AB4EEEE
:1002D000E77AF1EE10FA01F12181F0EE4CEA2A4BB7
:1002E0001A785DE018990020A0C10020B87F002096
:1002F000E9BF0020D8C000201DC10020D4C00020CC
:10030000BCBF00200AD7233CE8020020B8BF002071
:1003100000000000CCB90020A0BE00209CBE002040
:1003200030BE0020BCBE0020E8BF0020FCBF002083
:1003300035FA8E3C40C00020EC400020387B002085
:10034000742C0020000096428988083D0000C842B5
:10035000CDCCCC3D6F12033BACBF0020802C0020E5
:100360006C6300201F85EB5188C10020783B002082
:10037000747B002094BF0020C6630020C4BF00200F
:10038000C0BF0020DCBF00203CBF002094A00020A4
:100390002CBE0020B8BE002060B9002064BF002041
:1003A000CA4B93ED006A002A00F0B683022D00F0DC
:1003B000B586C74B03EBC50393ED008AD3ED016A05
:1003C0003DEEC87AF5EEC0EAA6EE878AF7EE007A2F
:1003D0003DEEC89AF1EE10FAB0EEC99AF1EE49FA84
:1003E00083ED008AEFEE8D7A05DDB5EEC0EAF1EE21
:1003F00010FA00F1D485F5EEC0EAF1EE10FA00F142
:10040000C885B44B1B78012B01F06780002B01F0ED
:1004100070809FEDB1FA002D02F09287F0EE007A25
:10042000B0EE487AAFEEA77AA9EE278AB4EEE87A62
:10043000F1EE10FA00F2CA84B4EEE88AF1EE10FA96
:1004400078EE687AC0F2CB84A44B3344D3ED006AD3
:10045000A34B66EEA75A93ED005AF5EEC05AF1EEA3
:1004600010FA58BF77EE687AB0EEE67A65EE275A52
:10047000F0EEE55AF4EEC75AF1EE10FA40F3AF840D
:10048000F1EE666AB0EE4E9A86EE85EAB5EEC06A87
:10049000F1EE10FA00F34A8398ED000A2AEE000A02
:1004A000022D20EE090A84ED000A00F04F86D8EDF7
:1004B000017A8C4B69EEA77AB0EE6E6AA7EE8F6A6E
:1004C000D3ED006AB1EE667AB4EEC76AF1EE10FAC7
:1004D000F0EE467A40F15E84834BD3ED006AF7EE8E
:1004E000007AF4EEE76AF1EE10FAACBF01230023C4
:1004F00043B1F0EEEEEAF0EEC77AF4EEEE7AF1EE0A
:1005000010FA01D584ED017AD8ED027A10ABF5EE40
:10051000C07A3344F1EE10FAD3ED008A00F3E083A1
:10052000724B84ED02CAB3F800A0714B3344C3EDA3
:10053000008ABAF1000F00F05D8384ED03CA099BC5
:10054000E7EC01DA002B40F0478394ED037A94ED59
:10055000006AD4ED017AD4ED026A76EE277A01358D
:1005600077EEA67A032D77EE877A08F11008C4EDAE
:10057000047A09F1240906F1040604F1140400F0D8
:100580000A86069B3344D3ED018AE9E5594B2B2AB1
:10059000D3ED009A7FF43AADDFF868819FED560AFB
:1005A00029EE800A37F07EFBA8F800002EE5534BB9
:1005B000534A19681288534BC96919805A8017B079
:1005C000BDEC108BBDE8F08F13F032FC079BDFF819
:1005D0003481C01AA8F8000081E44B4F4B4E07F558
:1005E000B67A07F18C0807F51379D4ED077AB7ECE2
:1005F000010AD4F8943120EE270A0AEB0500984747
:10060000434AD4F8043250199847D4F8B43008EB70
:10061000050098473F4AD4F8243150199847336869
:10062000980000F1A28424356C2D87ED020ADCD1FC
:10063000394A0592177803F00053099A927D22B146
:10064000364A1078002801F00B80099A527E002A61
:1006500040F06481002B40F09681314B069319469F
:10066000FFF7FABB2D48007800287FF46BAB606C75
:100670000D1A002DB8BF6D42B5F5804F41F39C8334
:1006800007EE900AA16CB8EEE77A501A002837EE10
:10069000467AB8BF4042B0F5804F84ED0B7A41F303
:1006A000878307EE901AE16CF8EEE77A5A1A002A6F
:1006B00077EEE67AB8BF5242B2F5804FC4ED0C7ABD
:1006C00041F373830B46FFF74DBB00BFFCBF002017
:1006D00040BF0020EBBF00200000000040C0002011
:1006E000CCB90020E0BF0020D8C00020387B00201B
:1006F000A02C0020E802002000007A44A4830020FF
:10070000DA3C0020E8840020149A0020A0A00020F9
:10071000F09B0020109B0020E58400209900002021
:1007200090A00020AD4BDFEDAE6A93ED006A069B12
:1007300026EE266A93ED027AD3ED037A66EE286AF6
:1007400027EE067A67EE867AF5EEC05AF1EE10FAD9
:10075000CDED136A8DED147ACDED157A3FF7BEAC71
:10076000A04FD7ED0B4A97ED066A97ED015AF0EED0
:10077000645AE6EE665AA4EEA66AF0EE466AB0EE59
:10078000456AA7EE656AE5EE075AB0EE467AA7EE2F
:10079000A67AE7EEC66AC7ED0B5A87ED017AC7ED78
:1007A000066AC4E4904A914E9148918B099205964D
:1007B000577832780368DFF84082069042F210766C
:1007C00006FB01F6B6FBF3F6B4F95030B8F90600B3
:1007D000B54207EE903A02F03C8194ED1A7AD4F8D3
:1007E0008410F8EEE77A4B1C37EE277A012BC4F819
:1007F000843084ED1A7A02F07A85D4ED1D5AD4ED56
:100800001F6A07EE103A37EEE56AB8EEC75A012DB7
:1008100086EE057A37EE257A77EEC77A84ED1E7A72
:10082000E7EE866A84ED1D7AF0EE667AC4ED206A02
:10083000C4ED1F6A02F08182B4F9523094ED1B7A44
:1008400007EE903AD4F89830F8EEE77A5A1C37EE73
:10085000277A012AC4F8982084ED1B7A02F01D82C1
:10086000D4ED225AD4ED246A07EE102A37EEE56A59
:10087000B8EEC75A012D86EE057A37EE257A77EE67
:10088000C77A84ED237AE7EE866A84ED227AF0EE69
:10089000667AC4ED256AC4ED246A02F07982B4F95F
:1008A000543094ED1C7A07EE903AD4F8AC30F8EE60
:1008B000E77A5A1C37EE277A012AC4F8AC2084ED77
:1008C0001C7A02F0FA80D4ED275AD4ED296A07EE9B
:1008D000102A37EEE56AB8EEC75A012D86EE057A82
:1008E00037EE257A77EEC77A84ED287AE6EE276A26
:1008F00084ED277AF0EE667AC4ED2A6AC4ED296A9F
:1009000002F06F82A8F80600D4F8B030059A069974
:100910001778013BC4F8B030FFF79EBA94F8E8228C
:100920005ABBD4ED107AFDEEE77A17EE902A002A32
:10093000B8BF5242099994F8F002B1F91A10002890
:1009400001F0858207EE901ADFED2A6AB8EEE77AA9
:1009500007EE902A37EE667AF8EEE77AB4EEE77A99
:10096000F1EE10FA42F3FF83D4F8EC22079844F634
:100970002061821A8A427FF76DAE002284F8F0224D
:10098000002B3FF46AAE94F8F43294F8F522013368
:10099000DBB29A4284F8F43202F0EA8094F8F83438
:1009A000002B3FF45AAE102F01F0868394F8F924FF
:1009B0004FF00009062A01F24885DFE812F06D0DBC
:1009C000E00CF10CA90B740C9C0E2C0EBCF1000F6A
:1009D00014D03DEEE8EAD4ED01EA80E4CCB9002081
:1009E00035FA8E3CEC40002070A00020E584002009
:1009F00090A000200000C842E8840020CF4BD049DE
:100A0000DFF888E331F91510DFF884A35EF806C03B
:100A1000DAED006A03EB4503F5EEC0DAB3F90C300A
:100A2000C91A07EE901AB8EEE70AF1EE10FA20EEB6
:100A30002C0AB7EE007AFFEE007AB5EEC00AD4BFFA
:100A4000F0EE675AF0EE475ACCBF4FF0010A4FF074
:100A5000FF3AF1EE10FAC8BFF0EE477ACCBF01239F
:100A60004FF0FF33B0EEC07ABCF1000F04D0D44594
:100A700002F035814EF80620B4EEE67AF1EE10FA77
:100A800002F32381AF4BF0EEE87A67EEAB7A93ED99
:100A9000007AB7EE006AF4EEC67AF1EE10FA28EEAC
:100AA000877A88BFF0EE467AB0EE408AA7EE878A52
:100AB000B5EEC08AF0EEC87AF1EE10FAF4EEE67AFE
:100AC000CCBF01234FF0FF33F1EE10FA02DD9A455F
:100AD00002F024814FF0000A002A42F02A819A4B4A
:100AE0001B78AB427FF475AF059B1B78272B02F078
:100AF0004A84022D7FF46DAF099B002B42F03986AA
:100B0000924B1A783DEEE8EA002A3FF464AF089B66
:100B100093F84E10FFF7ABBBB5EEC06AF1EE10FADA
:100B2000B0EE4E9AB0EE4EFA7FF7B6AC9BF81831A5
:100B3000002B3FF4B1AC864B864A334492ED007AE9
:100B4000D3ED007A844AE7EE0E7AD2ED006AB1EE78
:100B5000667AF4EEC77AF1EE10FA08D4F4EEE67A8B
:100B6000F1EE10FA8CBFB0EE667AB0EE677A7B4A8F
:100B700083ED007AD2ED006A27EE066AF1EE667A1E
:100B8000B4EEE76AF1EE10FA08D4B4EEE66AF1EEDC
:100B900010FA8CBFF0EE667AF0EE467A7DEEA7DAB8
:100BA0003FEE27FA002D7FF477AC059B1B78262BB0
:100BB00007D1B2EE040A27EE000A37F073F8684B4B
:100BC000D880684BD3ED007A0C9B6AEE277A67EEEB
:100BD000897AC3ED007A6AE4022D84ED01CA00F03F
:100BE000E581B0EE4C7A84ED00CA84ED02CA84ED52
:100BF00003CAACE498ED039AB5EEC09AF1EE10FA90
:100C00007FF79BAC584BD3ED007AF5EEC07AF1EE4E
:100C100010FA00F3EA80B7EE008A544BD7ED008A51
:100C20001B78AB427DEEE88A00F06981504A127869
:100C30007AB3504A1278012A00F04683022A25D15D
:100C400099ED027AD9ED067AD9ED056A99ED016A36
:100C5000D9ED035AC9ED066A67EE277A99ED077A4E
:100C6000C9ED058AE6EE267AD9ED086A99ED046A9F
:100C700089ED087AE5EEC77A99ED007AE6EE667AB4
:100C8000E8EE877AF0EE678AC9ED077AAB4200F0AA
:100C90000983394A394BD2ED007A1B7829EE279A1D
:100CA00029EE088A68EE288AC4ED038A002B3FF4F7
:100CB00046ACD4ED007A28EEA77AB5EEC07AF1EE14
:100CC00010FA7FF73CACF0EEE88AF0EEE77AF4EE4B
:100CD000E78AF1EE10FA7FF730AC84ED00CA2EE41B
:100CE000274B254A334493ED008A089B92ED007A06
:100CF00093F84E3038EE688A28EE078A2BB9214BDC
:100D0000B3F800A01AF4006F10D09BF8D83053B994
:100D10001D4B0E4A1B78127813F0010340F0058535
:100D2000002A40F05885174BB3F800A028EE0A8A35
:100D300068EE277AC4ED027AFFF7F7BB783B002014
:100D4000747B0020F0BF0020F4BF0020C6630020A9
:100D500040C00020CCB9002004C0002000C000200A
:100D6000E884002064BF002060BF00205DB900203F
:100D70005FB900205EB9002028BE0020EABF002035
:100D8000A02C0020387B0020DE7A0020902C002050
:100D9000ECBF0020F4EEE67AF1EE10FA8CBFB0EE74
:100DA000667AB0EE677A022D7FF496ABC34B1B7860
:100DB000012B02D0192B7FF48FABB4EECB9AF1EE5E
:100DC00010FACCBF01230023FFF792BBB4EEE88AF0
:100DD000F1EE10FA4CBF78EE687A77EE687AB0EEF2
:100DE0004E9AB0EE67EAFFF751BBB54B334493ED33
:100DF000008A27EE888AF7EE007AB4EEE78AF1EEF1
:100E000010FA88BFB0EE678A07E7AD4AB1F9003043
:100E1000D2ED007AD2ED016AB1F90220A949F4EECF
:100E2000E76AF1EE10FAB4BFB0EE676AB0EE666A38
:100E3000002BB8BF5B42002AB8BF52429342B8BFF2
:100E4000134607EE903AA04A0B7892ED005AF8EE5E
:100E5000E77A67EEAC7A002B00F0FE81B5EEC05A5F
:100E6000F1EE10FA40F32A82984BD3ED004AF5EEEA
:100E7000C04AF1EE10FA40F3218274EEE77ADFED1A
:100E8000945AC7EEA46A66EE255AF7EE007A85EE0C
:100E9000856AF4EEE76AF1EE10FA88BFF0EE676A51
:100EA000F5EEC06AF1EE10FA76EE277AB8BFF0EEF2
:100EB0004C6A66EEA77AB7EE006AF4EEC67AF1EEF7
:100EC00010FA88BFF0EE467AF5EEC07AF1EE10FA2D
:100ED000B8BFF0EE4C7A7F4BD3ED006A27EE267A4E
:100EE000E7EE27DAFFF7B4B9022D7FF4B1A9099B29
:100EF000002B794B18BFF0EE4CDA1A7802E6059A0F
:100F00001278282A7FF492AE28EEAA0A0B9336F0C4
:100F1000C9FE724A0B9B508088E605F000552B46AF
:100F2000B0EE480A0A9336F0BDFE6C4B03EB4A0163
:100F3000032721F8020C0A9BFEF770BFD9EDB37AA4
:100F4000D4F8743237EE808A08F1E00089EDB38A74
:100F50009847BAF1010FB0EE408A02F0D2823568AC
:100F600005F000552B46FEF754BF97EDB37AD4F841
:100F7000743277EE007A09EB0500C7EDB37A984733
:100F800024356C2D87ED020A7FF42FAB3368FFF711
:100F90004FBBB5EEC0EAF1EE10FA7FF732AA022A93
:100FA0007FF62FAAB0EE4EFAFFF735BA0C9F9BF8EA
:100FB0002831D7ED0C7AD7ED0A6A97ED0D7A77EEE6
:100FC000A67A77EE877AC7ED0E7A002B40F0E9809B
:100FD00000233B607B60BB60FB603B617B61BB616E
:100FE000FB613B627B62BB62FB623B637B63BB6317
:100FF000059B1B78052B00F0FA82394B1B78DB0729
:1010000008D5384B1B78DE0604D4374B5B78002BB1
:1010100040F0D686354C059B1B780022202BCBF860
:101020002C2100F04E81012B00F0D282052B00F024
:101030004484002306932378002B40F0B8802C4B87
:1010400007981B6893F8461031F0E8FD294B1B68A0
:10105000002B40F07381284B1B788BB1274D2878EB
:1010600058B1274F274E0024E0B23368B7EC010A8D
:101070009847287801348442F6DB234B1B68984755
:10108000059B1B78052B00F07682204A1478002CF3
:101090007EF433AF1E4DAA78002A40F0FB83059BF7
:1010A0001B78052B7EF429AF12F0C2FE0B4A059B7C
:1010B000001B1B78D080FEF720BF00BF20BE0020A1
:1010C00094C10020A0BF00209CBF0020A4BF00202E
:1010D0000000C8C298BF0020C6630020E88400203A
:1010E000DE7A0020A87D0020C23C0020B0640020F1
:1010F000B87F002024BE002054AF0020757100206E
:1011000028410020C0A20020C8A20020D47C0020DA
:10111000B87D0020000000005FED02DA022A3FF4F3
:1011200048A9042A3FF445A9B5EEC06AF1EE10FAC9
:1011300000F3988698ED000A2AEE000AB0EE4E9A67
:1011400020EE0E0AB0EE4EFA84ED000A664B6748B8
:101150001B689847664B93ED097A664B69EE876A80
:10116000B0EE6E6AA6EE8F6AD3ED007A0C9BB1EEFC
:10117000677AB4EEC76AF1EE10FA83ED0A0A3FF51A
:1011800015AEB4EEE76AF1EE10FA8CBFB0EE677AF6
:10119000B0EE467A0AE69BF828310C9F002B3FF40C
:1011A00017AF9BF8D830002B7FF412AF20E7524BDB
:1011B000524A1B781278DC0700F1A283002A3FF420
:1011C00045AF92004E494F4836F0F2FB3EE74E4B9A
:1011D0001B68990740F1E3814C4B4D49DFF858A15A
:1011E00031F915E0DAED00DA84ED01CA03EB450CC4
:1011F0006DEEACDABCF90CC0ACEB0E0C07EE90CA8D
:10120000F8EEE77A824267EEADDA3DEEE8EA7FF784
:1012100059A8B1F900C0B3F90C203E48ACEB02026A
:10122000002A0068B8BF52428242BFF656A8B1F900
:101230000220B3F90E30D31A002BB8BF5B4298429C
:101240007FF74BA80023344A1846137016F098FE17
:10125000D4ED01EAFFF743B8304BDFED316AD3ED4F
:10126000005AF4EEE65AF1EE10FA0FD5F7EE004A06
:1012700034EEE54ADFED2B6ADFED2B4A76EEE77AB6
:1012800064EE244AE7EEA45A25EE255AB5EEC05A7C
:10129000F1EE10FA12D9CAEE856AF7EE007AE6EEA0
:1012A000667A08E6059B1B78282B7FF4F2AC28EEC3
:1012B000AA0A36F0F7FC1D4B9880EAE4DFED1C7AB1
:1012C00009E61A4B1A60B4E61A4A02EBC502D2EDDF
:1012D000007A92ED017A78EEE78AE7EE287AF0EE6E
:1012E000678AC2ED007AD1E430BF002028BF002019
:1012F00064BF0020E0BF0020DE7A0020757100206E
:10130000DC3C0020284100201C720020783B00209B
:10131000747B0020C8BF0020C6630020A8BF002047
:10132000AE47813F00003443610BB63BE8840020A8
:1013300000000000D0B9002094BF0020B34F3B78DC
:10134000192B0AD80122B24902FA03F3194011B944
:10135000B04A134201D033F0AFFAAF4EAF4D33680D
:10136000980600F14182AE4CB4F90020B5F9043082
:10137000B5F906109A4203DB91420B46A8BF13460B
:10138000B4F90220B5F9100023809042B5F912306B
:1013900003DC9342A8BF13461846B4F90430B5F9EC
:1013A0001C1060809942B5F91E2003DC9A42A8BF48
:1013B0001A461146B4F90630B5F92820A1809A42A0
:1013C000B5F92A1003DC99420A46A8BF1A46B4F9B7
:1013D0000830B5F93410E2809942B5F9362003DCC3
:1013E0009A42A8BF1A461146B4F90A30B5F940200E
:1013F00021819A42B5F9421003DC99420A46A8BFFE
:101400001A46B4F90C30B5F94C1062819942B5F91D
:101410004E2003DC9A42A8BF1A461146B4F90E20AA
:10142000B5F95830A1819342B5F95A1003DC9142C5
:101430000B46A8BF1346E3817A4B9B8923B3DFF8A1
:101440001492DFF81482DFF8D4A109F1100539F9FC
:10145000023F00EE103A4046B8EEC00AF6F7D0FD63
:1014600036F020FCBAF90430BAF9062000B29842EE
:101470002ADB9042A8BF1046A945A9F8000008F150
:1014800024080AF10C0AE2D13B78013B182B00F248
:10149000F387DFE813F09305F107F107ED04F10797
:1014A000F107F107EF05F107F107F107F107F10780
:1014B000DE05C305F107F107F107F107ED040006AA
:1014C000F107F107DE059305A945A9F8003008F1F9
:1014D00024080AF10C0ABAD1D6E7B3EE0E7AB4EEBC
:1014E000C79AF1EE10FA7EF594AF27EE8EFAFEF76A
:1014F00092BF38EE68FAB0EECF7AB4EEC79AF1EE4A
:1015000010FA3EF786AFB5EEC0FAF1EE10FAACBFB6
:101510003FEE49FA39EE0FFAFEF77DBF069A424BCD
:10152000D2ED017A93ED007AF0EEE77AF4EEC77A25
:10153000F1EE10FA7EF5D1AED2ED027AF0EEE77A56
:10154000B4EEE77AF1EE10FA7EF7C7AED2ED037A89
:10155000F0EEE77AB4EEE77AF1EE10FA7EF7BDAE80
:10156000F0EE4E7A314B1B689A07B0EE67EA1BD556
:101570002F49304B4DE612F05BFC059B06991B781A
:101580002D4A401A052B908040F07A8112F050FCD1
:101590002A4B1B780446002B7FF481AD7AE582420A
:1015A00084ED01CA7EF78EAE254B26491A880023AA
:1015B0000B70002A40F0F684234A244B11781868F7
:1015C00081F0010115F0EAFDD4ED01EAFEF787BED6
:1015D00012F02EFC1E4ADBF83031126816490690D4
:1015E000C31A9A1ACBF83001CA808B8023E512F017
:1015F0001FFC0D9A104B801A5880FEE412F018FC64
:10160000059B0D901A78FEF7D2BC00BF20BE0020CB
:1016100030C1300102000002A0A00020A84200203A
:101620004841002018990020CCBF00201C720020E7
:10163000747B0020783B0020E8840020D47C0020CC
:1016400008850020C66300200A8500200C85002044
:10165000B0B80020464100208CBC002000D8F946DC
:10166000D4ED0E7A94F8E822D4ED076AFDEEE77A1D
:1016700017EE901A0029B8BF494207EE901AF8EE0B
:10168000E77A002A40F04C841FED0C6A94ED0F7A43
:101690008C4866EE866ABDEEC77AF4EEE76A17EE0E
:1016A000102AF1EE10FA4CBF01210021002AB8BF28
:1016B000524207EE902AF8EEE77A0078F4EEE76AF5
:1016C000D4ED107AFDEEE77AF1EE10FA17EE902ADB
:1016D00048BF41F00201002AB8BF524207EE902AEB
:1016E000F8EEE77AF4EEE76AF1EE10FA48BF41F05F
:1016F0000401014200F04F84012100220798C4F840
:10170000E40284F8E81284F8F022099A527E002A52
:101710003EF4A0AFFFF731B9012016F031FCDBF841
:101720001421079B9A1AFEF7AEBD674BD3ED006AF2
:10173000B7EE007AF4EEC76AF1EE10FAC0F2E58374
:10174000002A40F0E583614B93ED007AF0EEC86A21
:10175000F4EEC76AF1EE10FA7FF7E5AA5C4B93ED61
:10176000007AF0EEC96AF4EEC76AF1EE10FA7FF77C
:10177000DAAA0B99574B91ED007AD3ED006AB0EEDF
:10178000C77AB4EEE67AF1EE10FA7FF5CCAA0799A3
:10179000CBF81411504901230B70504B1B68934236
:1017A0007FF7C1AA4A4B93ED007AB0EEC99AB4EE26
:1017B000C79AF1EE10FA0DD40B9A464B92ED007ACF
:1017C000D3ED006AB0EEC77AB4EEE67AF1EE10FA25
:1017D0007FF7A9AA0023404A1846137016F0D0FBE1
:1017E000D8ED027AFFF79FBAEB7AFF2B00F09583D2
:1017F0003B4A12789A4240F290833A4A32F9139067
:10180000EB7D394CFF2BA4F8009001F04282344A62
:1018100012789A4241F23D82324A32F91380A4F89A
:1018200002800D2033F042F800283FF49DAD2F4B8D
:1018300095F916001A882E499BF834C1B3F902A015
:1018400095F90A3010FB02F281FB02E00011D21779
:10185000BCF1010F1FFA89F91FFA88F8A0EB020EFC
:1018600001F0518513FB0AF381FB0321DB17C3EB66
:1018700021139944F044A4F80090A4F8028073E581
:101880001C4A1478002C7EF438AB1B4DAA78002A31
:101890003EF433AB194E3378013B0A2B00F29487A8
:1018A000DFE813F0A607CA0886078F087708AE0896
:1018B0002708640842081208CE0712F0B9FA069009
:1018C000FFF7B9BBFC3B0020D8C00020D4BF0020EC
:1018D000D0BF0020D8BF0020C6630020C4BF0020B6
:1018E0003C6400207ABA002048410020747B00202C
:1018F0001F85EB51D47C0020B87D00200A5F0020BA
:10190000EA49EB4BD1ED017A93ED006A91ED005A73
:10191000D3ED016A91ED027AE64993ED024A4878E7
:10192000F5EEC07AF1EE10FAB5EEC05A26EE065A80
:10193000F7EE007AA6EEA65AFFEE005A54BFF0EE7C
:10194000654AF0EE674AF1EE10FAB5EEC07A54BF80
:10195000B0EE657AB0EE677AF1EE10FA54BFF0EEB1
:10196000653AF0EE673A58BFF0EE675AF1EEC57A85
:101970000028B4EEE66A18BFF0EE635AF1EE10FAF2
:10198000B4BFF0EE663AF0EE463AF4EEC43AF1EE49
:1019900010FA9FEDC95A4ABF9FEDC87ADFEDC75ACA
:1019A000F0EE447A27EE855A36EE263A9FEDC44A89
:1019B000C3EE053A48BFF0EE474AF4EEC43AF1EE02
:1019C00010FA0BD5B4EEE66ADFEDBC6AF1EE10FA60
:1019D000D8BFB0EE667A88BFF0EE664A9FEDB95A7E
:1019E0009FEDB66ADFEDB86A77EEC57AF4EEC67A97
:1019F000F1EE10FAB8BFF0EE467A67EEA67A002A4A
:101A00003FF424AB8B78B149DFEDB16A91ED005A18
:101A1000B048B14990ED004AD1ED003A06EE103AD7
:101A2000B8EE463AB3EE046A23EE263A35EE066A7D
:101A3000002B41F0F781A94BA949D3ED016AD3ED01
:101A4000022A93ED033A67EE266AE4EEA26AE5EE17
:101A5000836AB7EE003AF5EEC06AF1EE10FA48BFBD
:101A6000F0EE446A67EEA66AF4EEC36AF1EE10FA8D
:101A700088BFF0EE436AB0EE453AA3EEA63AB4EE64
:101A8000C36AF1EE10FAF0EE436A9ABFB3EE043A7D
:101A900076EEC36AF0EE446A012AC1ED006A3FF4B3
:101AA000D5AAD3ED056AD3ED062A93ED073A67EE82
:101AB000266AE4EEA26AE5EE836AB7EE003AF5EE36
:101AC000C06AF1EE10FA48BFF0EE446A67EEA66A0B
:101AD000F4EEC36AF1EE10FA88BFF0EE436AB0EE9E
:101AE000453AA3EEA63AB4EEC36AF1EE10FAF0EE70
:101AF000436A9ABFB3EE043A76EEC36AF0EE446AE4
:101B0000022AC1ED016A3FF4A1AAD3ED096AD3ED1F
:101B10000A2A93ED0B3A67EE266AE4EEA26AE5EE36
:101B2000836AB7EE003AF5EEC06AF1EE10FA48BFEC
:101B3000F0EE446A67EEA66AF4EEC36AF1EE10FABC
:101B400088BFF0EE436AB0EE453AA3EEA63AB4EE93
:101B5000C36AF1EE10FAF0EE436A9ABFB3EE043AAC
:101B600076EEC36AF0EE446A032AC1ED026A3FF4DE
:101B70006DAAD3ED0D6AD3ED0E2A93ED0F3A67EE01
:101B8000266AE4EEA26AE5EE836AB7EE003AF5EE65
:101B9000C06AF1EE10FA48BFF0EE446A67EEA66A3A
:101BA000F4EEC36AF1EE10FA88BFF0EE436AB0EECD
:101BB000453AA3EEA63AB4EEC36AF1EE10FAF0EE9F
:101BC000436A9ABFB3EE043A76EEC36AF0EE446A13
:101BD000042AC1ED036A3FF439AAD3ED116AD3EDAB
:101BE000122A93ED133A67EE266AE4EEA26AE5EE56
:101BF000836AB7EE003AF5EEC06AF1EE10FA48BF1C
:101C0000F0EE446A67EEA66AF4EEC36AF1EE10FAEB
:101C100088BFF0EE436AB0EE453AA3EEA63AB4EEC2
:101C2000C36AF1EE10FAF0EE436A9ABFB3EE043ADB
:101C300076EEC36AF0EE446A052AC1ED046A3FF409
:101C400005AAD3ED156AD3ED162A93ED173A67EE80
:101C5000266AE4EEA26AE5EE836AB7EE003AF5EE94
:101C6000C06AF1EE10FA48BFF0EE446A67EEA66A69
:101C7000F4EEC36AF1EE10FA88BFF0EE436AB0EEFC
:101C8000453AA3EEA63AB4EEC36AF1EE10FAF0EECE
:101C9000436A9ABFB3EE043A76EEC36AF0EE446A42
:101CA000062AC1ED056A3FF4D1A91BE088C10020D6
:101CB00094C1002060400020F304B53F0000000004
:101CC000D7B35D3F9A99193E9696963F2CC0002057
:101CD0000AD723BCDCC0002028C0002054C000204C
:101CE00028410020D3ED196AD3ED1A2A93ED1B3A4F
:101CF00067EE266AE4EEA26AE5EE836AB7EE003A82
:101D0000F5EEC06AF1EE10FA48BFF0EE446A67EEF5
:101D1000A66AF4EEC36AF1EE10FA88BFF0EE436AE9
:101D2000B0EE453AA3EEA63AB4EEC36AF1EE10FA6D
:101D3000F0EE436A9ABFB3EE043A76EEC36AF0EE71
:101D4000446A072AC1ED066A3FF480A9D3ED1D6AF3
:101D5000D3ED1E2A93ED1F3A27EE267AA4EEA27A3F
:101D6000A5EE837AB5EEC07AF1EE10FA48BFB0EE78
:101D7000447A67EE877AB7EE007AF4EEC77AF1EE2E
:101D800010FA88BFF0EE477AA3EEA75AB4EEC56A00
:101D9000F1EE10FAF0EE457A03D8B3EE044A37EECE
:101DA000C44A81ED074AFFF751B9E364FDF7DABF92
:101DB000A2641146FEF775BC61640846FEF760BC7C
:101DC0009BF82931C54C002B7FF425A92378002BE3
:101DD0007FF421A99BF82A31002B7FF41CA9C04B6A
:101DE0001B68DD0601F1858497ED097ADFEDBD7A88
:101DF000B0EEC77AB4EEE77AF1EE10FA81F2AC8376
:101E000097ED047AB0EEC77AB4EEE77AF1EE10FA05
:101E100081F2A28397ED0E7AB0EEC77AB4EEE77A3C
:101E2000F1EE10FA81F298830023CBF82C31059B58
:101E30001B78202B7FF4F7A8DBF82C31AA4A00335B
:101E400018BF0123012153801180FFF7F2B891429E
:101E5000BEF600AC01220799C4F8EC1284F8F02217
:101E6000FEF7F8BBB0EE4E9AB0EE4EFAFEF75EBE4D
:101E70009E4B1A6812B1B4F9081011609B69002BCF
:101E800001F07981B4F90A201A600327042202259F
:101E90003368990601F15E81DA027FF5DCA8944B84
:101EA000DC7B112C3FF7D7A8924F37F9143000EEA6
:101EB000103A2846B8EEC00AFDF710F8C4F112082F
:101EC0004FF0010905EB0900C14509EB0403C0B25D
:101ED00009F101093FF4BFA837F9133000EE103AB9
:101EE000B8EEC00AFCF7FAFFB9F10E0FEAD1FFF71E
:101EF000B2B89FED810ADFF8F08126EE800A35F056
:101F0000D1FEA8F80200FEF749BB002A3EF40BAF51
:101F1000DBF81421079B9A1A3FE4B5F908906FE4A7
:101F20009FED767A66EE876AF4EEE76AF1EE10FAD4
:101F300041F31481D4ED0F7AFDEEE77A17EE902A83
:101F4000002AB8BF524207EE902AF8EEE77AF4EE84
:101F5000E76AF1EE10FA41F30181D4ED107AFDEE5B
:101F6000E77A17EE902A002AB8BF524207EE902A6D
:101F7000F8EEE77AF4EEE76AF1EE10FA41F3EE805C
:101F8000D4F8E412079E4CF25035711AA9427FF73B
:101F9000BCAB84F8E8020999497E00293EF45AABAB
:101FA000FEF7C8BC56494A69002A3EF496A90A6859
:101FB000F0EE4CEA13604B74FEF791B94C4B4B4A70
:101FC0009B7B1268002B41F0B2814E4B1B7813F0C3
:101FD000010341F0AC81002A01F08B8213600120E3
:101FE0003368990603D43A78052A41F0C180851CEC
:101FF000471CEDB2FFB2B4F9003000EE103AB8EE73
:10200000C00AFCF76BFFB4F9023000EE103A384614
:10201000B8EEC00AFCF762FF33683DE7334B1A683D
:1020200012B1B4F9001011609A6912B1B4F902103A
:1020300011601A6B12B1B4F9041011609B6C002B83
:1020400001F05A82B4F906201A60052706220425F9
:102050001EE7DFF8B490002539F9023F00EE103A90
:10206000E8B2B8EEC00A0135FCF738FF062DF3D10F
:102070002846B5E71D4B1A6812B1B4F90610116075
:102080009B69002B01F07780B4F908201A600327C0
:1020900004220225FCE6DFF87490002539F9023BA2
:1020A00000EE103AE8B2B8EEC00A0135FCF716FFB0
:1020B000042DF3D1284693E711F0BAFE059B1F7853
:1020C000102F05BFDFF8208094F8F92494F8F92444
:1020D000A8F800208146FEF76DBC00BFB064002068
:1020E000A0A0002000001644E884002028990020C9
:1020F000189900207ABA002000007A440008ED46C2
:1021000010850020DE7A00204A4100204E41002048
:10211000DA4B1A46B2EC011A93ED033AD2ED002ADB
:10212000D3ED094AD3ED021A93ED082AD3ED053A0F
:1021300093ED074A93ED0B5AD3ED0D5A93ED0F6AC9
:10214000D3ED116A93ED137AD3ED157A93ED049ADA
:10215000D3ED068A93ED0A0AD3ED0C0A93ED0E8AAD
:1021600062EEA22A23EE033A64EEA44AE1EE012ACB
:10217000102FA1EEA13AE2EE024A93ED101A93ED70
:10218000142AD3ED121A63EEA33A24EE044A25EE84
:10219000055A65EEA55A26EE066A66EEA66A27EE91
:1021A000077A67EEA77AE9EE093AE2EE027AA8EE3C
:1021B000A84AA0EE005AE0EEA05AA8EE086AE1EEA6
:1021C000016AA1EEA17AB1EEE22AF1EEC32AB1EEE4
:1021D000E33AF1EEC43AB1EEE44AF1EEC54AB1EEAB
:1021E000E55AF1EEC65AB1EEE66AF1EEC76AB1EE13
:1021F000E77A03ED1E3A43ED1D3A03ED1C4A43ED29
:102200001B4A03ED1A5A43ED195A03ED186A43EDC0
:10221000176A03ED202A43ED1F2A03ED167AD3ED4A
:10222000175A93ED196AD3ED1B6A93ED1D7AD3ED1E
:102230001F7A93ED1E5A93ED163AD3ED183A93EDAB
:102240001A4AD3ED1C4A65EEA55A26EE066A66EEDA
:10225000A66A27EE077A67EEA77AE3EE035AA3EEA3
:10226000A36AE4EE046AA4EEA47AE5EE057AB1EE80
:10227000E55AF1EEC65AB1EEE66AF1EEC76AB1EE82
:10228000E77A03ED155A43ED145A03ED136A43ED53
:10229000126A03ED117A01F0098294F8F9240132EF
:1022A000D2B284F8F9247649764BB1F800801B78D5
:1022B00007EE908A591C0F29F8EE674A01F39D80BA
:1022C0000C2B04EB830503F10200DFED6F5A00F2E3
:1022D000578705F2145503F5A373D5ED007A069ED2
:1022E000B0EE656A04EB830300252EE027EEA77AA3
:1022F000B4EEE65A27EE277A66EEA67AF1EE10FAE9
:1023000036EEA64A00F10101A7EEA67A27D4D3ED56
:10231000017A26EEA67AB4EEE74A67EE266A27EE41
:10232000A77AF1EE10FAE7EE876A08D507EE101AE1
:10233000B8EEC77A36EE266AE6EE875A35460230A0
:102340000E2803F1080300F31E87D3ED006A37EE71
:10235000A75A26EEA67A002DC8D027EE267AD3ED0E
:10236000017A05EE100A67EEA76AB8EEC55A36EE96
:10237000076A66EEA76AE5EE075A411CD6E7D4F86D
:102380000425B4F80815414834F08AFB059B1F78F2
:10239000102F01F0978194F8F934013384F8F9345F
:1023A0003A4BB4F8FC04D4F810251946B1EC016A94
:1023B000D1ED007A77EEA77AF0EE006AB0EE677A98
:1023C000A6EE267A013803EBC001D6EE267A08394C
:1023D0001032F6EE003A27EE237A67EEA37A83ED09
:1023E000207AC3ED217A103391ED027A91ED036AE0
:1023F00053ED016A53ED027A52ED014A12ED025A91
:1024000037EE674A76EEC65A77EE277AE4EE845ABC
:102410000138A1F10801E5EE047A02F1080203F1A6
:10242000080336EE267AE4EE877AE5EE475A67EE41
:10243000A37A25EEA37AC3ED1C7A83ED1D7AD3D15E
:10244000102F00F0448794F8F924114B0693114B98
:1024500094F8F8140132A3FB0203D01A03EB5003E3
:102460009B08C3EBC3030139D31A84F8F81484F82A
:10247000F9340699FDF7F0BC0020B1E57C9F0020FF
:102480000C3C00200E3C002000000000FC9E0020C0
:1024900090A0002025499224B4F8FC14DB48D4F81D
:1024A00000254FEA510E4FEA8E0600EB8105C90860
:1024B00006EB000300F0A08003EB011C1036A91905
:1024C0000CF1100C1030103302F1100705F110065A
:1024D00016ED031A16ED042A50ED041A50ED030A06
:1024E00016ED015A16ED026A50ED025A50ED014AFE
:1024F00051ED042A51ED033A51ED026A13ED043A0D
:1025000013ED034A13ED027A53ED017A11ED010A3E
:1025100071EE828A30EE818A40ED048A00ED038AF2
:1025200075EE868A34EE858A40ED028A00ED018AD6
:1025300073EE228A34EE238A43ED048A03ED038A84
:1025400077EE268A37EE808A43ED028A03ED018A10
:1025500033EEC44A31EEC22A57ED033A70EEC11A87
:1025600032EEC33A23EEC28A57ED042A61EEA30A83
:1025700022EEC41AA1EEA28A10339C4563EE221A01
:10258000A3EE231A00F1100007F11007E4EE231A5E
:1025900006F1100601F11001E2EE220A06ED078AAB
:1025A00046ED080A01ED081A41ED071A35EEC66A34
:1025B00036EEC77A74EEC55A57ED056A17ED065A1E
:1025C00070EE677A25EEA63A66EEC63A25EE674AC1
:1025D00067EE054AE5EE853AA6EE053AA7EE264AED
:1025E000E7EEA64A06ED063A46ED053A01ED064A43
:1025F00041ED054A7FF46CAF1FFA8EF631468348F1
:1026000029F072F831462846D4F8002529F06CF8F4
:10261000059B1F7814E77E4A94F8FA34069294F8E2
:10262000742302F1DE05C2F12002D0B205EB4313A0
:10263000860804EB830500F0DE87360106F1100CF6
:102640007449754AAC4405F1100313ED024A13EDC9
:10265000035A13ED017A13ED046A51ED024A51ED6C
:10266000035A51ED046A51ED017A64EE244A65EE95
:10267000255A66EE266A67EE277A10339C4542EDAE
:10268000024A42ED035A42ED046A42ED017A01F139
:10269000100102F11002D8D1604B5C4935449A19FF
:1026A0000E4410F003011BD095ED007AD2ED007AB4
:1026B00067EE877A0129C6ED007A11D095ED017A8F
:1026C000D2ED017A67EE877A0229C6ED017A07D04A
:1026D00095ED027AD2ED027A67EE877AC6ED027A3C
:1026E00094F87453002D40F08B86102F00F018875B
:1026F00094F8F924ABE694F8FA54494A04EB4503FC
:10270000D2ED007AB3F8803608EE103AB8EEC87A07
:1027100067EE277A17EE900A34F08EFB0022414BC9
:1027200006460F4634F066FE08B93E4F002639468D
:10273000304634F0B1FE07EE900AB8EE480A67EE74
:10274000E70A394B324A0692E0EE000A05EBC5056E
:1027500003EB850567EE807A2846C7EEA00A11686C
:10276000D5F818A0D5F81C802E6A95ED058A29F0B9
:102770002BFE059B85ED058A1F78C5F818A0102F44
:10278000C5F81C802E6200F0858794F8FA34274A39
:1027900094F8F9140133A2FB0302520802EB42023F
:1027A0009B1ADBB2013184F8FA3484F8F91436E765
:1027B0001F4FDFF888801DF0C1F87B68D8F8002033
:1027C00064339342C0F01C872B79012B00F0A98061
:1027D000022B7EF464AC3378012B7EF460AC154B95
:1027E0001B78002B7EF45BAC0BF01AF9FEF757BC9C
:1027F000114B1B78DB0700F12D872B79012B00F0A3
:10280000EB85022B7EF44BACE9E700BFFC9E002079
:1028100090A00020203C00200C9F0020103C0020B5
:10282000903C002000405A40609C0020ABAAAAAA1D
:10283000C03E002071400020DE7A0020308500205C
:10284000B84BDFF828835B68D8F80010C8338B4298
:1028500004D31DF093F80028B6D0AA78032A00F01C
:1028600054872B79012293423270CAD1AE4B1B7828
:10287000D80740F1B385DBF83811D8F80020337859
:102880009142A9D8012B3EF40AACA84F3A78002A0D
:102890003EF405AC0B2B0DD801229A4040F6030103
:1028A00012EA01050CD112F4C06F03D0093B012BD1
:1028B00040F273879B4BD8F800205A600B2333708B
:1028C00000233B70FEF7EBBB994B1B78002B00F00D
:1028D0000B86162031F0EAFF002840F00586934B66
:1028E0001B78002B40F00086092333700AF01AF998
:1028F0006AE71DF023F88F4B052000210090A3F11B
:102900000802CDE9011153200AF078FE00287FF477
:102910005BAF844A0823106033702B79012B7EF45F
:10292000BEABDFF84882A1E7162031F0BFFF0028D8
:10293000DCD0814B1B88002BD8D1804B45201F68F1
:102940001DF040F80E201DF03DF8384609F0F8FF64
:10295000079F384609F0F4FF794A7A4B12681A60EB
:1029600038460A2333700BF067FDBFE71CF0E6FF23
:102970000AF00EF900283FF427AF1CF0FFFF0028F3
:102980003FF422AF6E4A6F4B12681A600A2333700D
:10299000C3E71CF0D3FF6C4B022000210090A3F191
:1029A0000802CDE9011148200AF028FE00287FF432
:1029B0000BAF5C4B4FF0FF3106221860596032704C
:1029C000ABE71CF0BBFF614A0292A2F10C03292184
:1029D00001930091A2F10A035021163A49200AF00E
:1029E0000DFE00287FF4F0AE594B1B681F061AD568
:1029F0004C4B4FF0FF3105221860596032708CE764
:102A00001CF09CFF534A0292A2F10C030721019390
:102A10000091A2F108030021143A47200AF0EEFDCC
:102A200000287FF4D1AE3F4B00224FF0FF311A60F7
:102A300007225960327070E7DFF83081394AD8F8E0
:102A40000030536044490023136003220B6032704E
:102A500063E7F8EEE77A012300219D42C4ED1A7A7C
:102A6000C4ED1E7AC4ED1D7A2162E167C4F884309A
:102A700000F04684B4F9523007EE903A0122F8EEA5
:102A8000E77A00239542C4ED1B7AC4ED237AC4EDA6
:102A9000227A6362C4F89030C4F8982000F007816D
:102AA000B4F9543007EE903AF8EEE77A00220123A9
:102AB000C4ED1C7AA262C4F8AC300023012DC4ED31
:102AC000287AC4ED277AC4F8A4307DF41BAF07EE52
:102AD000906AD4ED1C5A099BDFED206AB3F91430DB
:102AE0001F4AA8F80600B8EEE76A07EE103AC5EEEE
:102AF000867A1C4B11781B680022B8EEC77AE7EE85
:102B0000667AC4ED0A7A9A62C3E90B2229B1164BA0
:102B10001B6833F400637DF4F7AE012024F07AFCE7
:102B2000FDF7F2BEC03E0020DE7A0020714000209A
:102B30006340002004960408AC3E0020A83E00201C
:102B40009C3E0020983E0020A0950408C2930408F3
:102B5000A0A00020BC950408806400200AD7233C74
:102B6000FE3B0020A4830020887D002030850020CB
:102B700094EDBE8AD4EDBF6A94EDC70AD4EDC24A83
:102B800094EDC87A94EDC35AD4EDC67AD4EDC55A03
:102B900094EDC46A94F87453DFF8848268EE266A70
:102BA00004EB8503A4EEA60A00220F2FA5EE267AD9
:102BB00084F8F422B8F9040083EDDE0A67EEC07AE7
:102BC000A5EEC07AE6EE267A84EDC77AC4EDC87A1F
:102BD00000F0B38594EDC05AD4EDC10AD4EDD04ACB
:102BE00094EDD97A94EDCB1AD4EDD41AD4EDD15A10
:102BF00094EDD54AD4EDDA6A94EDCC2A94EDCF6AFF
:102C0000D4EDD87AD4EDCE2A94EDCD3AD4EDD73A9E
:102C1000A8F8040028EE055A28EE208AE1EE054ABD
:102C200004EB850105F16002A8EE217A0C23013541
:102C3000E8EE046A04EB820205F01F05E2EE055A95
:102C400084F8F834002326EE646A67EEC77A94EDC0
:102C5000D64AC1EDFE4AE2EEE45A059984F874536F
:102C6000A3EE056A0F78C4F8FC32E7EE636AC4F895
:102C70000033C4F80433E8EE047AC4EDD05A84ED8E
:102C8000D16AC4EDD96A82EDBE7AC4EDDA7AFDF775
:102C90008ABEB5F91480FEF7C2BD0023012DC4ED34
:102CA000237AC4ED227AC4F890307DF4F8AD07EEB3
:102CB000906AD4ED1B6AF8EEE77AB54286EEA77A01
:102CC00084ED097A7DF4EBADEAE69A457DF4DAAE5F
:102CD0004EF806A00246BAF1000F3DF4D3AEF0EE76
:102CE00040DAD7EEA6DA4B4BD3ED006A9FED4A7A75
:102CF000DFED4A7A6DEEA6DAB0EE4C8AF4EEC7DA72
:102D0000F1EE10FA88BFF0EE47DAF4EEE7DAF1EE12
:102D100010FAB8BFF0EE67DAFDF7DEBEF0EE48DA83
:102D2000D5EEA6DA3B4BD3ED007A6DEEA7DA4FF085
:102D3000000A84ED01CAFDF7D2BE012B40F3E08208
:102D400007EE101AB8EEC77AC7EE876AB1EEE68AC8
:102D5000132A17D047B107EE907AF8EEE77AF4EE2F
:102D6000C87AF1EE10FA29D407EE906AD4ED1A6A07
:102D7000F8EEE77AB54286EEA77A84ED087A7DF41C
:102D80005BAD77E6B0EE480A34F08CFF00B2E1E7C5
:102D9000012A8CDD07EE103AB8EEC77AC7EE876AD3
:102DA000F1EEE67A002F82D007EE107AB8EEC77AFD
:102DB000F4EEC77AF1EE10FA7FF779AF099B059927
:102DC0009A8B0F78A8F8060042F2107303FB02F307
:102DD000069A06991268B3FBF2F3C4F8B030FDF717
:102DE0003BB8012A7FF773AE07EE103AB8EEC77A08
:102DF000C7EE876AF1EEE67A002F3FF468AE07EE81
:102E0000107AB8EEC77AB4EEE77AF1EE10FA7FF5F1
:102E10005EAED3E7F8BF002000007A4400007AC419
:102E2000E8840020EE4BEF49D3ED016A93ED022ACE
:102E3000D3ED032A67EE266AE4EE826AE5EEA26A23
:102E4000F7EE002AF5EEC06AF1EE10FA48BF66EE22
:102E5000836A67EEA66AF4EEE26AF1EE10FA88BFC2
:102E6000F0EE626AF0EE452AE3EEA62AB4EEE26ADC
:102E7000F1EE10FAF0EE626A9ABFF3EE042A76EEF3
:102E8000E26AF0EE446A012AC1ED006A3EF4DEA86F
:102E9000D3ED056A93ED062AD3ED072A67EE266A7D
:102EA000E4EE826AE5EEA26AF7EE002AF5EEC06A69
:102EB000F1EE10FA48BF66EE836A67EEA66AF4EE9A
:102EC000E26AF1EE10FA88BFF0EE626AF0EE452A8F
:102ED000E3EEA62AB4EEE26AF1EE10FAF0EE626AD0
:102EE0009ABFF3EE042A76EEE26AF0EE446A022A12
:102EF000C1ED016A3EF4AAA8D3ED096A93ED0A2A4E
:102F0000D3ED0B2A67EE266AE4EE826AE5EEA26A4A
:102F1000F7EE002AF5EEC06AF1EE10FA48BF66EE51
:102F2000836A67EEA66AF4EEE26AF1EE10FA88BFF1
:102F3000F0EE626AF0EE452AE3EEA62AB4EEE26A0B
:102F4000F1EE10FAF0EE626A9ABFF3EE042A76EE22
:102F5000E26AF0EE446A032AC1ED026A3EF476A802
:102F6000D3ED0D6A93ED0E2AD3ED0F2A67EE266A94
:102F7000E4EE826AE5EEA26AF7EE002AF5EEC06A98
:102F8000F1EE10FA48BF66EE836A67EEA66AF4EEC9
:102F9000E26AF1EE10FA88BFF0EE626AF0EE452ABE
:102FA000E3EEA62AB4EEE26AF1EE10FAF0EE626AFF
:102FB0009ABFF3EE042A76EEE26AF0EE446A042A3F
:102FC000C1ED036A3EF442A8D3ED116A93ED122AD3
:102FD000D3ED132A67EE266AE4EE826AE5EEA26A72
:102FE000F7EE002AF5EEC06AF1EE10FA48BF66EE81
:102FF000836A67EEA66AF4EEE26AF1EE10FA88BF21
:10300000F0EE626AF0EE452AE3EEA62AB4EEE26A3A
:10301000F1EE10FAF0EE626A9ABFF3EE042A76EE51
:10302000E26AF0EE446A052AC1ED046A3EF40EA895
:10303000D3ED156A93ED162AD3ED172A67EE266AAB
:10304000E4EE826AE5EEA26AF7EE002AF5EEC06AC7
:10305000F1EE10FA48BF66EE836A67EEA66AF4EEF8
:10306000E26AF1EE10FA88BFF0EE626AF0EE452AED
:10307000E3EEA62AB4EEE26AF1EE10FAF0EE626A2E
:103080009ABFF3EE042A76EEE26AF0EE446A062A6C
:10309000C1ED056A3DF4DAAFD3ED196A93ED1A2A52
:1030A000D3ED1B2A67EE266AE4EE826AE5EEA26A99
:1030B000F7EE002AF5EEC06AF1EE10FA48BF66EEB0
:1030C000836A67EEA66AF4EEE26AF1EE10FA88BF50
:1030D000F0EE626AF0EE452AE3EEA62AB4EEE26A6A
:1030E000F1EE10FAF0EE626A9ABFF3EE042A76EE81
:1030F000E26AF0EE446A072AC1ED066A3DF4A6AF23
:1031000093ED1D2AD3ED1E2AD3ED1F6A27EE027A16
:10311000A4EEA27AA5EEA67AB5EEC07AF1EE10FA88
:1031200048BF27EE037A27EE877AF7EE007AB4EEEF
:10313000E77AF1EE10FA88BFB0EE677AF0EE457AE2
:10314000E3EE877AB4EEE76AF1EE10FA3EF629AEC6
:10315000FEF723BE28461546FEF74DBF079AC4F872
:10316000E422FEF7D2BA079AC4F8EC22FDF772BA4D
:103170000546FEF791BE032704220225FEF788BE0E
:10318000B0EE656A002501F5A27304EB830306988F
:103190000CE026EEA77A07EE901AF8EEE77A36EE04
:1031A000076AE7EE275A05460F291DDCD3ED017AA1
:1031B000B3EC017A013137EE075A67EEA76A002DAA
:1031C000E7D1B4EEE75A67EE076AF1EE10FA27EEA0
:1031D000A75A26EE877AE7D5A5EE277ADBE700BF68
:1031E00054C0002028410020B5EEC06AF1EE10FA6C
:1031F00040F30381C5EE867AD04BB7EE006A37EE16
:10320000C66AD3ED007A66EE277AFDEEE77A17EE0E
:10321000903A7C2B40F365814345A8BF434604EEBA
:10322000903AF8EEE44A94F8FA1401EBC10304EB87
:10323000830303F5C56503F2146EDEED006A95EDB8
:10324000007A03F22C6003F5C366D6ED005AD0ED88
:10325000007AA4EEA67A03F5C46C03F22466E4EEC9
:10326000A57A03F21C63F0EE476A9CED007AE6EE65
:10327000C77ABDEEE67AC5ED007A17EE10CA96ED74
:10328000007AD3ED007A27EE667ABCF17C0FA4EECB
:10329000A77A80ED007A40F38F80C445A8BFC4466A
:1032A00007EE90CAF8EEE77AFCEEE77A17EE903A6E
:1032B0009BB204EB4100A0F8803611B90F2F00F04B
:1032C0008281112F00F00381102F7FF4BEA810F02F
:1032D000AFFD059BDFF870821F78994B94F8F924B5
:1032E0000693A0EB0900A8F80200FFF7B0B800238E
:1032F000012DC4ED1E7AC4ED1D7AE3677DF49CAA0E
:103300009FED908A24E55B420AFB03F381FB03C136
:10331000DB17C3EB2113121A9E441344C644A9EBD6
:103320000309A4F802E0A4F80090FEF71DB8002AF3
:1033300000F0DF80B4F90A3013600120FEF750BEC0
:10334000059B1B78262B7DF469A8B0EE490A8DED0C
:103350000F6ACDED0E7A34F0A5FCDDED0E7ADFF8C4
:10336000E8A127EEAA0AAAF8000034F09BFCB0EE10
:103370004F0AAAF8020034F095FC9DED0F6AAAF8F6
:103380000400FDF74BB8B2EE049A20EE090A34F0BF
:1033900089FC6D4B0E93B0EE6D0A1880A3F802A065
:1033A00034F080FC0E9B28EE090A988034F07AFCF9
:1033B0000E9BD880FDF70DBB7D237AE70F2F00F021
:1033C0001281112F7CF405ADB0EE480A34F06AFC8E
:1033D0005D4BD880FCF7FDBCDFF8748131F050FF05
:1033E00000283FF448AAD8F80020337802F59C5210
:1033F0000832CBF83821FFF7EFB99FED526A12E798
:1034000094F8FA64800000F2145E04EBC6165FEADA
:1034100095081844A64406F55E7634D04FEA08189D
:1034200008F1100CB44406F1100300F110010EF184
:10343000100213ED024A13ED035A13ED017A13ED56
:10344000046A51ED024A51ED035A51ED046A51EDFF
:10345000017A64EE244A65EE255A66EE266A67EE26
:10346000277A10339C4542ED024A42ED035A42ED61
:10347000046A42ED017A01F1100102F11002D8D183
:1034800046444044C64415F003053FF42EA996ED8A
:10349000007AD0ED007A67EE877A012DCEED007AC2
:1034A0003FF423A996ED017AD0ED017A67EE877A91
:1034B000022DCEED017A3FF418A996ED027AD0EDF7
:1034C000027A67EE877ACEED027AFFF70EB9DFF85F
:1034D000788094F8F92428F81130194B0693FEF7F8
:1034E000B6BFDFED1A4A9EE607980AF0A5FFFFF780
:1034F000FDB90120FEF774BD052706220425FEF75D
:10350000C7BC059B1F780F2F00F0BA80032F3568CA
:103510003DF403AD89ED028A05F00055FCF784BC4B
:1035200010F086FCDFF82080059B94F8F9241F78C2
:10353000A0EB0900A8F80200FEF789BF083C0020B4
:1035400090A0002000000000E88400200000FA4263
:10355000308500200000C8420699D1ED027AF0EED5
:10356000E77AFCEEE77A4FF6EF7217EE903A103BEF
:103570009BB293421AD9D1ED017AF0EEE77AFCEED4
:10358000E77A17EE903A103B9BB293420ED9D1EDF9
:10359000037AF0EEE77AFCEEE77A4FF6CC7217EE9C
:1035A000903A333B9BB293423EF63EACDBF82C3173
:1035B000002B40F09380079B03F59233F833CBF850
:1035C0002C31FEF734BC1FED1D0A7B4B069326EE13
:1035D000000A34F067FBDFF8E48194F8F924A8F8D6
:1035E0000600FEF734BFB0EE480A34F05BFB734BC5
:1035F0001880FCF7EEBB724B724E1A46FFF751B8BB
:1036000040201CF07FF900287FF4DEA83B68DFF83B
:10361000D881DFF8D8A14FF040090DE01CF0D2F9B5
:10362000DAF800203B68013A0133B9F10109CAF820
:1036300000203B6000F0978043441B7E1846002B1F
:10364000ECD100234FF0FF323B6004237A603370EB
:10365000FFF763B92BF024FB074668B1DFF89081D0
:10366000D8F80030834276D0D8F8DC309F4269D059
:10367000D8F8B8319F4257D00AF090F8FFF7A4B8B5
:1036800034F010FB35684D4B05F0005558802B4643
:10369000FCF7C4BB10F0CCFBDFF82081059BA0EB4E
:1036A00009001F78A8F80200FFF76FB810F0C0FB00
:1036B000DFF80881059BA0EB09001F78A8F804003B
:1036C000FEF7EBBD10F0B4FBDFF8F080059BA0EB3C
:1036D00009001F78A8F80200FEF75DBE079A9A421B
:1036E0007EF6A5AB202025F0DBF9FCF71DFAFEF7EE
:1036F0009EBB31F083FA00287EF476AB31F012FFE6
:1037000000283DF488ACFEF76FBB2F4F386823F0DC
:1037100044FC2E4B1B780022022B3A607FF4A1A8B8
:1037200023F0E8FDFFF79DB8384623F036FCDC2295
:103730000021274834F0A2F99EE734F0B3FA00B232
:10374000FFF748BA384623F028FCDC220021214844
:1037500034F094F98CE723F020FCDC220021404671
:1037600034F08CF980E743441B7E002B7FF42CA8B7
:1037700067E7194BD4ED01EA1A78184BB1EE68EA05
:1037800093ED006A002A7DF4C7ACB0EE4E9AB0EE1D
:103790004EFADFED13DAFCF779BE45201CF012F982
:1037A000FF201CF00FF90F481CF0F8F828461CF019
:1037B00009F9FFF77FB800BF90A00020E88400203F
:1037C000103C0020FC9E002084640020DF3E00208E
:1037D000EC970020109700203CBF0020FCBF002089
:1037E00000000000E0D00408449304088064002036
:1037F000349600202DE9F04F83B01C4606468846DB
:10380000174610F015FB8A4B1B78002B72D02F2F18
:1038100070D8DFF83CA2DAF80430002B6AD1152FFB
:103820006BD80123834903FA07F20A4240F0ED8086
:10383000814912F03E0F9B460CBF4FF47A730B4642
:103840000193002C5FD100F51C501030019BCAF889
:1038500004008AF80DB0CAF80830B8F1000F47D05C
:1038600042463946754834F009F9754A1389B8F16A
:10387000010FB3FA83F34FEA531335D0B2F868104F
:10388000002918BF0023B8F1020F2DD0B2F8C810DC
:10389000002918BF0023B8F1030F25D0B2F8281172
:1038A000002918BF0023B8F1040F1DD0B2F8881109
:1038B000002918BF0023B8F1050F15D0B2F8E811A0
:1038C000002918BF0023B8F1060F0DD0B2F8481236
:1038D000002918BF0023B8F1070F05D0B2F8A822BD
:1038E000002A08BF1C4600E01C4684F00104E4B234
:1038F0008AF80C4003B0BDE8F08F4FF47A7301935F
:103900004FF0010B9DE708F1FF3942F228305FFAD2
:1039100089F910F0DFFA09F10109CDF800804FF4C0
:103920007A7010F0D7FA009B002B58D0454DDFF885
:103930002481002404E001344C4505F160054ED09B
:10394000E3B29E4201D0FF2EF5D13D4963001A1922
:1039500001EB42124FF0010C82F814C0297AB8B280
:103960000029E8D0DAF8041031B19AF80C1019B92E
:103970009AF80D10002940D1314AA880234402EB67
:1039800043134FF0000C1A7D98F8001083F814C010
:1039900042EA4000021282EA101242402A4B02F030
:1039A0000F0242EA00121B68002934D1012105F1FF
:1039B00014009847E9682B68B5F806C0B1F82C21C7
:1039C000DB6842EA0C02A1F82C2158601A68013425
:1039D00042F001024C451A6005F16005B0D10020AB
:1039E0000BF1FF3BF5F786F81BF0FF0B97D1019821
:1039F00003B0BDE8F04F10F06DBA14492144887A45
:103A00000028B9D082F814C0B6E74FF47A73019356
:103A10004FF00A0B15E72868E968407900F0FC00D0
:103A20000C30084404219847EB688000188182E735
:103A3000BCA2002080173000A0860100922B00203D
:103A4000D0A20020D4A20020C4A20020882B0020F5
:103A5000842B0020CCA200202DE9F0472DED028B15
:103A6000C04D2B78002B40F09280BF4C2378D907B3
:103A700036D4FBF7BDFEBD4B1A68002A3CD1237833
:103A8000DA0703D5BDEC028BBDE8F08710F0D0F962
:103A9000B74BB84A1B68C31A9342064600F28C80A3
:103AA000B54F3B68002BEDD1B44B03F1780103E037
:103AB0000633994200F08A811A781E2AF8D1987844
:103AC000DA78904202D35A79002AF1D01E21AC480C
:103AD000F6F7FEFD002800F0798102233B60D1E774
:103AE000A84AA94B1178186801F0010113F056FBA0
:103AF0009E4B1A68002AC2D0A44B9F491B78002015
:103B0000086023B1A24BD3F8B030002BBAD1A14C3E
:103B1000002A92FAA2F3B3FA83F3D4F8402108BF43
:103B20004FF0FF3301339A42ACD09B48C4F8403188
:103B3000DBB2A0FB03208008984900EB80029B1AAF
:103B400043F205254FF00534DBB200F0FF020D8192
:103B5000C1E90044002800F06A811920012A887216
:103B600000F0C080023AD2B20732C8720446520056
:103B70000C200C54451C0230824201EB000600F080
:103B8000D880402806F8014CF3D10246B6E07F4ABF
:103B90001378002B7FF469AF8149824B888B1C68B6
:103BA0007B4942F2107303FB00F30120B3FBF4F3F3
:103BB0001070C1F8B03058E77B4BDFF80CA21B78CF
:103BC000DAF80090002B40F004816B4FDFF8C481DD
:103BD00094F800C0694B00224CF0030121703A6058
:103BE00003F17801C8F80C21C8F8102102E006336F
:103BF00099420DD01A781F2AF9D19878DA78904234
:103C000002D35A79002AF2D04CF0070C84F800C095
:103C1000664AB2F90030002BB8BF5B42B3F5E17FD2
:103C20003DDAB2F90230002BB8BF5B42B3F5E17F59
:103C300035DA5F4B5F4C93ED057AD3ED077AD3ED20
:103C4000096A93ED030A77EEA67A30EE070AF7EEDB
:103C5000000AB0EE007AE7EEC70A30EE000AF6F787
:103C600045FDBEEE008A20EE088AB0EE480AF6F75F
:103C700011F8FDEEC87A84ED010A17EE903ADFEDF7
:103C80004E7A2033402BC4ED027AC4ED037A00F261
:103C9000B780B0EE480AF5F78BFF84ED040A6B7825
:103CA000DFED466A07EE103A07EE906AB8EEC77A83
:103CB000F8EE677A0023E7EE267A19F0800FC8F84D
:103CC0004031FCEEE77AC8ED4F7A27D03C4B1B78A9
:103CD0009B0723D53B4B9B7C042B1FD9062023F04D
:103CE00099FB1EE03222CA720C20002B3FF44DAF2C
:103CF0000524012B0C5400F1010208D1FF238B5441
:103D0000BDEC028B0E20BDE8F04723F083BB851C81
:103D100019263E2D8E5411D92A46EFE7052023F0AF
:103D200079FB0023C8F84431C8F84831C8F82C3171
:103D3000A8E632243E2A4C55D7D9DFE7022B4C5552
:103D400000F10302DAD0051D3E2D8E54E4D8032B7A
:103D50004C5500EB0402D1D0831D3E2B8E5473D9F9
:103D60001A46CBE7DC3E0020DE7A0020887D00206A
:103D7000AC6400207F4F1200D07D0020A8410020BD
:103D8000903E0020F9840020FC840020FE3B0020AF
:103D9000E8990020842B0020CDCCCCCC9446002088
:103DA00070A0002090A00020BCA20020747B002006
:103DB000702600202000002000000000002474492C
:103DC000A87D0020907D0020A0A0002001233B6062
:103DD00058E61E2031F00AFB00283FF4F6AE1E2103
:103DE0001B481C4FF6F774FC09F4805358B93A6825
:103DF000022A08D0184A1070DBB1DFF86480E7E6C9
:103E0000B0EE670A49E7144ADFF8548001211170C7
:103E1000002288F82921002B7FF4DAAE0F4AFF2018
:103E200011781522FFF7E6FCDAF80090D0E60A20B8
:103E30005BE70A4ADFF828801178FF201422FFF799
:103E4000D9FCDAF80090C3E6C21DCC5456E700BF97
:103E5000903E0020D07D0020B064002075710020CD
:103E6000842B00202DE9F04FDFF84CC204460A30C5
:103E70000CEB000E87B09EF80C801CF800900391AC
:103E80004FF41A7C404601920CFB04FA04930EF0A6
:103E900099FF064648460EF095FF009040460EF00A
:103EA000F3FA9DF84450804B0590484603F5A67BF5
:103EB0000EF0EAFA15F008039DF8407002930BEB40
:103EC0000A08DDE9001200F09180002900F0E58089
:103ED00091F807C01CF0020F40F0DF80724B03EB3B
:103EE0000A0C07F002030093CCF88C11CCF888017F
:103EF000CCF8840130B14FF00B0C04EB0C0180F8CE
:103F000006C0C171684B049E4FF41A7909FB04394D
:103F10000AF1480089F85071039FC9F87871584434
:103F2000624FC9F84C710AF5A47100275944C9F8C9
:103F300060014FF48070C9F87C2189F85151C9F8AB
:103F40006411C9F85801C9F85C013146D9F88C01EF
:103F5000C9F8546189F8A443C9F86C71C9F868714B
:103F6000C9F87471C9F87071C9F8A073A9F8987389
:103F7000FBF7C8F805F00101D9F88C0127F094FF90
:103F8000009A4B484B49C9F8AC730AF519750AF504
:103F900017735D44C9F8B003C9F8A8139B44002AFD
:103FA0005CD0D9F89001002858D0D9F88C2103684A
:103FB0001268934252D0012389F8A5333146FBF7AA
:103FC000A1F85946D9F8900127F0D2FE3A46294681
:103FD000D9F88C010EF036FD029B002B4FD04046E5
:103FE000FBF766F8404607B0BDE8F08F17F0010315
:103FF000019318D117F00203009383D0B9F1000F99
:104000004BD0294B4FF41A7C0CFB043C019BCCF8A1
:104010008801002B3BD100293FD0CCF88C1100281F
:104020007FF469AF6EE7002E37D096F807C01CF01A
:10403000020F32D11C4B03EB0A0C059BCCF88431E8
:10404000059BCCF88C61002BD4D04FF00C0E04F102
:104050000B0C83F806E083F807C0CBE7124A4FF455
:104060001A7303FB0424002384F8A5335A46294617
:10407000D4F88C010EF0E6FC029B002BAFD1404639
:10408000FBF70CF801214046FBF758F8A7E7CCF8FE
:10409000901100287FF42FAF34E74FF0000840461E
:1040A00007B0BDE8F08F00BF842B002024960408E1
:1040B000E5EF000855F1000888AF002030B4454B0B
:1040C0001B78012B14BF0024032439B30429038C6B
:1040D00047D0082961D023F480531B041B0C0384B0
:1040E000838B058C40F6FF41194045F6FF732B404A
:1040F00043EA023241F4807192B241EA043142F45F
:10410000805281830284838B23F440631B041B0C45
:104110008383838B9BB2838330BC7047018C21F0F7
:1041200001010904090C0184018B038C89B223F07D
:104130000A0321F0F3011B0442F0010241F00101E6
:104140001B0C134341EA041101830384038B23F006
:104150000C031B041B0C0383038B9BB2038330BC37
:10416000704723F010031B041B0C0384058B038C86
:104170009BB223F0A00340F6FF4143EA021229401C
:1041800041F4807192B241EA043142F0100201839D
:104190000284038B23F44063DBE723F480731B0466
:1041A0001B0C0384818B038C9BB223F4206389B2A4
:1041B00043EA022221F0F30141F0010192B241EA07
:1041C000041142F4807281830284838B23F00C03F8
:1041D0009CE700BFA4A00020F8B550F8043C10F8FC
:1041E0000E4C5E7902461868C4B114460B4632F88C
:1041F0000C1C14F80F7C24F80A3C0D4A5B1A9BB285
:10420000002524F8083C314622F817302A4604F8E5
:104210000E5CFFF753FF04F80D5CF8BD012302F8B4
:104220000E3C22F80C1C31460222BDE8F84045E75E
:10423000303A0020134B1A680AB1002111609A69C4
:104240000AB1002111601A6B0AB1002111609A6C49
:104250000AB1002111601A6E0AB1002111609A6F33
:104260000AB100211160D3F890200AB10021116039
:10427000D3F8A8300BB100221A60034B00221A7049
:10428000704700BFE0A1002054AF00202DE9F04F9F
:104290000C68B94EB94F25883668B6FBF2F285B086
:1042A000013B013ABC429BB292B2ADB2BDF838803C
:1042B0009DF83CC011D0B24EB4420ED0B4F1804F44
:1042C0000BD0A6F58036B44207D006F58066B4421E
:1042D00003D006F58066B44202D125F07005ADB278
:1042E000A84EB44211D006F58066B4420DD025F434
:1042F000407506F56C46ADB2B4422580E362228576
:1043000040F04E810023238602E02580E36222856F
:104310000123A3824A79CB79BCF1000F01D083F04D
:10432000010313F0020140F0FA804FF480665B0055
:1043300003961026019603F00203029189468B46EC
:104340004FF480454FF4805E4FF480764FF0010CBF
:104350000C2A00F2CA80DFE802F098C8C8C869C811
:10436000C8C837C8C8C80700218C844E21F48051C2
:104370000904090C2184B4F820C0A788A18B1FFA76
:104380008CFC21F4E6412CF4005C09044EEA0C0E8E
:10439000090CB4424EEA0333BFB241F4C04100F00D
:1043A000CF8006F58066B44200F0CA80A780A18362
:1043B000C4F840802384A38B23F400631B041B0CEC
:1043C00043F40063A38396E0258C6C4F25F480753D
:1043D0002D042D0C2584B4F820A0B4F804C0A58BBE
:1043E0001FFA8AFA25F073052AF4007A2D0446EAAA
:1043F0000A062D0CBC4246EA03231FFA8CFC45F04A
:10440000600500F0C1805E4EB44200F0BD80A4F8AB
:1044100004C0A583C4F83C802384A38B23F0080345
:104420001B041B0C43F00803A38364E0218C534D51
:10443000019F21F010010904090C2184B4F820C067
:10444000A688218B1FFA8CFC21F4E6412CF0200C6D
:10445000090447EA0C07090CAC4247EA0313B6B259
:1044600041F4C0417BD005F58065AC4277D0A68091
:104470002183C4F838802384238B23F400631B0436
:104480001B0C43F40063238335E0218C3B4D21F06A
:1044900001010904090C2184B4F820E0A788218BCC
:1044A0002EF0020E21F073014FEA0E4E09044CEA81
:1044B00003034FEA1E4E090CAC424EEA0303BFB29F
:1044C00041F0600140D005F58065AC423CD0A7804A
:1044D0002183C4F834802384238B23F008031B0436
:1044E0001B0C43F00803238305E0042AC4D0082AE8
:1044F00093D0002AF0D0B4F8443043F40043A4F839
:1045000044302188234641F0010123F8341B002167
:104510009D18C0E90054995005B0BDE8F08F002502
:10452000DB00402703F00809AE46039501952E46AF
:104530002B46AC464FF4806102974FF0040B07E71F
:1045400027F480472F4331E74FF6F3751D4027F4DA
:10455000407745EA0903374343EA0B03B7E723F003
:104560008003029D43EA091323F040032B43039D7C
:1045700026F440662E437AE7A0A200200000014006
:10458000000401400010004023F4006343EA0923C3
:1045900023F480632CF4405C0B434EEA0C0C36E7AA
:1045A000024B9C423FF4AEAEB2E600BF00040140B5
:1045B000F0B583B006460C460EF004FC05463046C6
:1045C0000DF062FFF8B1F5B1104E012225217061A6
:1045D0008171C271022112F039FD0027DFF838C065
:1045E0000B4B93FBF4F39BB20A4A0093294692FBD0
:1045F000F4F330469BB20197ACF80040FFF746FE5B
:1046000033681F60777403B0F0BD00BF10850020D1
:1046100020A1070040420F0028850020F8B5244C57
:1046200094F81C3683B104280ED8224B224E94F8FD
:104630003456B4F8362603EB80000027D0F8100378
:104640003760B4F83A3605B1F8BD07EE902A9FED11
:104650001B7A9FED1B6AF8EEE77A642267EE877A91
:1046600007EE100AB8EEC77A02FB030367EE877AFB
:1046700007EE103AB8EEC77AD4F82C3687EE870AE0
:104680000D4606EE903AF8EE666A66EE866A20EE11
:10469000260A33F007FBD4F824260A4B10601B6867
:1046A000B4F8381619442944C4F84016F8BD00BFC0
:1046B000842B002044930408147D00200AD7233C57
:1046C000CA269B3E30850020052819D8052917D811
:1046D000884215D070B40B4B01EBC10103EB4101D3
:1046E00000EBC00040000E684D688C68CA68C65078
:1046F000184445608460C2600B8A038270BC7047B6
:10470000704700BF865E0020064B074A05288CBF15
:1047100058785870054B00EBC00003EB4000106068
:1047200030F05CBFD8980020BC7F0020865E00205F
:104730002DE9F04F864B2DED028B1B68DA048FB00C
:10474000044600F1D386834B1B78022B00F0DC86F5
:10475000042B01F06880012B00F042827E4BDFF8D1
:104760003CA201937D4B7E4A9C42927800F26C827F
:10477000002A40F06C827B4B029330F0D3FE744BE6
:104780001E68019BB3F90670F304804600F182862F
:10479000754B9B8A6425FF1A05FB07F5C3F5FA6381
:1047A00095FBF3F5642DA8BF642525EAE575EDB208
:1047B000029B1A786D4B1B681F0202F0010240F148
:1047C000EF80002A00F0EF80674B1B7FAB4241F285
:1047D0008D81B8F1000F40F0ED809AF81831002B70
:1047E00040F0E880624B63491B680027CF6293F872
:1047F0002C00614B4F608F611F605F609F600028DD
:1048000040F0D8805D4B8AF828011F78002A40F0DC
:10481000D9805B4B9FED5B7A5B7807EE903AF8EEC0
:10482000E77A202F67EE877AFCEEE77A17EE905A48
:1048300000F07F82544F2C44CAF83C41534B1B7804
:10484000002B40F08382484B019A998AB2F900000C
:10485000DA8A8142B4BF8023002382420198B0F9F2
:104860000200C8BF43F040039B088142BCBF63F015
:104870007F03DBB282420198B0F90400C8BF43F065
:1048800040039B088142BCBF63F07F03DBB28242DE
:104890000198B0F90600C8BF43F040039B0881426D
:1048A000BCBF63F07F03DBB282429AF84D26C8BFDB
:1048B00043F040039A4201F0F081354A8AF84D36C0
:1048C00011780022AAF84E268AF85026002901F015
:1048D000B4815F2B00F03A826F2B00F037822D4BB2
:1048E00000221A60029B1A78194BD0071B6807D464
:1048F0009AF8502622B9BAF94E26322A01F3B28626
:10490000254A03925D0740F128829AF852365BB13E
:10491000029B1B78DC0707D5134B019A9B8AB2F9DF
:1049200006209A4201F3508210211048F5F7D0FE7C
:10493000002801F00F809AF858362BB99AF85336B0
:1049400013B93223AAF8563601238AF8583604E2FE
:10495000A0A00020EE3700207ABA0020404B4C0087
:10496000E07A0020DE7A002058AF0020903E002040
:10497000B87F0020EC40002040C00020E5840020EB
:10498000DC3E002000247449387B00204062002077
:1049900020000020D07D00201C720020842B0020ED
:1049A00070023FF50EAF00238AF81831B8F1000FFE
:1049B0003FF418AF01238AF82831B94B1F78002A39
:1049C0003FF427AFB74B5978002900F0A1819AF83E
:1049D0002911002940F09C81B3490978002940F051
:1049E00097819AF82A11002940F09281AF490978FD
:1049F000C90600F18D81DAF844210392F20601F133
:104A0000F8861A790492AA4261D8019AA849B2F9A3
:104A10000020B1F812C0A7486FF47A76911989B2D4
:104A200040F2E636B142CCF5FA6B90F800E090F82F
:104A3000019055D80CEB0E06964281F26287A2EBEC
:104A40000C026421A2EB0E0201FB02F2ABEB0E01A1
:104A500092FBF1F2D2B20E2A42D8019AB2F90220A8
:104A60006FF47A70111889B240F2E630814237D87B
:104A7000B24242F39180A2EB0C02A2EB0E00642240
:104A8000ABEB0E0102FB00F292FBF1F2D2B20E2A66
:104A900026D8019AB2F904206FF47A71511889B2BC
:104AA00040F2E63081421BD80CEB09018A4242F306
:104AB0006280A2EB0C02A2EB09016422ABEB0909B4
:104AC00002FB01F292FBF9F2D2B20E2A08D8049A44
:104AD00052004B2AA8BF4B22D2B2AA4201F29486BE
:104AE000754ADFED767A92ED097AB0EEC77AB4EEC8
:104AF000E77AF1EE10FA41F1878692ED047AB0EE92
:104B0000C77AB4EEE77AF1EE10FA41F17D8692EDC4
:104B10000E7AB0EEC77AB4EEE77AF1EE10FA41F110
:104B20007386039A0AB9CAF844415A88DAF84411DC
:104B3000DAF848314A2D88BF52084FF47A705B1A70
:104B4000234400FB02F2934202D901228AF8292170
:104B5000002901F064865A4A9FED5A7A527807EE8E
:104B6000902AF8EEE77A202F67EE877AFCEEE77A54
:104B700017EE905A07D15449544AA1FB03139B09DD
:104B80000121D3809180524B1E68F2067FF552AE10
:104B9000464B1B78DB063FF54DAEF7043FF54AAEBA
:104BA00030F02CF84B4F00287FF445AE3B881E05B3
:104BB0003FF541AE484B1B78002B01F09286B8F1CF
:104BC000000F41F0158725B1DAF83C319C4201F223
:104BD000F387102022F01EFC01238AF84C362DE6C4
:104BE000DFF828A1DAF84436E31A002B24DB3B4A2D
:104BF0003B4B517C2E4A33F81130507C04F59C42DB
:104C000020329908CAF8442618B1C1F57F730333DE
:104C100099B23448344E0278344D36F812702B680D
:104C200026F81210DB1B0B44013231492B6002F0D5
:104C30000F021B0902700B802E4B01932E4B2F4A43
:104C40009C4292787FF694AD002A00F07A872C4B34
:104C50002A4A1E780293092092F821502FF026FE4E
:104C600006F00107814620B1264B9B79022B00F00C
:104C7000E783012D40F0E4834FF0000B1F4B224EE1
:104C800093F82030DFF87C80062B00F2C785DFE840
:104C900013F07803B3073103440351036403C703DC
:104CA000E5840020C23C0020B0640020A87D0020E4
:104CB00058AF0020D0630020EC4000200000C84224
:104CC000DC3E002000247449D34D6210E8840020AB
:104CD000A0A00020387B0020200000200C870020AE
:104CE00030870020EF370020F4370020F037002015
:104CF000143800207ABA0020404B4C00E07A0020A3
:104D0000DE7A00202063002030850020842B0020E4
:104D10001C4B9FED1D7A5B7807EE903AF8EEE77A30
:104D2000202F67EE877AFCEEE77A17EE905A7FF431
:104D30002CAF164B00215960002A3FF47BAD144B79
:104D40001E6822E74FF4C873AAF8C830104B114A06
:104D50001B6803925D073FF5D8ADDFF840B09FEDCB
:104D60000E8A0DF1280808AD00220421C8F804209D
:104D700008920A920C926A600BF178065C460D91DB
:104D800015E000BFDC3E002000247449E8840020C8
:104D9000A0A000201C7200208096984AA841002004
:104DA000B9F1280F40F26D810634A64249D06379EB
:104DB000002BF9D194F800900CA84946F5F788FC2F
:104DC0000028EDD04946BA48F5F782FC002840F0AB
:104DD0005E814946B748F5F77BFC002840F05181D9
:104DE0000FF026F807EE900AF8EE677AF4EEC87A2C
:104DF000F1EE10FAD8DBA278E07882421AD263781A
:104E00000199043340F6330C31F913306345A8BFE0
:104E10006346B3F5617F4FF0190140F2833CB8BFA0
:104E20004FF4617311FB02C29A4203DA11FB00C115
:104E30009942B9DA21789F480634F5F739FCA64241
:104E4000B5D19DF829609DF821009DF820209DF89E
:104E500028C09DF8221070409DF82A608DF821002E
:104E60008CEA020271408DF820209DF82B609DF89D
:104E700023208DF8221072408DF8232001269BF804
:104E800005300EA95A0901EB820203F01F0106FA50
:104E900001F1ABB19BF8003052F818CC580903F07F
:104EA0001F0355F8202011EA0C0F06FA03F343EA1A
:104EB00002010ABF22EA030345F8201045F820301A
:104EC0000BF1060B5C45DAD17B4B794A1B7895E8F0
:104ED000030082E80300002B40F08384774B1B78AB
:104EE000002B00F0348301217148F5F7F1FB3C8879
:104EF000002840F02081724BDB78002B40F01B81B2
:104F000024F001039BB2A3423B8009D06D4B41F2D8
:104F10000241FF220E2019809A7022F07BFA3C8811
:104F200063480221F5F7D4FB23B2002800F00C817E
:104F300023F001039BB2A3423B8009D0614B41F2B5
:104F40000241FF2219800E209A7022F063FA3C88F9
:104F5000A60740F13E8656480A21F5F7B9FB00281E
:104F600000F00A81250540F1ED84574A574B11782E
:104F70005868A40701F0020100F0B181003118BFA8
:104F8000012112F00BF9524B4FF4FA62C3F8E02002
:104F90001F214748F5F79CFB30B9029A137859074F
:104FA00044BF23F004031370039B3C881B6813F079
:104FB0000A0F1BD003213E48F5F78AFB002800F0BA
:104FC000AE84660740F14E8639480721F5F780FB2D
:104FD000002800F09284650640F13C860C2134489C
:104FE000F5F776FB002840F030843C8830480821F3
:104FF000F5F76EFB002800F0548144F48073A3425F
:105000003B8008D02F4B41F20241FF220E20198035
:105010009A7022F0FFF92F4B1B78082B00F04D817E
:105020000E2B00F04A812C4B1B685C0500F1BE8002
:10503000029B1B78D90740F1C980284B01241C70C2
:1050400028211B48F5F744FB9AF80831002867D15E
:10505000002B49D1002C4CD10B211548F5F738FB1A
:10506000002858D01E4B1A78824203D01D4A4FF0B8
:105070007E511160187001200FB0BDEC028BBDE8AD
:10508000F08F2A464146204630F0D6F98CE64FEAAA
:10509000591C09F01F0158F82C3001228A4023EADC
:1050A00002034946284648F82C30F5F701FB7BE619
:1050B000903E0020E0310020BCA20020D47C0020E3
:1050C000E07A002094460020F9840020FC8400202F
:1050D000781E002060400020A0A00020507C00200E
:1050E0001DC10020E802002000208AF80801002CE1
:1050F000B2D0B54B93F82530012BADD1B34B1B7813
:10510000002BA9D1172022F085F90B21B048F5F723
:10511000DFFA0028A6D1AF4B1868C0F30070A1E7F2
:10512000039A1268920793D5002B93D1CAF80C31D9
:10513000CAF81031D9E7039B1B689A077FF5E0AEE8
:10514000E30740F1978523B223F002039BB2A34209
:105150003B803FF400AFA04B41F20241FF220E2002
:1051600019809A7022F056F999483C880A21F5F77F
:10517000AFFA00287FF4F6AE984BDB7823B1984B5A
:10518000DB79022B3FF4EEAE24F400639BB2A34222
:105190003B803FF4EAAE904B41F20241FF2219807E
:1051A0000E209A7022F036F93C88DEE6122030F0AC
:1051B0001DF99AF8B646002840F0B885029B1B7886
:1051C000D80700F1A484002C40F0F585854B1E78AB
:1051D000002E64D1844B1C68002C3FF431AFDFF803
:1051E0003C82824C18F8030C277D4146A8F1030548
:1051F00030F06EF9002800F01984002F40F06A8426
:1052000005F10801687930F063F9002841F0ED827A
:105210007749A87A30F05CF9002800F01A84022F50
:1052200041F028837349E87B30F052F9002841F0BF
:105230001D837149287D30F04BF9002800F01A8455
:10524000042F41F00F836D49687E30F041F900284A
:1052500041F004836A49A87F30F03AF9002800F051
:105260001A84062F41F0F682664995F8230030F043
:105270002FF9002841F0EA82634995F8280030F0C0
:1052800027F9002800F01A84082F41F0DB825F49DB
:1052900095F82D0030F01CF9002840F01A84002405
:1052A000CEE624F480739BB2A3423B807FF4AAAE87
:1052B000574B1B78082B7FF4B3AE3A8822F040039B
:1052C0009BB29A423B803FF4AEAE434B41F2024167
:1052D000FF220E2019809A7022F09CF8A3E6B1FA02
:1052E00081F1490911F05AFF4A4B42F21072C3F89A
:1052F000E0204DE6002D40F03F83002F40F0438337
:10530000364A336852699A4280F04783334947F2FC
:1053100030520323CA6181F82030022023F0C0FB01
:10532000FAF702FC2D493268CB69134404228B61E1
:1053300081F82020002D01F0BF82284A336892694D
:105340009A4280F06B82294B1878002800F0448341
:10535000314A136823F0020313603268B8F8023050
:10536000642101FB03231D4900224FF480600B617F
:1053700081F82020CA7023F063FB184991F820308F
:1053800082E4002F00F03F8230F0CCF8012800F0DA
:105390002684B9F1000F40F01083002D40F03E82CA
:1053A0000E4A336812699A4252D298F80730022B9B
:1053B0004ED02FF0FDFF0949032240F6B83381F8A3
:1053C0002020CB61A9E700BF58AF0020B4B800206F
:1053D000903E0020A0A0002094460020E07A00200B
:1053E00020630020507C0020007C00202000002052
:1053F000513E0020563E00205B3E0020603E0020D3
:10540000653E00206A3E00206F3E0020743E002072
:1054100060400020781E0020887D0020473E00204C
:1054200065B3AD4A052382F82030002F3FF46EAFFC
:105430002FF0A6FFA84B4FF0030B93F8203023E486
:1054400016F002053FF418AC00254FF0020B15E4EE
:10545000A14A012382F8203098F80730012B00F090
:105460006F84C1F0DF80022BF6D12FF0A1FF9A49A3
:10547000062240F6B83381F82020CB61002F3FF49C
:1054800045AF2FF07DFF4FF0030B584621F0C2FFD0
:10549000FFF773B918219148F5F71AF900287FF43E
:1054A00077A98F4B1D7B002D7FF472A96FF47A7C56
:1054B00007EB0C0292B240F2E6318A4201F25B81C4
:1054C0008849DA884B8A99188F4200F393849B1A93
:1054D0009F42BFF66DA9DF1B642505FB07F5A3F509
:1054E0007A7395FBF3F3DDB2FFF762B900217B48D5
:1054F000F5F7EEF800287FF426A9FAF715FB7A4BAA
:105500001B78022B7FF424A9764A7849D37B527CFE
:105510000191013B31F913301AB1C3F53B630833F4
:105520001BB2A3F57A7307EE903A9FED717A714A38
:10553000DFF8DCA1F8EEE77A67EE877AFDEEE77A2E
:1055400017EE903A83F30A031380FFF70BB9DFF8E5
:10555000C491694E09F1FF3409F196054FF0010835
:10556000A346494619F8010C2FF0B2FF10B3B9F861
:105570000540FCB999F8040099F8023000EB4001AD
:105580000AEB8101013BD1F8682603EB4303334466
:1055900093420FD09AF89426C1F8683608FA00F0C2
:1055A00022EA000099F80330C1F86C468AF89406A4
:1055B00081F8643609F10A094D45D2D14F49504A64
:1055C000504B09681B78D2F800904F4D05915C460E
:1055D00004934FF0FF3B0026A0466B68002B6CD075
:1055E0001C78002C69D0AA68A9EB0202002A0EDB05
:1055F0009AF894260121B14022EA01028AF8942601
:10560000424A09F5FA704FF0FF31A8601160049A20
:10561000002A52D02A7859780432D2B200293ED1D9
:1056200030490198498A30F912009AF8942601F11C
:10563000C80C604540F35F8242FA06F1C8079A78C9
:105640003BD4002A0CBF01200220069222F002F86F
:10565000631E069A1F2B00F2DD87DFE813F0DE05DC
:10566000BF07A207260413048307640745072B0717
:105670001107F706DB072604F506830764074507CD
:10568000DB06C106A7068F0671065606DB07DE0598
:105690005406BF073B06DB077106210607060129F2
:1056A00000F05482BBF1FF3F40F089829AF89426C3
:1056B0000123B34013438AF894360136042E05F1D2
:1056C0000C058AD144460497DFF84C80CDF818A029
:1056D00004F19609019F24E0E07A0020903E00202A
:1056E0000CC0002058AF0020EE3700207ABA00200E
:1056F000AAF1823F1438002068960408BC7F00207D
:1057000030850020C54D0020E8310020F002002047
:10571000842B0020CD4400201A3200200A344C454E
:105720005AD0227938F9021F0432D2B237F9125016
:10573000A942F3D0E688002EF0D094F803A0AB4B3A
:105740000AF1FF3B0BEB4B01194491F8251300299B
:10575000E4D1611C20782FF0BBFE0028DED0A44BE2
:10576000A8F800501868059B2189002B00F0628280
:10577000002800F05F82A5F2DC559E4B01FB05F589
:1057800083FB0531ED17C5EB61110E44BBF11F0F13
:1057900000F25082DFE81BF0F703D403BF033402AA
:1057A000B0032A051305FC04EA04D804C6044E021B
:1057B0003402C0042A051305FC04AB0496047604E5
:1057C00067044F043D044E02F7033704D4032E044C
:1057D0004E024F0417046203049FDDF818A0FFF780
:1057E00082BB1E202FF002FE00283FF477AB1E2163
:1057F0008148F4F76DFF00283FF470AB142021F0CE
:1058000009FEFFF76BBB4FF48060B9F1000F01F0A8
:105810005E8023F02DF9794A00231361BBF1000F5C
:105820003EF4ABAF31E6DFF800A20EF001FBDAF890
:105830004836734AC31A93427FF7FEA9714A724BE6
:10584000019200221A80FEF78DBF704AB2F9003033
:10585000002BB8BF5B42B3F5E17FBFF6C6ABB2F930
:105860000230002BB8BF5B42B3F5E17FBFF6BDABA2
:10587000674B93ED057AD3ED077AD3ED096A93ED83
:10588000030A77EEA67A30EE070AF7EE000AB0EECA
:10589000007AE7EEC70A30EE000AF4F727FFBEEE03
:1058A000008A20EE088A9FED5B0A38EE000AFDEEC2
:1058B000C07A17EE903A2033402B40F2C5829FED1C
:1058C000560A564CDFED547A84ED010ABDEEC87AD3
:1058D000C4ED027A17EE103A2033402BC4ED037A60
:1058E00000F24C87B0EE480AF4F762F90A2084ED22
:1058F000040A21F08FFDFFF778BB24F040039BB230
:10590000A3423B803FF46AAB454B41F20241FF2288
:105910000E2019809A7021F07DFDFFF75FBB24F007
:1059200004039BB2A3423B803FF44EAB3C4B41F29D
:105930000241FF2219800E209A7021F06BFD3C88F5
:10594000FFF742BB44F40063A3423B807FF423ACE7
:10595000FFF70BBB9AF85336002B3FF4FEA9029BCE
:105960001B7813F001037FF4F8A901228AF853365B
:105970008AF85426FFF7F1B9204A052382F820302F
:10598000002F3FF4BDAC2FF0FBFC1C4A336852697A
:105990009A424FF0030BFFF4B9AC224B1B78002B5B
:1059A0007FF4B4AC002F3FF4B1AC002D3FF436AF20
:1059B000124B93F82030FFF767B998F80630012BA7
:1059C0007FF4EBAC2FF0F4FC0C4903224FF47A7314
:1059D00081F82020CB61A0E42EF068FF00283FF47E
:1059E000B7ACBBF1000F3EF4C8AE4EE544930408DB
:1059F000B87F0020D34D6210903E0020E07A002056
:105A000060E316007ABA002014380020747B00206E
:105A100070260020DB0FC93F00000000200000209E
:105A200094460020C6630020842B002008F1050165
:105A300068792FF04DFD00283FF4EAAB012F40F0CC
:105A4000D48605F10D01A87A2FF042FD002840F020
:105A50001187C149E87B2FF03BFD00283FF4E9ABFB
:105A6000032F40F00387BD49287D2FF031FD00282A
:105A700040F0F886BA49687E2FF02AFD00283FF4EE
:105A8000E9AB052F40F0EA86B649A87F2FF020FD4C
:105A9000002840F0DF86B44995F823002FF018FD68
:105AA00000283FF4E9AB072F40F0D086AF4995F8C6
:105AB00028002FF00DFD002840F0C486AC4995F871
:105AC0002D002FF005FD00283FF4E9AB092F3FF42E
:105AD000E6AB0926334603EB83031D44A54B6978E7
:105AE000AA78267519705A70FFF7D9BB01238AF876
:105AF0001831FEF75FBFC839884280F29A8532417B
:105B0000D1079B783FF5D9AD5A4201209DE5002C85
:105B10007FF493AA984C94F8DA30002B40F08B81F4
:105B200094F8B631002B40F07C8194F89232002B2F
:105B300040F06D8120F034FB01238AF8B636FFF780
:105B400077BA8E4A01239370FFF781B801990C2C24
:105B500031F912B09A7800F0D485BBF5617FC0F2BC
:105B6000418140F633018B45A8BF8B46182CABF51D
:105B7000617B4FF4966191FBF2F29BFBF2FB5FFAC3
:105B80008BFB1CD15A46C82AA8BFC822D1B27C4878
:105B9000006890F81CC08C4511D0B2EB0C02794B18
:105BA000017748BF0732D2109978531CDBB2002925
:105BB00040F04D8113B1184621F04CFD6B681B7805
:105BC0000C2B3FF473AD704B1C60704BC3F800B0EE
:105BD0006CE5022022F04CFF3C88FFF7BCB932682C
:105BE000B8F80230642101FB0323644A1361B9F160
:105BF000000F3FF4D2ABE0E6002D7FF4AEAB2BE418
:105C0000604D059BA97886F308065FFA86FB83F84A
:105C10000AB019B131460D202FF0B8FCBAF10D0FC2
:105C200006D0059BAA7883F809B0002A40F079864F
:105C3000534B18682CF0ECFD70E500215448F4F744
:105C400047FD002865D000238AF85136FDF704FF90
:105C5000FEF748BE44F04003A3423B807FF454AEBD
:105C6000FFF7BCB944F00403A3423B807FF45EAE6F
:105C7000FFF7AAB944F00103A3423B803FF463AAB3
:105C8000444B41F20241FF2219809A700E2021F00C
:105C9000C1FB3C8823B2FFF757BA3F483F49006831
:105CA000BAF94E46C56981FB05018911ED17681ADD
:105CB00000F5FF407F30844240F3C68438490978BC
:105CC0000029BAD05F2A00F03B856F2B7EF407AE27
:105CD000B4F5FA7FFFF63AA89AF85036002B7FF415
:105CE00035A8029A1278012112EA01048AF85016A6
:105CF00040F04885FDF7B0FE2A4B1B68002B3FF4AF
:105D000025A8294B294A8AF850461B680392FFF7B9
:105D100021B8029B234A1B78CAF84001DC071060B7
:105D200000F1D884204B1B68FEF7E2BD1221184811
:105D3000F4F7CEFC00283BD0002C7FF479A9E9E6EB
:105D40002FF036FB0D49032240F6B83381F82020AE
:105D5000CB61FFF7E2BA00BF563E00205B3E002059
:105D6000603E0020653E00206A3E00206F3E00201D
:105D7000743E0020D47A002034960020E07A00207F
:105D8000B87F0020B87D0020B4640020F00200201D
:105D9000903E002094460020A4830020D34D621042
:105DA00020000020D07D0020A0A000201C72002038
:105DB000002C3FF43DA920F0F3F921F09BFA0023D9
:105DC0008AF8B636FFF734B90021B948F4F780FCF9
:105DD00000287EF4A9AD32238AF85206AAF8563676
:105DE000FEF7A2BD182C40F0E7844FF0000B594697
:105DF0005A46CCE6F91A891AC3F5FA6364259B1A48
:105E000005FB01F595FBF3F5EDB2FEF7D1BCD4F837
:105E1000B80121F0C2F8DC220021A64831F02EFEA4
:105E200088E6D4F8DC0021F0B8F8DC220021A24892
:105E300031F024FE79E6206821F0AFF8DC22002161
:105E4000204631F01BFE6BE6F3F7B2FE39E559460A
:105E5000182006932FF09AFB069BABE6974DB6F5FC
:105E6000FA6F3146AA78A8BF4FF4FA6121EAE171CE
:105E70000183002A3FF4DEAE20202FF087FB904BF9
:105E80001868D7E605998D4B91F80BB09B78934431
:105E90008BF3080B81F80BB0002B40F04A85884B40
:105EA00018682CF0B5FC6B6889E60598834B90F870
:105EB0000AB0997893448BF3080B80F80AB039B193
:105EC00059460D20CDE906232FF060FBDDE90623BE
:105ED0000D2CE4D005999B7891F809B093448BF38D
:105EE000080B81F809B0002BD9D00E2059462FF0AD
:105EF0004DFB734B1868D4E7704D059BAA7886F369
:105F00000801D972002A3FF495AE05202FF03EFB20
:105F10006B4B18688EE6642EA8BF6426059B674D00
:105F200026EAE6765E702FF059FBAA78002A3FF445
:105F30007FAE032031462FF029FB614B186879E6CC
:105F4000642E5E4D059BA978A8BF642626EAE676F6
:105F50005FFA86FB83F806B019B131461B202FF09B
:105F600015FBBAF11B0F3FF463AE059BAA7883F8CB
:105F700007B0002A3FF45CAE1C2031462FF006FB30
:105F80004F4B186856E64D4D059BA97886F30806D9
:105F90005FFA86FB83F803B019B1314619202FF060
:105FA000F5FABAF1190F3FF443AE059BAA7883F8CE
:105FB00004B0002A3FF43CAE1A2031462FF0E6FA36
:105FC0003F4B186836E6B6F5FA6FA8BF4FF4FA668D
:105FD00026EAE676394D1FFA86FBAA78A0F80CB0BF
:105FE000002A3FF427AE1F2031462FF0CFFA344B62
:105FF00018681FE6642EA8BF642626EAE6765FFAD4
:1060000086FB2E4DB1E786F308065FFA86FB2B4D23
:10601000CBE7642E294D3146A8BF64210129AA7817
:10602000B8BF012180F84710002A3FF403AE1720C3
:106030002FF0ACFAFCE5B6F5FA6F204DA8BF4FF48F
:10604000FA6626EAE676A9781FFA86FBA0F812B06F
:1060500029B11E2031462FF099FA194B1868BAF170
:106060001E0FBAD1E6E5154D059BAA7886F3080107
:106070005971002A3FF4DEAD15202FF087FA104B3E
:106080001868D7E5C82EA8BFC82626EAE6760B4DC5
:106090005FFA86FBAA7880F80AB0002A3FF4CAADFE
:1060A000142031462FF072FA054B1868C2E500BF84
:1060B000903E0020EC97002010970020B87D002033
:1060C000B87F0020C82EA8BFC82626EAE676B54DC0
:1060D0005FFA86FBAA7880F809B0002A3FF4AAADDF
:1060E000132031462FF052FAAF4B1868A2E5C82EA4
:1060F000A8BFC82626EAE676AA4D5FFA86FBAA78EC
:1061000080F808B0002A3FF495AD122031462FF0F8
:106110003DFAA54B18688DE586F308065FFA86FB05
:10612000A04D7EE59F4DC82E3146AA78A8BFC82154
:1061300021EAE1718175002A3FF47CAD0B202FF03C
:1061400025FA994B186875E5964DC82E3146AA7800
:10615000A8BFC82121EAE1714175002A3FF46AAD68
:106160000A202FF013FA904B186863E58D4DC82E66
:106170003146AA78A8BFC82121EAE1710175002A39
:106180003FF458AD09202FF001FA874B186851E50C
:10619000C82E844DA8BFC82626EAE676A9785FFAFD
:1061A00086FB80F810B029B1112031462FF0EEF9AE
:1061B0007D4B1868BAF1110F7FF46CAF3AE5C82E29
:1061C000784DA8BFC82626EAE676A9785FFA86FB4E
:1061D00080F80FB029B1102031462FF0D7F9724B5B
:1061E0001868BAF1100F7FF475AF23E5C82E6D4D16
:1061F000A8BFC82626EAE676A9785FFA86FB80F86B
:106200000EB029B10F2031462FF0C0F9664B186847
:10621000BAF10F0F7FF473AF0CE50598614B90F85E
:1062200003B0997893448BF3080B80F803B039B12D
:1062300059461920CDE906232FF0A8F9DDE90623F8
:10624000192C3FF42CAE05999B7891F804B0934437
:106250008BF3080B81F804B0002B3FF420AE1A201A
:1062600059462FF093F9504B18681AE64E4B1868B0
:106270004C4BB0F818B09B789344BBF5FA6FA8BFAD
:106280004FF4FA6B2BEAEB7BA0F818B0002B3FF42D
:1062900008AE202059462FF079F9434B186800E6E4
:1062A000414B18683F4BB0F80CB09B789344BBF55A
:1062B000FA6FA8BF4FF4FA6B2BEAEB7BA0F80CB097
:1062C000002B3FF4EEAD1F2059462FF05FF9364BFF
:1062D0001868E6E5334B05999B7891F807B093442D
:1062E000BBF1640FA8BF4FF0640B2BEAEB7B81F886
:1062F00007B0002B3FF4D3AD1C2059462FF046F9D0
:10630000294B1868CDE5274B9DE7274B1868254B8F
:1063100090F847B09B789344BBF1640FA8BF4FF04F
:10632000640BBBF1010FB8BF4FF0010B80F847B011
:10633000002B3FF4B6AD594617202FF027F9AEE5F4
:10634000194B1868174BB0F812B099789344BBF505
:10635000FA6FA8BF4FF4FA6B2BEAEB7BA0F812B0F0
:1063600049B11E205946CDE906232FF00FF90E4BF7
:106370001868DDE906231E2C95D192E50599094B95
:1063800091F805B09B7893448BF3080B81F805B026
:10639000002B3FF484AD152059462FF0F7F8024B3F
:1063A00018687EE5B87D0020B87F0020AA4B1868E9
:1063B000AA4B90F80AB09B789344BBF1C80FA8BFD2
:1063C0004FF0C80B2BEAEB7B80F80AB0002B3FF4B0
:1063D00068AD142059462FF0D9F89F4B186860E536
:1063E0009D4B18689D4B90F809B09B789344BBF186
:1063F000C80FA8BF4FF0C80B2BEAEB7B80F809B0A1
:10640000002B3FF44EAD132059462FF0BFF8924BAE
:10641000186846E5904B1868904B90F808B09B7848
:106420009344BBF1C80FA8BF4FF0C80B2BEAEB7B1E
:1064300080F808B0002B3FF434AD122059462FF0FD
:10644000A5F8854B18682CE5844B43E5824B18680A
:10645000824B90F816B09B789344BBF1C80FA8BF4D
:106460004FF0C80B2BEAEB7B80F816B0002B3FF403
:1064700018AD0B2059462FF089F8774B186810E5B6
:10648000754B1868754B90F815B09B789344BBF129
:10649000C80FA8BF4FF0C80B2BEAEB7B80F815B0F4
:1064A000002B3FF4FEAC0A2059462FF06FF86A4BE0
:1064B0001868F6E4684B1868684B90F814B09B783D
:1064C0009344BBF1C80FA8BF4FF0C80B2BEAEB7B7E
:1064D00080F814B0002B3FF4E4AC092059462FF0AB
:1064E00055F85D4B1868DCE45B4B18685B4B90F823
:1064F00010B099789344BBF1C80FA8BF4FF0C80BF8
:106500002BEAEB7B80F810B049B111205946CDE958
:1065100006232FF03BF8504B1868DDE90623112CB9
:106520007FF447AFBDE44C4B18684C4B90F80FB06C
:1065300099789344BBF1C80FA8BF4FF0C80B2BEA62
:10654000EB7B80F80FB049B110205946CDE9062306
:106550002FF01CF8404B1868DDE90623102C7FF45F
:1065600042AF9EE43C4B18683C4B90F80EB09978D3
:106570009344BBF1C80FA8BF4FF0C80B2BEAEB7BCD
:1065800080F80EB049B10F205946CDE906232EF010
:10659000FDFF314B1868DDE906230F2C7FF43DAF7A
:1065A0007FE405992D4B91F801B006939344BBF11C
:1065B000640FA8BF4FF0640B2BEAEB7B81F801B0AE
:1065C0002FF00CF8069B9B78002B3FF468AC03205F
:1065D00059462EF0DBFF204B186862E405981F4BEC
:1065E00090F806B099789344BBF1640FA8BF4FF0C0
:1065F000640B2BEAEB7B80F806B039B159461B20BF
:10660000CDE906232EF0C2FFDDE906231B2C7FF423
:1066100062AE44E4104B18682CF0FAF84FF0FF3BE0
:10662000FFF744B82EF0C4FE0D4B93F82030FEF770
:106630002BBB0123B34022EA030209F5FA738AF85F
:106640009426AB60FFF739B8491B0C4424B2AAF872
:106650004E46FFF733BB00BFB87F0020B87D002057
:10666000E07A0020C44A116811F020017EF448A9A4
:106670009AF84D260120572A8AF8500600F0FE802D
:106680005B0702D55A2A00F09D825D2A00F09F81A7
:106690005E2A00F09A815B2A00F08E81562A00F073
:1066A000B081972A3EF44EABA72A00F02F823B8898
:1066B0009E0740F01182A2F1B703072B00F2A681DA
:1066C000DFE813F0A002A401A401A4019E02A4012A
:1066D0009C029302A94B1B78002B3EF437ABA84BCE
:1066E000DB78002B7EF432AB9AF851360133DBB203
:1066F000032B8AF851367EF629ABF9F715FAFEF727
:10670000F1B8A0490879002851D0C822BBF5617FB3
:1067100040DA4FF0000B5A46497891423FF44FAAB5
:10672000994B079310460692FDF7EEFF079B069ADA
:106730009B78002B40F0CF80531CDBB2FFF73ABAB6
:10674000B4F5FA7FFEF602AB9AF85036002B7EF4D1
:10675000FDAA029A8D4912780B60012312EA030404
:106760008AF850362CD0F9F7DFF9894B0393894B1F
:106770001B68FEF7EFBA6425FEF71AB8B0EE670A99
:10678000FFF7B4B8CAF84031824B814A1B680392C4
:10679000FEF7E0BA40F633008345A8BF8346ABF569
:1067A000617B9BFBF2FB5FFA8BFB5A46B4E74FF42D
:1067B000966090FBF2F2A9E74FF0000BFFF7FFB9EC
:1067C0000F2020F027FE6C49BAF84E360A688AF886
:1067D0005046FA3B22F02002AAF84E366D4B0A6072
:1067E0006B4A1B680392FEF7B5BA01263346FFF7E2
:1067F00072B904932EF002FA049B00287EF401A9DA
:10680000B8F1000F7EF4FDA8039A2AB1DAF84831F6
:106810009B1A2344CAF848310023CAF844315E4B1E
:106820009FED5E7A5B78202F07EE903A00F089802A
:10683000F8EEE77A67EE877AFCEEE77A17EE905A81
:10684000FEF7A1B908263346FFF745B907263346B8
:10685000FFF741B906263346FFF73DB90526334613
:10686000FFF739B904263346FFF735B90326334617
:10687000FFF731B902263346FFF72DB94849494A97
:106880008C8B4949106842F2107202FB04F2B2FB91
:10689000F0F2C1F8B020190603D516F015FF3D4BF4
:1068A0001B683B4A0392126852077EF553AA0A22DC
:1068B000AAF8C620FEF74EBA31493268CB691344B4
:1068C0008B61BBF1000F3DF458AFFEF7DEBD22F047
:1068D000B7F8FEF7A0BF59460C202EF057FE069AD7
:1068E0002AE7B8F1000F3EF474A99AF84C36002B51
:1068F0003DF4A4AF20F074FD00238AF84C36FDF778
:106900009DBFACEB0E0191427EF7A7A8881A6422C6
:10691000A1F57A7102FB00F292FBF1F2D2B2FEF71E
:106920009AB80E2031462EF031FE204B1868FFF742
:1069300081B9052059462EF029FE1C4B1868FFF737
:10694000B0BA1B4ADAF848311A49F8EEE77AA2FBE6
:106950000323029A67EE877A12789B09FCEEE77AA6
:10696000CB8002F00102002317EE905A8B80002AA0
:106970003DF460AFFEF7E3B9887D0020C54D0020EF
:10698000E07A0020D8980020B87D0020D07D00203B
:106990001C720020A0A00020DC3E002000247449CE
:1069A00070A0002090A00020E8990020B87F00206F
:1069B000D34D6210E884002001200AF0E3FF974BDA
:1069C0000393974B1B68FEF7C5B90220F5E7954A7C
:1069D000954B9648106000221A702CF0E1F80120C7
:1069E00020F038FE8D4B03938D4B1B68FEF7B2B938
:1069F0009AF84C362C44CAF83C41002B3DF41EAFAB
:106A000078E70CF071FE9AF84D264AE6792A5DD0B7
:106A10007A2A37D09E2A03D10021012030F0ACFF22
:106A20009AF84D369D2B03D10021FF2030F0A4FFB2
:106A30009AF84D36AE2B03D10121002030F09CFF97
:106A40009AF84D36AD2B03D1FF21002030F094FF92
:106A50009AF84D36EF2B36D0FD2B31D0FB2B2CD0B6
:106A6000FE2B27D0F72B13D07B2B7EF46FA94FF48E
:106A7000FA610220FDF7D2FD684B0393684B1B6857
:106A8000FEF768B96A4A137A43F001031372CFE73D
:106A900000210420FDF7C2FDBAF84E26604B5F4985
:106AA0001B680391963AAAF84E2600228AF85026CF
:106AB000FEF750B900210320ECE700210220E9E7AE
:106AC00000210120E6E700210846E3E7584A137A4F
:106AD00023F001031372A3E70021A2F1B7030C9185
:106AE000072B93D801A151F823F000BF6D6B01086B
:106AF0000D6A01080D6A01080D6A0108656B01083D
:106B00000D6A01085B6B01081F6B01084949444B82
:106B10000A781B6842F004020A70FDF7F1BE0223F6
:106B2000ADF83030444BBDF830409989DA89BDF872
:106B30003200214402449981DA810CF0D5FDBAF883
:106B40004E263649364B0391FA3A00211B68AAF8C3
:106B50004E268AF85016FEF7FDB84FF6FE73ADF8D4
:106B60003030DFE70223ADF83230DBE74FF6FE735B
:106B7000ADF83230D6E7ACEB090C6245BDF6A7AFF5
:106B8000ACEB02026421ACF57A7C01FB02F292FBD1
:106B9000FCF2D2B2FDF799BFACEB0E0191427DF74A
:106BA00078AF881A6422A1F57A7102FB00F292FB99
:106BB000F1F2D2B2FDF76BBFF8F7B6FF8AF84C8658
:106BC000FDF73CBE9AF853269AF85236F2B983F094
:106BD00001038AF85236BBB90C2020F01BFC0F4B86
:106BE00003930F4B1B68FEF7B5B80220FDF78CFD31
:106BF0000A4B03930A4B1B68FEF7ACB80320F5E77A
:106C00000020F3E70120F1E70B20E6E7034B8AF8C9
:106C100053168AF854060393FDF777BE1C720020C2
:106C2000A0A00020B87F0020D89800203C5D002064
:106C300024620020A87D0020783B00201F4B18789C
:106C400010B31F4A138903B31E4A9FED1F6AD2ED8A
:106C5000026A07EE903AF8EEE66AF8EE677A07EE17
:106C6000103A77EEE66AB8EEC77A66EE866AC6EE46
:106C7000877AFDEEE77A17EE900A6428A8BF6420B1
:106C800020EAE070C0B27047704710B40F4B5478E0
:106C90001B88117804FB1032091B642300FB01F0F0
:106CA00003FB02F3B3FBF0F06428A8BF642020EAE2
